S01700005354345F52433030375F35385350322E7372656306
S315080080000000022011FF020861FF020861FF020852
S3150800801061FF020861FF020861FF02080000000014
S3150800802000000000000000000000000061FF0208D8
S3150800803061FF02080000000061FF020811FE020845
S3150800804061FF020861FF020861FF020861FF02087A
S3150800805061FF020861FF020861FF020861FF02086A
S3150800806061FF020861FF020861FF020861FF02085A
S3150800807061FF020861FF020861FF020861FF02084A
S3150800808081FE020895FE020861FF020861FF0208E8
S3150800809061FF020861FF020861FF02081DFE02086F
S315080080A061FF020861FF020861FF020861FF02081A
S315080080B0C9FE0208E1FE020861FF020861FF020824
S315080080C061FF020861FF020861FF020861FF0208FA
S315080080D061FF020861FE020871FE020861FF0208DC
S315080080E049FE020861FF020861FF020861FF0208F3
S315080080F061FF020861FF020861FF020861FF0208CA
S3150800810061FF020809FF020861FF020861FF020811
S3150800811061FF020861FF020861FF020861FF0208A9
S3150800812061FF020861FF0208A5FE0208F9FE0208BF
S3150800813061FF0208000000000000000061FF02085D
S3150800814061FF020861FF020861FF020861FF020879
S3150800815061FF020801FF0208B9FE020861FF020872
S3150800816061FF020861FF020861FF020861FF020859
S3150800817061FF020861FF020861FF020800000000B3
S315080081800000000061FF0208000000000000000077
S3150800819061FF0208000000000000000061FF0208FD
S315080081A000000000000000000000000061FF020857
S315080081B061FF020861FF020861FF020861FF020809
S309080081C061FF020843
S315080081D010B5054C237833B9044B13B10448AFF3F3
S315080081E000800123237010BDF8090020000000005C
S315080081F0383B030808B5034B1BB103490348AFF3E3
S31508008200008008BD00000000FC090020383B030878
S3150800821081F0004102E000BF83F0004330B54FEA29
S3150800822041044FEA430594EA050F08BF90EA020F96
S315080082301FBF54EA000C55EA020C7FEA645C7FEA29
S31508008240655C00F0E2804FEA5454D4EB5555B8BF4C
S315080082506D420CDD2C4480EA020281EA030382EABD
S31508008260000083EA010180EA020281EA0303362D4F
S3150800827088BF30BD11F0004F4FEA01314FF4801C22
S315080082804CEA113102D0404261EB410113F0004F34
S315080082904FEA03334CEA133302D0524263EB4303EB
S315080082A094EA050F00F0A780A4F10104D5F1200E89
S315080082B00DDB02FA0EFC22FA05F2801841F10001E4
S315080082C003FA0EF2801843FA05F359410EE0A5F1B8
S315080082D020050EF1200E012A03FA0EFC28BF4CF0E9
S315080082E0020C43FA05F3C01851EBE37101F000459F
S315080082F007D54FF0000EDCF1000C7EEB00006EEBAC
S315080083000101B1F5801F1BD3B1F5001F0CD3490835
S315080083105FEA30004FEA3C0C04F101044FEA44528C
S3150800832012F5800F80F09A80BCF1004F08BF5FEA13
S31508008330500C50F1000041EB045141EA050130BDF3
S315080083405FEA4C0C404141EB010111F4801FA4F196
S315080083500104E9D191F0000F04BF01460020B1FAEB
S3150800836081F308BF2033A3F10B03B3F120020CDA23
S315080083700C3208DD02F1140CC2F10C0201FA0CF001
S3150800838021FA02F10CE002F11402D8BFC2F1200C66
S3150800839001FA02F120FA0CFCDCBF41EA0C0190401C
S315080083A0E41AA2BF01EB0451294330BD6FEA040465
S315080083B01F3C1CDA0C340EDC04F11404C4F1200250
S315080083C020FA04F001FA02F340EA030021FA04F362
S315080083D045EA030130BDC4F10C04C4F1200220FAB9
S315080083E002F001FA04F340EA0300294630BD21FAF7
S315080083F004F0294630BD94F0000F83F4801306BFBD
S3150800840081F480110134013D4EE77FEA645C18BFB0
S315080084107FEA655C29D094EA050F08BF90EA020F47
S3150800842005D054EA000C04BF1946104630BD91EA3F
S31508008430030F1EBF0021002030BD5FEA545C05D142
S315080084404000494128BF41F0004130BD14F5800481
S315080084503CBF01F5801130BD01F0004545F0FE41F5
S3150800846041F470014FF0000030BD7FEA645C1ABF2A
S31508008470194610467FEA655C1CBF0B46024650EA61
S31508008480013406BF52EA033591EA030F41F400218D
S3150800849030BD00BF90F0000F04BF0021704730B513
S315080084A04FF4806404F132044FF000054FF00001E8
S315080084B050E700BF90F0000F04BF0021704730B5A9
S315080084C04FF4806404F1320410F0004548BF40427E
S315080084D04FF000013EE700BF42004FEAE2014FEAD3
S315080084E031014FEA02701FBF12F07F4393F07F4FAE
S315080084F081F06051704732F07F4208BF704793F0B1
S315080085007F4F04BF41F40021704730B54FF46074C3
S3150800851001F0004521F000411CE700BF50EA0102C6
S3150800852008BF704730B54FF000050AE050EA01026F
S3150800853008BF704730B511F0004502D5404261EBDF
S3150800854041014FF4806404F132045FEA915C3FF420
S31508008550D8AE4FF003025FEADC0C18BF03325FEABD
S31508008560DC0C18BF033202EBDC02C2F1200300FA6E
S3150800857003FC20FA02F001FA03FE40EA0E0021FA93
S3150800858002F11444BDE600BF70B54FF0FF0C4CF481
S31508008590E06C1CEA11541DBF1CEA135594EA0C0F33
S315080085A095EA0C0F00F0DEF82C4481EA030621EA6E
S315080085B04C5123EA4C5350EA013518BF52EA0335A9
S315080085C041F4801143F4801338D0A0FB02CE4FF05B
S315080085D00005E1FB02E506F00042E0FB03E54FF08B
S315080085E00006E1FB03569CF0000F18BF4EF0010E83
S315080085F0A4F1FF04B6F5007F64F5407404D25FEA7F
S315080086004E0E6D4146EB060642EAC62141EA555131
S315080086104FEAC52040EA5E504FEACE2EB4F1FD0C73
S3150800862088BFBCF5E06F1ED8BEF1004F08BF5FEAF1
S31508008630500E50F1000041EB045170BD06F00046A3
S3150800864046EA010140EA020081EA0301B4EB5C0450
S31508008650C2BFD4EB0C0541EA045170BD41F4801148
S315080086604FF0000E013C00F3AB8014F1360FDEBF6D
S31508008670002001F0004170BDC4F10004203C35DA49
S315080086800C341BDC04F11404C4F1200500FA05F3CC
S3150800869020FA04F001FA05F240EA020001F000426D
S315080086A021F0004110EBD37021FA04F642EB0601E3
S315080086B05EEA430E08BF20EAD37070BDC4F10C040D
S315080086C0C4F1200500FA04F320FA05F001FA04F2D1
S315080086D040EA020001F0004110EBD37041F10001BD
S315080086E05EEA430E08BF20EAD37070BDC4F12005C8
S315080086F000FA05F24EEA020E20FA04F301FA05F230
S3150800870043EA020321FA04F001F0004121FA04F2D7
S3150800871020EA020000EBD3705EEA430E08BF20EAA7
S31508008720D37070BD94F0000F0FD101F000464000E1
S3150800873041EB010111F4801F08BF013CF7D041EA63
S31508008740060195F0000F18BF704703F00046520067
S3150800875043EB030313F4801F08BF013DF7D043EA38
S315080087600603704794EA0C0F0CEA135518BF95EAEE
S315080087700C0F0CD050EA410618BF52EA4306D1D175
S3150800878081EA030101F000414FF0000070BD50EA94
S31508008790410606BF1046194652EA430619D094EA1E
S315080087A00C0F02D150EA013613D195EA0C0F05D108
S315080087B052EA03361CBF104619460AD181EA03015C
S315080087C001F0004141F0FE4141F470014FF0000014
S315080087D070BD41F0FE4141F4780170BD70B54FF0AF
S315080087E0FF0C4CF4E06C1CEA11541DBF1CEA13552F
S315080087F094EA0C0F95EA0C0F00F0A7F8A4EB050411
S3150800880081EA030E52EA03354FEA013100F0888007
S315080088104FEA03334FF0805545EA131343EA1263D0
S315080088204FEA022245EA111545EA10654FEA002685
S315080088300EF000419D4208BF964244F1FD0404F53E
S31508008840407402D25B084FEA3202B61A65EB03059A
S315080088505B084FEA32024FF480104FF4002CB6EB57
S31508008860020E75EB030E22BFB61A754640EA0C00D7
S315080088705B084FEA3202B6EB020E75EB030E22BF17
S31508008880B61A754640EA5C005B084FEA3202B6EB58
S31508008890020E75EB030E22BFB61A754640EA9C0017
S315080088A05B084FEA3202B6EB020E75EB030E22BFE7
S315080088B0B61A754640EADC0055EA060E18D04FEAA5
S315080088C0051545EA16754FEA06164FEAC30343EA45
S315080088D052734FEAC2025FEA1C1CC0D111F4801F12
S315080088E00BD141EA00014FF000004FF0004CB6E70B
S315080088F011F4801F04BF01430020B4F1FD0C88BFAA
S31508008900BCF5E06F3FF6AFAEB5EB030C04BFB6EBB4
S31508008910020C5FEA500C50F1000041EB045170BDA7
S315080089200EF0004E4EEA113114EB5C04C2BFD4EBD4
S315080089300C0541EA045170BD41F480114FF0000E58
S31508008940013C90E645EA060E8DE60CEA135594EAD4
S315080089500C0F08BF95EA0C0F3FF43BAF94EA0C0FD7
S315080089600AD150EA01347FF434AF95EA0C0F7FF44C
S3150800897025AF104619462CE795EA0C0F06D152EAA0
S3150800898003353FF4FDAE1046194622E750EA410684
S3150800899018BF52EA43067FF4C5AE50EA41047FF495
S315080089A00DAF52EA43057FF4EBAE12E74FF0FF3CFA
S315080089B006E000BF4FF0010C02E000BF4FF0010CCB
S315080089C04DF804CD4FEA410C7FEA6C5C4FEA430C44
S315080089D018BF7FEA6C5C1BD001B050EA410C0CBF93
S315080089E052EA430C91EA030F02BF90EA020F0020F5
S315080089F0704710F1000F91EA030F58BF994208BF5C
S31508008A0090422CBFD8176FEAE37040F00100704718
S31508008A104FEA410C7FEA6C5C02D150EA013C07D16F
S31508008A204FEA430C7FEA6C5CD6D152EA033CD3D0BA
S31508008A305DF8040B704700BF8446104662468C46B4
S31508008A401946634600E000BF01B5FFF7B7FF0028E7
S31508008A5048BF10F1000F01BD4DF808EDFFF7F4FF10
S31508008A600CBF012000205DF808FB00BF4DF808ED9B
S31508008A70FFF7EAFF34BF012000205DF808FB00BFBE
S31508008A804DF808EDFFF7E0FF94BF012000205DF8E0
S31508008A9008FB00BF4DF808EDFFF7CEFF94BF012095
S31508008AA000205DF808FB00BF4DF808EDFFF7C4FF8E
S31508008AB034BF012000205DF808FB00BF4FEA410CD7
S31508008AC07FEA6C5C02D150EA013C0AD14FEA430CBA
S31508008AD07FEA6C5C02D152EA033C02D14FF00000F7
S31508008AE070474FF0010070474FEA410212F5001235
S31508008AF015D211D56FF47873B3EB625212D94FEAD7
S31508008B00C12343F0004343EA505311F0004F23FAC0
S31508008B1002F018BF404270474FF00000704750EA15
S31508008B20013005D111F0004008BF6FF000407047D2
S31508008B304FF00000704700BF4A0011D212F500122C
S31508008B4011D20DD56FF47873B3EB62520ED44FEA97
S31508008B50C12343F0004343EA505323FA02F0704717
S31508008B604FF00000704750EA013002D14FF0FF3055
S31508008B7070474FF0000070474FEA4102B2F1E043F8
S31508008B8024BFB3F5001CDCF1FE5C0DD901F0004CE6
S31508008B904FEAC0024CEA5070B2F1004F40EB830036
S31508008BA008BF20F00100704711F0804F21D113F162
S31508008BB03872BCBF01F00040704741F480114FEA9B
S31508008BC05252C2F11802C2F1200C10FA0CF320FA24
S31508008BD002F018BF40F001004FEAC1234FEAD32341
S31508008BE003FA0CFC40EA0C0023FA02F34FEA4303AB
S31508008BF0CCE77FEA625307D150EA01331EBF4FF034
S31508008C00FE4040F44000704701F0004040F0FE404E
S31508008C1040F40000704700BF034613F8012B002AF2
S31508008C20FBD1181A01387047000000000000000048
S31508008C3001F0FF01102A2BDB10F0070F08D010F8FF
S31508008C40013B013A8B422DD010F0070F42B3F6D103
S31508008C50F0B441EA012141EA014122F007047FF01C
S31508008C6000070023F0E80256083C85EA010586EA73
S31508008C70010685FA47F5A3FA87F586FA47F6A5FAAF
S31508008C8087F68EB9EED1F0BC01F0FF0102F00702BB
S31508008C9032B110F8013B013A83EA010313B1F8D166
S31508008CA00020704701387047002D06BF3546033847
S31508008CB0073815F0010F07D1013015F4807F02BF80
S31508008CC0013015F4C03F0130F0BC0138704700BFD1
S31508008CD070470120704790F85000704790F8790067
S31508008CE07047E02914BF00200120704740F65C2336
S31508008CF0994209D043690BB9038BD3B140F24C535F
S31508008D00994208D00020704742F2E810824214BF08
S31508008D10002001207047B2F51A7F0CD040F22F438D
S31508008D209A420AD040F2D530824214BF0020012070
S31508008D307047002070470120704701207047019A4C
S31508008D40C3BB80F85D10D37803F00301032920D054
S31508008D5013F0020F2ED092F90230002BB4BF022373
S31508008D60032303EB43030344917801F00F0183F8CF
S31508008D705110918883F85210937990F878209A4286
S31508008D8038BF80F8783090F85E30013380F85E306E
S31508008D90704792F90210002904DB13F0020F09D07C
S31508008DA00323DEE790F85610012363F3870180F862
S31508008DB05610D6E77047A0F10400FFF7C0BFF8B514
S31508008DC004460146002210464FF0080E4FF00F0CDD
S31508008DD00127134681F8510012F0FF0F36D081F8AB
S31508008DE0520081F853003E4603EB4303234493F8AD
S31508008DF0535066F3870583F8535001320331042A2A
S31508008E00E7D104F1640504F1740601E0B54207D020
S31508008E1055F8040B0028F9D003689B689847F5E7CE
S31508008E20002384F8413084F8423084F8463084F8C8
S31508008E30473084F87C3084F85030012284F85E206C
S31508008E40236684F8783084F87930F8BD81F852E0E2
S31508008E5081F853006646C7E738B504461A4B03F14E
S31508008E60080202603C334360002380F8413080F8F2
S31508008E70433080F8463080F84830C16480F8503076
S31508008E80012280F85E20036680F8783080F8793011
S31508008E9043668366C3660367FFF791FFE56C85B192
S31508008EA0AB6F53B105F178020123184652F8041F37
S31508008EB021B10133102BF8D103E000201E3045F80C
S31508008EC02040204638BD00BF503B03082DE9F04737
S31508008ED088B00446884691469A46FFF770FF94F88C
S31508008EE05030002B40D1E66C33681B6800213046B1
S31508008EF09847054600283CD00768002F3BD004F168
S31508008F005103036080F806A003AB009312230022E6
S31508008F101146E06C02F0F8FB2F60054640B10D28BB
S31508008F200CBF0546E12523689B68204698471CE048
S31508008F3033685D684B46002241463046A84784F8A8
S31508008F405000D0B19DF8133084F852309DF81D308A
S31508008F5084F85430BDF81430A4F87630BDF81630CD
S31508008F60A4F87430E02500E0D925284608B0BDE805
S31508008F70F087D625F9E7D725F7E7D425F5E710B51D
S31508008F800446FFF71CFFE06C03689B6894F85010D2
S31508008F909847002010BDF0B585B0044604AB4022C2
S31508008FA023F8022D00F1C90690F8572090F85010C2
S31508008FB090F8780001900096E06C02F0ACF918B1D0
S31508008FC004F16405743415E0BDF80E30002BF7D0B3
S31508008FD004F1640504F1740701E0BD42F0D055F8C8
S31508008FE0040B0028F9D003681B6831469847F4E754
S31508008FF0A54207D055F8040B0028F9D003685B682A
S315080090009847F5E705B0F0BD30B589B0B0F88630B9
S3150800901023F00103A0F8863090F8515090F850409C
S31508009020C06C00230793069105920492039302935A
S315080090300193009320232A46214602F0ADFA09B08F
S3150800904030BD10B501460023A0F88630032280F80B
S3150800905089200C2480F88A4080F88B308931FFF704
S31508009060D3FF10BD08B5B0F8863023F01003A0F87A
S3150800907086301A2380F889300C2380F88A30012339
S3150800908080F88B30C36843B1032380F88C30042200
S3150800909000F18901FFF7B8FF08BD022380F88C307C
S315080090A0F5E708B50146B0F8863023F02003A0F8A6
S315080090B08630092380F88930102380F88A30002307
S315080090C080F88B3003228931FFF79EFF08BD08B56B
S315080090D00146B0F8863023F04003A0F88630012315
S315080090E080F88930102380F88A30002380F88B3086
S315080090F003228931FFF788FF08BD08B50146B0F895
S31508009100863023F00203A0F88630092380F88930D8
S31508009110042380F88A30072380F88B30037F80F891
S315080091208C30437F80F88D30837F80F88E30C37F04
S3150800913080F88F3090F8203080F8903090F8213001
S3150800914080F89130002380F892300A228931FFF79F
S315080091505BFF08BD08B50146B0F8863023F0080362
S31508009160A0F88630192380F88930042380F88A30DD
S315080091700A2380F88B30037F80F88C30437F80F891
S315080091808D30837F80F88E30C37F80F88F3090F8DB
S31508009190203080F8903090F8213080F89130012303
S315080091A080F89230002380F8933080F8943080F865
S315080091B095300D228931FFF727FF08BDF8B5074618
S315080091C00E46132380F889300C2380F88A30084627
S315080091D0FFF722FD013087F88B000024E5B2304600
S315080091E0FFF71AFD631CA84206D9725D57FA84F484
S315080091F084F88C201C46F1E757FA84F4002384F897
S315080092008C303046FFF708FD021D92B207F189013E
S315080092103846FFF7F9FEF8BD08B50146B0F88630BE
S3150800922023F08003A0F88630012380F889300423D0
S3150800923080F88A30052380F88B30332380F88C3009
S315080092408B2380F88D309E2380F88E30302380F86B
S315080092508F300A2380F8903008228931FFF7D4FE30
S3150800926008BD08B50146022380F88930042380F832
S315080092708A30002380F88B3003228931FFF7C4FE39
S3150800928008BD08B5B0F8862022F48172A0F88620B9
S31508009290052280F88920042280F88A200D2280F889
S315080092A08B200A7880F88C204A7880F88D208A7876
S315080092B080F88E20CA7880F88F200A7980F8902066
S315080092C04A7980F89120182280F89220CC2280F8DA
S315080092D09320012280F89420002280F8952080F8B7
S315080092E0962080F8972080F89820102200F18901AE
S315080092F0FFF78AFE08BD08B500F11C01FFF7C1FF9C
S3150800930008BD2DE9F04104460D2380F88930042371
S3150800931080F88A30172380F88B30037F80F88C30EA
S31508009320437F80F88D30837F80F88E30C37F80F846
S315080093308F3090F8203080F8903090F8213080F8FF
S31508009340913090F843306BB3062380F8923090F84A
S315080093507A30DBB100F1140300F193021A3013F8E6
S31508009360011B02F8011B8342F9D104F1980304F1A9
S31508009370A201002203F8012F9942FBD11A2204F117
S3150800938089012046FFF740FEBDE8F08100F11C0385
S3150800939000F19302223013F8011B02F8011B8342E5
S315080093A0F9D1E2E707693846FFF736FC84F89200F8
S315080093B00025EEB2B0463846FFF72EFC6B1CB042CD
S315080093C006D9BA5D54FA85F585F893201D46F0E767
S315080093D00F2ED3D806F19203234404F19302904446
S315080093E0C6F10F0658FA86F6002203F8012FB34293
S315080093F0FBD1C3E708B501460E2380F8893004235C
S3150800940080F88A30062380F88B30037F80F88C300A
S31508009410437F80F88D30837F80F88E30C37F80F855
S315080094208F3090F8203080F8903090F8213080F80E
S31508009430913009228931FFF7E7FD08BD08B50146D5
S315080094400C2380F88930042380F88A30062380F8B4
S315080094508B30037F80F88C30437F80F88D30837F94
S3150800946080F88E30C37F80F88F3090F8203080F8EF
S31508009470903090F8213080F8913009228931FFF731
S31508009480C3FD08BDF0B585B0044604AB402223F8F9
S31508009490022D90F8542090F8501090F8780001901A
S315080094A004F189000090E06C01F035FF10F0FB0034
S315080094B068D194F88930013B162B63D8DFE813F09E
S315080094C045006400D6001D01F1005A01FF00620044
S315080094D062006200620062006200170062006200B9
S315080094E0620062006200620062004501560194F85B
S315080094F08E30002B46D1B4F8862042F00103A4F83A
S315080095008630B4F88C3041F201018B4214D041F216
S3150800951009018B4236D104F1140304F18F0104F1D9
S315080095201A0511F8010B03F8010BAB42F9D142F009
S315080095302102A4F8862025E094F88F3084F840307C
S3150800954042F04102A4F886201CE094F88830042BE7
S3150800955013D994F8433013B994F848306BB1002303
S3150800956084F8883084F8413084F8433084F84630EB
S3150800957084F848300A2384F8803094F88830013318
S3150800958084F8883005B0F0BD94F88B70002FF9D0B8
S31508009590FB00DBB294F843C02EE084F87E1084F812
S315080095A07D60002384F87F30012384F87B3000EB4C
S315080095B0400004EB40028C3204F11C0304F1220043
S315080095C012F8011B03F8011B8342F9D1B4F886305F
S315080095D043F08003A4F88630D4E794F848502DB1B8
S315080095E011F0050F02D016F0C80F1CD10130C0B219
S315080095F00333DBB2874232D0E21892F88D6092F8D4
S315080096008E1092F88F20BCF1000FE6D0002AE4D124
S3150800961011F0050FEAD016F00C0FBED194F8485099
S31508009620002DE0D1E2E784F87E1084F87D6084F8A6
S315080096307F2000EB400004EB40038C3304F11C024E
S3150800964004F1220013F8011B02F8011B8242F9D12A
S31508009650B4F8863043F08003A4F8863092E784F89D
S315080096607E1084F87D6084F87F208BE7B4F8863016
S3150800967043F48072A4F8862094F88B206AB994F88B
S315080096808D20120202F4706294F88C100A436283E9
S3150800969043F48173A4F8863074E7062384F880308F
S315080096A070E794F88B30002B7FF46CAFB4F88630F3
S315080096B023F0020343F00403A4F8863062E794F823
S315080096C08B30002B7FF45EAF94F8923084F822300A
S315080096D063B104F1220304F1920104F13F0011F889
S315080096E0012F03F8012F0AB18342F8D1B4F8863066
S315080096F043F00803A4F8863044E704F11C0304F198
S315080097008B0204F1220012F8011B03F8011B8342A5
S31508009710F9D194F8912084F87D2094F8923084F851
S315080097207E3094F8931084F87F1013F0050F05D057
S3150800973012F0C80F1CBF012384F84730B4F88630EE
S3150800974043F01003A4F886301CE794F843302BB98D
S3150800975023693BB12046FFF7D4FD13E72046FFF700
S31508009760D0FD0FE72046FFF745FE0BE72046FFF73B
S3150800977065FE07E794F8433013B194F841306BB1AE
S3150800978094F84830002B3FF4FDAE94F84630002B91
S315080097907FF4F8AE012384F84630F3E6012384F813
S315080097A04130EFE608B50146112380F889300423D5
S315080097B080F88A30022380F88B30438B80F88C300F
S315080097C0C3F3032380F88D3005228931FFF71CFC8B
S315080097D008BD10B5B0F8862022F00402A0F886204D
S315080097E0062280F88920042480F88A40032480F819
S315080097F08B4080F88C10C1F3032180F88D1013215B
S3150800980080F88E1000F18901FFF7FEFB10BD08B540
S315080098100146242380F889300C2380F88A300323F4
S3150800982080F88B30042380F88C30082380F88D303C
S31508009830002380F88E3006228931FFF7E5FB08BD44
S3150800984070B5044690F88030102B1CD8DFE813F06A
S31508009850110025004E005900640075007E008F0037
S31508009860A400B300C500E100F60052011B00680120
S315080098707901B0F8823001339BB2A0F88230B0F893
S3150800988084209A4200D370BDFFF7DBFB012384F8DE
S3150800989080300023A4F88230F5E7B0F8823001332F
S315080098A09BB2A0F88230B0F8862012F0010F14D1CE
S315080098B0B0F884209342E6D902EB82035B009BB2A0
S315080098C0B3F5FA6F88BF4FF4FA63A0F88430002323
S315080098D080F88030A0F88230D5E70023A0F88230DF
S315080098E0022380F88030FFF792FFCCE7B0F8863085
S315080098F013F0010FC7D0032380F88030FFF7D1FBA0
S31508009900C1E7B0F8863013F0200FBCD0FFF7DFFBB5
S31508009910042384F88030B6E7B0F8863013F0400F99
S31508009920B1D0C16829B1FFF749FC052384F8803016
S31508009930A9E7062380F88030A5E7B0F8863013F04B
S31508009940010FA0D0062380F880309CE790F84830B5
S3150800995013B990F8433033B12046FFF75DFC07236F
S3150800996084F880308FE70A2380F880308BE7B0F8D8
S31508009970863013F0800F86D0FFF773FC94F87B309F
S315080099801BB9082384F880307DE72046FFF7E2FB01
S315080099900C2384F8803076E7B0F8863013F0010F90
S315080099A03FF471AF002380F87B30FFF7A4FC09234E
S315080099B084F8803067E7B0F8863013F4807F3FF488
S315080099C062AF13F0020F05D0FFF7ECFE0A2384F806
S315080099D0803058E7FFF78FFC55E790F84130002BA9
S315080099E07FF451AF90F84330002B7FF44CAF90F8DA
S315080099F04630002B7FF447AF90F84830002B7FF4B1
S31508009A0042AFFFF72FFB012323720B2384F8803024
S31508009A1039E7B0F8863013F0100F07D113F0040FAA
S31508009A203FF431AF102380F880302CE7002303720F
S31508009A30FFF790FB0C2384F8803024E7B0F88630D3
S31508009A4013F0080F3FF41FAF00F122050822514911
S31508009A50284627F05EFF90B9012384F84230002398
S31508009A6084F8443084F8453084F87A3016224A4916
S31508009A70284627F04EFF90B9012384F84430E36F57
S31508009A8023F0FF03454A934222D094F8433053B358
S31508009A9094F87B303BB3082384F88030F3E616222B
S31508009AA03F49284627F035FF38B9012384F87A302C
S31508009AB084F8443084F84530E1E7132239492846CA
S31508009AC027F027FF0028DAD1012384F87A30D6E771
S31508009AD013223549284627F01CFF0028D5D1012333
S31508009AE084F87C30D1E72046FFF707FB0D2384F87E
S31508009AF08030C8E6B0F8863013F0020F3FF4C3AEE4
S31508009B0090F87C3013B1012380F846300023637245
S31508009B10A372E372A4F886300F2384F88030B2E685
S31508009B20B0F8823001339BB2B3F57A7F02D8A0F839
S31508009B308230A8E60023A0F882300A2380F8803015
S31508009B40A1E6B0F8863013F0040F3FF49CAE00256A
S31508009B50A0F88650402632462946893027F0A0FDCF
S31508009B603246294604F1C90027F09AFD84F8435085
S31508009B7084F8425084F8415084F87B5084F8485061
S31508009B8084F8475084F8465084F87C500A2384F8B1
S31508009B90803078E6ACBA0308B8BA0308000825008E
S31508009BA0D0BA0308E8BA0308FCBA030890F8793073
S31508009BB00BB90020704710B5044605F057FD236E13
S31508009BC0C01A00280EDB05F051FD94F878301844C9
S31508009BD020662046FFF756FC2046FFF731FE204652
S31508009BE0FFF7D9F9002010BDF0B583B002AF03F135
S31508009BF00F0404F4FC74ADEB040D02AE8DF80810E6
S31508009C00C1F3032141F020017170191DB1700912C9
S31508009C10F170337100217171397EB171397FF1713B
S31508009C209BB253B1511EF41D5D1E12FA85F211F84E
S31508009C30015F04F8015F9142F9D190F85A2090F833
S31508009C405010C06C0096083301F088FC10B9043730
S31508009C50BD46F0BD642005F00FFDF8E770B582B08B
S31508009C60BDF81850022680F8096180F80A210422F6
S31508009C7080F80B21002280F80C2180F80D512D1256
S31508009C8080F80E511D7880F80F515B7880F81031F6
S31508009C90019201230093082300F20912FFF7A4FF9B
S31508009CA002B070BD70B582B0069D032680F80961C2
S31508009CB080F80A21082280F80B21002280F80C215E
S31508009CC01E7880F80D615B7880F80E312B7880F865
S31508009CD00F316B7880F810319DF81C3080F81131FF
S31508009CE080F8122180F8132180F8142101920123AB
S31508009CF000930C2300F20912FFF776FF02B070BD3D
S31508009D0030B583B0042580F8095180F80A21082265
S31508009D1080F80B21002280F80C211D7880F80D515F
S31508009D205B7880F80E3180F80F2180F81021012326
S31508009D3080F81131022580F81251FF2580F8135159
S31508009D4080F81451019200930C2300F20912FFF7D0
S31508009D504BFF03B030BD70B582B0052580F80951B8
S31508009D6080F80A210A2280F80B21002280F80C21AB
S31508009D701D7880F80D515B7880F80E3180F80F2138
S31508009D8080F8102180F8112180F81221012380F82B
S31508009D901331022580F81451A02680F8156180F841
S31508009DA01651019200930E2300F20912FFF71CFFC9
S31508009DB002B070BD70B582B0069D062680F80961AE
S31508009DC080F80A21042280F80B21002280F80C2151
S31508009DD01E7880F80D615B7880F80E312B7880F854
S31508009DE00F316B7880F81031019201230093082314
S31508009DF000F20912FFF7F8FE02B070BD70B582B026
S31508009E00069D072680F8096180F80A21042280F851
S31508009E100B21002280F80C211E7880F80D615B78F2
S31508009E2080F80E312B7880F80F316B7880F8103176
S31508009E30019201230093082300F20912FFF7D4FECA
S31508009E4002B070BD10B58AB001238DF820300AAA79
S31508009E50002302F8073D8B1D13F8014D02F8014F48
S31508009E608B42F9D190F8512090F85010C06C00231D
S31508009E70079308AC069408240594049403930323D3
S31508009E800293F523019309230093212301F084FB10
S31508009E900AB010BD10B58CB005238DF824301023F8
S31508009EA08DF82B3001238DF82C3002238DF82D30B8
S31508009EB012238DF82E304B1E09AA053113F8014FCF
S31508009EC002F8014F8B42F9D190F8512090F85010C2
S31508009ED0C06C0023079309AC06940B2405940494DC
S31508009EE00393032302930523019309230093212354
S31508009EF001F052FB0CB010BD2DE9F04F93B00446AB
S31508009F00984690F85470002380F85430C56C2B6836
S31508009F101B6890F8501028469847002800F0F180F2
S31508009F2081464FF4967005F0A7FB94F8503000224E
S31508009F301146E06C01F039FC064650B1002389F859
S31508009F40063023689B6820469847304613B0BDE81C
S31508009F50F08F002389F806302B681B6894F8501098
S31508009F6028469847002800F0CE8080F8068004F13D
S31508009F7051094B46012294F85010E06C00F09FFFFF
S31508009F8006460028DDD1B4F8762040F24C539A42B2
S31508009F9046D0002F00F08D800025DFF87081DFF8AD
S31508009FA070A1DFF870B1EBB2626F42450CBFCDF815
S31508009FB00CB0CDF80CA0221D049200228DF82820A2
S31508009FC0ADF82A208DF83C208DF83D208DF83E20EE
S31508009FD08DF844200BA9CDF8151007919DF81400AB
S31508009FE08DF821008DF82000099194F8501003A8E7
S31508009FF00090E06C01F0B0FB06460028A1D194F869
S3150800A0005E20032A59D80135EBB29F42CBD80023EC
S3150800A0101A4694F85010E06C01F0C7FBD12690E779
S3150800A020B4F87430B3F51A7F07D040F22F42934242
S3150800A03003D040F2D5329342ABD1642005F01CFB25
S3150800A040012394F8512094F85010E06C01F0C4FBF9
S3150800A050064600287FF475AF63690BB9238B6BB18D
S3150800A060B4F87430B3F51A7F03D040F22F42934206
S3150800A07019D104F114012046FFF7E4FE002394F8F1
S3150800A080512094F85010E06C01F0A6FB00231A4604
S3150800A09094F85010E06C01F088FB23689B68204612
S3150800A0A09847D12651E704F114012046FFF7F2FE3E
S3150800A0B0E4E794F85E20032AA9D94B4694F8501091
S3150800A0C0E06C00F0FCFE064600287FF43AAF94F8F0
S3150800A0D05D3094F8512094F85010E06C01F07CFB48
S3150800A0E0064600287FF42DAF6423A4F884300023A5
S3150800A0F0A4F8823084F880302372012384F87930FA
S3150800A10023E7D62621E7D6261FE700BFE8215C0A03
S3150800A110A8BA03089CBA030870B582B004460E466E
S3150800A120154690F83030042B00F2E480DFE803F09F
S3150800A130030D1E254A0002230372D0F80920026186
S3150800A14043750375012380F830302A46314604F1F9
S3150800A150100002F029FE0346002874D0D4F809300E
S3150800A1601A7884F831205B7884F8323004F12203B7
S3150800A170C4F80930032384F8303094F83230023BAF
S3150800A1801F2B16D8DFE803F0131510431515151500
S3150800A1901515151515151515151515151515151561
S3150800A1A01515151515151546002384F8333007239C
S3150800A1B02372D4F809302361237A6375237504233F
S3150800A1C084F8303094F83230042B3FD0052B6AD00F
S3150800A1D0022B24D0237F002B00F08580012B40F032
S3150800A1E08D80E28B002A00F087802B886BB1013ABC
S3150800A1F0E2833368013333602B88013B9BB22B80A3
S3150800A200E28B002A78D0002BF1D100231BE005232E
S3150800A2102372CEE794F83130023B2372C9E72A4607
S3150800A220314604F1100002F0BFFD034658B194F818
S3150800A230253084F8343004F12003C4F809300023AB
S3150800A24084F830300123184602B070BD2A463146DC
S3150800A25004F1100002F0A8FD03460028F3D094F894
S3150800A2602530E02BE7D194F82630012BE3D194F87A
S3150800A27038309BB194F82730002BDCD0012384F8C2
S3150800A280333094F8223084F8363094F8233084F842
S3150800A290373094F8273084F83530CCE794F82730EF
S3150800A2A0012BC8D1EAE72A46314604F1100002F02C
S3150800A2B07BFD03460028C6D094F83330002BBAD06D
S3150800A2C060680028B7D094F8373094F8362094F8A8
S3150800A2D03410056804F12006019694F83560009656
S3150800A2E02D68A847A7E794F83130023BE38301239A
S3150800A2F0237776E70123A6E700232377E38B002B52
S3150800A30099D000239FE710B582B00446ADF8061031
S3150800A3100092BDF806303BB10DF1060269462046AB
S3150800A320FFF7FAFE0028F4D102B010BD70B582B06E
S3150800A33004460E46154690F83030042B00F2E480A9
S3150800A340DFE803F0030D1E254A0002230372D0F846
S3150800A3500920026143750375012380F830302A46C7
S3150800A360314604F1100002F01FFD0346002874D0A0
S3150800A370D4F809301A7884F831205B7884F83230BA
S3150800A38004F12203C4F80930032384F8303094F822
S3150800A3903230023B1F2B16D8DFE803F013151043A3
S3150800A3A0151515151515151515151515151515154F
S3150800A3B0151515151515151515151546002384F8C3
S3150800A3C0333007232372D4F809302361237A63755F
S3150800A3D02375042384F8303094F83230042B3FD0A8
S3150800A3E0052B6AD0022B24D0237F002B00F0858012
S3150800A3F0012B40F08D80E28B002A00F087802B88A5
S3150800A4006BB1013AE2833368013333602B88013B31
S3150800A4109BB22B80E28B002A78D0002BF1D1002347
S3150800A4201BE005232372CEE794F83130023B2372F2
S3150800A430C9E72A46314604F1100002F0B5FC034686
S3150800A44058B194F8253084F8343004F12003C4F860
S3150800A4500930002384F830300123184602B070BD55
S3150800A4602A46314604F1100002F09EFC03460028F5
S3150800A470F3D094F82530FF2BE7D194F82630012B3A
S3150800A480E3D194F838309BB194F82730002BDCD010
S3150800A490012384F8333094F8223084F8363094F85F
S3150800A4A0233084F8373094F8273084F83530CCE7F1
S3150800A4B094F82730012BC8D1EAE72A46314604F139
S3150800A4C0100002F071FC03460028C6D094F8333019
S3150800A4D0002BBAD060680028B7D094F8373094F8C3
S3150800A4E0362094F83410056804F12006019694F88D
S3150800A4F0356000962D68A847A7E794F83130023BE7
S3150800A500E3830123237776E70123A6E7002323774E
S3150800A510E38B002B99D000239FE710B582B0044641
S3150800A520ADF806100092BDF806303BB10DF10602F3
S3150800A53069462046FFF7FAFE0028F4D102B010BD9E
S3150800A54010B50446436803B1984723689B692046BB
S3150800A550984710BD70477047704708B50022427586
S3150800A56080F82520026180F82A200368DB6998476D
S3150800A57008BD10B582B004468189027D0132D2B287
S3150800A580027500F12803009300F118038068FFF7AD
S3150800A59011FC23689B6820469847092384F82A30CB
S3150800A5A002B010BD90F82A30002B4FD1F0B583B019
S3150800A5B00446806890F8463033B1437A23B9637D00
S3150800A5C013B994F825302BB1236913F0010F15D16F
S3150800A5D003B0F0BD0123437284F82530A068418B8F
S3150800A5E0A1810022226122751123009304F126031A
S3150800A5F0FFF734FB022384F82A30E9E704F126073B
S3150800A60004F11605227DA1890126019600953B468F
S3150800A610FFF748FB304605F02FF8227DA189002375
S3150800A620019300953B46A068FFF73CFB237D334426
S3150800A6302375304605F020F82B46227DA189A068AF
S3150800A640FFF75EFB042384F82A30C1E77047000051
S3150800A65010B5044618482060A16039B1486E30B379
S3150800A660886E00B3C86E00B3086FD0B11349216075
S3150800A670002184F82410E1612162A06880F848204E
S3150800A680A2681361702384F8263084F82710712392
S3150800A69084F8283084F829102046FFF75EFF204604
S3150800A6A010BD032004E0012002E0022000E00020A3
S3150800A6B001EB80014C66D9E718BB03089C3B0308ED
S3150800A6C010B584B0034690F82420012A84BF0022DE
S3150800A6D080F8242090F8241041F0700104AA02F8AA
S3150800A6E0011D81898068DC7D01949B7D009301238F
S3150800A6F0FFF77AFA04B010BDF0B583B0044690F8B7
S3150800A7002A30023B072B09D8DFE803F03D4F04A3A4
S3150800A71010687A8D036913F0020F01D103B0F0BDFA
S3150800A720FFF7CEFF062384F82A30F7E7036913F00C
S3150800A730100FF3D000F1280700F11805027D818972
S3150800A7400126019600953B468068FFF7ABFA30462E
S3150800A75004F092FF227DA1890023019300953B46D0
S3150800A760A068FFF79FFA237D33442375304604F02B
S3150800A77083FF2B46227DA189A068FFF7C1FA08232B
S3150800A78084F82A30CAE7036913F0040FC6D0027D9D
S3150800A7900132D2B2027500F1160381898068FFF78B
S3150800A7A0AFFA032384F82A30B8E7036913F0020FD7
S3150800A7B0B4D0FFF785FF012004F05EFF227D013249
S3150800A7C0D2B22275A1891323009304F12803A06845
S3150800A7D0FFF744FA072384F82A309FE7036913F042
S3150800A7E0400F9BD0027D0132D2B2027500F11803E8
S3150800A7F081898068FFF784FA082384F82A308DE770
S3150800A800036913F0200F89D08268002382F8463046
S3150800A810826882F848300125457503681B699847A0
S3150800A82084F82A507AE7036913F0800F3FF476AF6D
S3150800A830027D0132D2B20275818900F126030093A6
S3150800A84000F116038068FFF7B5FA052384F82A3065
S3150800A85064E7036913F0080F3FF460AF81898068E5
S3150800A860FEF7B7FF4FF6FF73A3810023236184F831
S3150800A8702A3053E770B582B083685A7A52B993F88A
S3150800A88047203AB1427D2AB990F8252012B90A7AAA
S3150800A890022A06D086890A78F3B29A4215D002B0FF
S3150800A8A070BD4C7B0A7B42EA0422112AF2D10022AF
S3150800A8B083F8472084680123637280F8253083680B
S3150800A8C05B8B838180F82A20E4E74A78331243F0C9
S3150800A8D020039A42E3D10C4605468B79CA7943EAA6
S3150800A8E00221012908D090F82810994200F0078122
S3150800A8F02846FFF701FFD2E7237A012BF8D0032B6E
S3150800A9001ED0022B4FD0052B6BD0042B00F0918064
S3150800A910062B00F0B380072BEAD1237B827D9A426F
S3150800A92000F0E1802A7E9A42E2D1627B6B7E9A42EF
S3150800A930DED1637A2B752B6943F080032B61D7E749
S3150800A940627C237C53EA0223D2D1E27CA37C53EABD
S3150800A9500223CDD1A37B90F826209A4213D095F8EE
S3150800A96028209A42C4D1E27B95F829309A42BFD171
S3150800A970637A2B75237B2B76637B6B762B6943F087
S3150800A98040032B61B4E7E17B90F827209142E6D19A
S3150800A990637A0375237B8375637BC375036943F009
S3150800A9A004030361A4E7627B237B43EA0223112B9A
S3150800A9B00CD0132B9CD1637A0375A37B0376E37BB8
S3150800A9C04376036943F01003036191E7637A0375DD
S3150800A9D0A37B8375E37BC375036943F001030361B6
S3150800A9E086E7627C237C53EA022381D1237B90F895
S3150800A9F026209A4211D095F828209A427FF478AFFB
S3150800AA00627B95F829309A427FF472AF637A2B7588
S3150800AA102B6943F020032B616AE7617B90F82720B6
S3150800AA209142E8D1637A0375036943F0020303612F
S3150800AA305EE7237B90F826209A4212D095F82820C4
S3150800AA409A427FF455AF627B95F829309A427FF493
S3150800AA504FAF05F11803627A3146A868FFF77BF90C
S3150800AA6046E7617B90F827209142E7D100F116036B
S3150800AA70627A31468068FFF76EF939E7237B90F8EA
S3150800AA8026209A421AD095F828209A427FF430AFA9
S3150800AA90627B95F829309A427FF42AAF627A2A7542
S3150800AAA005F11803009305F128033146A868FFF756
S3150800AAB0A5F92B689B682846984719E7617B90F8A3
S3150800AAC027209142DFD1627A027500F116030093BE
S3150800AAD000F1260331468068FFF790F92B689B68DA
S3150800AAE02846984704E7617BC27D91427FF41AAFF6
S3150800AAF0637A0375036943F008030361F8E690F87F
S3150800AB00293093427FF4F4AE237AA12B7FF4F0AE7A
S3150800AB102679711E03685B6904F10902C9B2984770
S3150800AB20637A012B10D0022B7FF4E2AE286A002844
S3150800AB303FF4DEAEB31E02680A3400941468DBB232
S3150800AB4000222946A047D3E6E86900283FF4D0AE9C
S3150800AB50B31E02680A3400941468DBB20022294640
S3150800AB60A047C5E603292BD8DFE801F0020C16201A
S3150800AB70007A00F00F00072824D001288CBF002097
S3150800AB8001207047007A00F00F000138C0B2022891
S3150800AB908CBF002001207047007A00F00F000338B0
S3150800ABA0C0B202288CBF002001207047007A00F04E
S3150800ABB00F000538C0B202288CBF0020012070475C
S3150800ABC0002070470120704708B5032908D9806816
S3150800ABD0C0F31700044B5B5CD84000F0010008BDC9
S3150800ABE0FFF7C0FFFBE700BFBC3B03080A4B5A5CF4
S3150800ABF00123934090F84320B0F8441042EA01221A
S3150800AC0022EA030180F84310090AA0F844101A4200
S3150800AC1014BF012000207047BC3B0308082904D054
S3150800AC2009290CBF007B00207047C07A7047014491
S3150800AC300879704770B5044601295BD91346002A7E
S3150800AC4058D01278012A0DD0112A56D1032954D981
S3150800AC50CA1ED2B23C2A28BF3C22D91C043026F090
S3150800AC60FBFC08E04A1ED2B23C2A28BF3C22591CEB
S3150800AC70043026F0F1FCA268C2F31702236CC3F372
S3150800AC8017039A4236D022EA030384F843301B0A94
S3150800AC90A4F84430236C62F317032364002120468A
S3150800ACA0FFF760FF0646054601212046FFF75AFFD3
S3150800ACB010B146F00205EDB202212046FFF752FF19
S3150800ACC010B145F00405EDB203212046FFF74AFF0F
S3150800ACD010B145F00805EDB294F84E30AB4209D0F4
S3150800ACE025EA030394F8432063F3030284F8432018
S3150800ACF084F84E5094F84D3003B970BD23681B682C
S3150800AD0004F1460120469847F7E781B130B40D466D
S3150800AD10C37C8B4214D002460223DCB2917EA94240
S3150800AD2007D001330732102BF7D1002006E0083090
S3150800AD3070473CB10830C4EBC404204430BC7047AB
S3150800AD400124F7E70020F9E711F0800F46D1F0B4A7
S3150800AD500746072B44D812B1C079072843D0F87C98
S3150800AD60D0B13D460224E0B2AE7E2EB1013407359D
S3150800AD70102CF8D1002034E098B3A9B972B1C0EB11
S3150800AD80C0033B4441221A73FB790133FB71C0EBC4
S3150800AD90C0000744387B24E00120EEE7C0EBC0037F
S3150800ADA03B4401221A73F2E74FF00004C1F3020193
S3150800ADB061F3C5046AB144F04004FB790133DBB2A0
S3150800ADC0FB7163F30204C0EBC00007443C73E0B2B6
S3150800ADD007E06FF3861463F30204F4E70020704774
S3150800ADE00020F0BC70470020FBE70000F0B4144BCD
S3150800ADF003600023C3710373012242738373051D25
S3150800AE0085600371082141710F2161F387038371FE
S3150800AE10034600F1690700241646DC741E755C7546
S3150800AE20C2EBC20101448D6001320733BB42F4D143
S3150800AE30002380F8B830034B11221A70F0BC704713
S3150800AE4034BB0308140A002070B4B1B900F1080332
S3150800AE508BB3186858B35B797BB30178914226D0D7
S3150800AE60013BDBB2013303EB43030344033098424F
S3150800AE701CD001789142F9D119E00E46C37C8B4269
S3150800AE8012D001460223DDB28C7EB44205D00133CE
S3150800AE900731102BF7D1002009E055B100F108035E
S3150800AEA0C5EBC5052B44D3E70125F7E7002070BCA1
S3150800AEB070470020FBE70020F9E70020F7E70BB30F
S3150800AEC0F0B41F4639B9083000B301710760427102
S3150800AED00020F0BC7047C37C8B4211D00446022385
S3150800AEE0DEB2A57E8D4205D001330734102BF7D18B
S3150800AEF0D620EEE746B10830C6EBC6063044E3E78F
S3150800AF000126F8E7D8207047D620E2E7D620E0E702
S3150800AF1070B582B00C4616460C4D00221021284604
S3150800AF2005F0B2FA44F002048DF804408DF8056085
S3150800AF304FF0FF33022201A9054807F0B1FE0122AE
S3150800AF401021284605F0A0FA02B070BD0010024094
S3150800AF50981F00202DE9F84F824616461F469DF891
S3150800AF602890002500EB810802F11E0B17E036B386
S3150800AF705AF82B0003685B6939469847D8F8780071
S3150800AF8003681C684B463A463146A0470D282AD125
S3150800AF90EBB2022B2BD8642004F06EFB0135D8F8EF
S3150800AFA0780003685C684B463A463146A047E02875
S3150800AFB0DDD00D280CD00028E0D004460CE0012294
S3150800AFC0E8215046FFF7A4FF662004F055FBD5E7B5
S3150800AFD0EBB2022B03D904462046BDE8F88F64205D
S3150800AFE004F04AFBDAE704460028F5D000E00446F8
S3150800AFF03EB11E365AF8260003685B6939469847FB
S3150800B000EAE70122E8215046FFF782FF662004F0AE
S3150800B01033FBE1E770B584B004AC04F8091D104DA4
S3150800B02000221021284605F02FFA0E4E4FF0FF3366
S3150800B03001222146304607F033FE04A9002301F811
S3150800B040013D4FF0FF330122304608F016F8012281
S3150800B0501021284605F018FA9DF80F0004B070BDB7
S3150800B06000100240981F00202DE9F84F04468A4632
S3150800B07017469B4604F0FAFA00F59C550835002653
S3150800B080B146B0464AEA07074FF0F00A04F0EEFA6E
S3150800B090401B002820DA3A4651462046FFF738FF7B
S3150800B0A0C82604F0E3FA401B00280BDA314620468E
S3150800B0B0FFF7B0FF10F0800FF3D08022C82120469A
S3150800B0C0FFF726FFF8212046FFF7A4FF00F00F063A
S3150800B0D0042E04D00E2E0CD03046BDE8F88F09F1A8
S3150800B0E001091FFA89F9BBF1000FCFD0D945CDD197
S3150800B0F0F2E708F101085FFA88F8B8F1030FC5D13D
S3150800B100EAE700002DE9F04F87B000908B460292DF
S3150800B1109A46109E9DF844300193BAF800904B78F1
S3150800B12003930023AAF800308B7813F0020F14BF9C
S3150800B13020221022E821FFF7EBFE029B9BF8002055
S3150800B14000210098FFF790FF0546062859D00028E9
S3150800B15040F08480C821009C2046FFF75BFF10F072
S3150800B160040F78D030212046FFF754FF044648459F
S3150800B170C8BF5FFA89F4BAF80020A9EB020212B236
S3150800B18022EAE272A242A8BF224617460DF1180823
S3150800B190082308F8013D00221021314805F074F90A
S3150800B1A04FF0FF33012241462E4807F079FDFFB2E2
S3150800B1B03A460021304626F073FA4FF0FF333A46F6
S3150800B1C03146284807F059FF3E44012210212448F9
S3150800B1D005F05AF90422C8210098FFF799FEBAF833
S3150800B1E0003023449BB2AAF80030039A944221D334
S3150800B1F04B451FD2019B002B9FD0184604F03CFA02
S3150800B2009BE7F821009C2046FFF704FF80F010001A
S3150800B210C0F300109BF8023060F341038BF802304C
S3150800B22013F0020F14BF20221022E8212046FFF750
S3150800B2306FFE82E7A846F8210098FFF7EBFEC0F3F9
S3150800B24000109BF8023060F341038BF80230404649
S3150800B25007B0BDE8F08F4FF0F008F8E78046F6E74C
S3150800B26000100240981F0020F8B50F4681BB00F178
S3150800B2700804002C49D02168002948D01D460646F6
S3150800B2803946FFF7E1FD2860002842D083789B08FD
S3150800B2900F2B28BF0F231A4601239340013B069A1A
S3150800B2A013803A46E0213046FFF732FED821304671
S3150800B2B0FFF7B0FEA3791BB396F8B82042F0020256
S3150800B2C00243D2B2D8213046FFF722FE0020F8BD4D
S3150800B2D0C17CB94212D005460224E1B2AE7EBE4216
S3150800B2E005D001340735102CF7D1D620EFE751B138
S3150800B2F000F10804C1EBC1010C44BAE70121F7E7E4
S3150800B30000F0F902DEE7D620E1E7D620DFE7D7200E
S3150800B310DDE7DB20DBE730B585B004461D460023B4
S3150800B3200393ADF80A300DF10A03009303ABFFF758
S3150800B3309BFF034610B1184605B030BDBDF80A207C
S3150800B3409DF824300193089B00932B4603992046C9
S3150800B350FFF7D8FE0346EEE7F0B583B00D4617466D
S3150800B3601C46114E00221021304605F08DF845F096
S3150800B370020502A901F8015D0C4D4FF0FF330122C9
S3150800B380284607F08DFC4FF0FF333A4621462846FB
S3150800B39007F086FC3C4401221021304605F074F87B
S3150800B3A0204603B0F0BD00BF00100240981F0020E1
S3150800B3B02DE9F04F87B003921D4602934E78731E0F
S3150800B3C0DBB23F2B00F2C88004468B4604F04EF9E8
S3150800B3D000F59C5808F108089BF8023003F00103B1
S3150800B3E0002B14BF80224022E8212046FFF790FD5B
S3150800B3F0002D00F0AF804FF0C80A00230093049692
S3150800B400109EBDF81030029A934228BF1346059342
S3150800B410DBB21D46019333462A4610212046FFF724
S3150800B4209BFF2A4638212046FFF772FD9BF800202D
S3150800B43042F02002F0212046FFF76AFD51462046D9
S3150800B440FFF7E8FD10F0800FF8D08022514620461D
S3150800B450FFF75EFDF8212046FFF7DCFD10F00F052B
S3150800B46003D04FF00009009F58E0029B059A9B1AEB
S3150800B4709BB202931644002BC3D15BE009F1010984
S3150800B4801FFA89F9039BFBB199451DD152E0013793
S3150800B490FFB2032F18D14DE0F8212046FFF7BAFD79
S3150800B4A080F02000C0F340109BF8023060F30003E0
S3150800B4B08BF8023003F00103002B14BF80224022D0
S3150800B4C0E8212046FFF724FD009A38212046FFF799
S3150800B4D01FFD327810212046FFF71AFD019A382100
S3150800B4E02046FFF715FD9BF8002042F02002F021C8
S3150800B4F02046FFF70DFD51462046FFF78BFD10F05D
S3150800B500800FF8D0802251462046FFF701FDF8212A
S3150800B5102046FFF77FFD10F00F05A6D004F0A6F829
S3150800B520A0EB08000028A0DA062DB5D00E2DAED067
S3150800B530042DA3D0F8212046FFF76CFDC0F3401078
S3150800B5409BF8023060F300038BF80230284607B0F8
S3150800B550BDE8F08F0025EDE7DA25F7E730B585B0C9
S3150800B56004461D4600230393ADF80A300DF10A037D
S3150800B570009303ABFFF778FE034610B1184605B0F3
S3150800B58030BDBDF80A20089B00932B460399204638
S3150800B590FFF70EFF0346F1E72DE9F04F8BB006469D
S3150800B5A091461D46BDF86080BDF864700023069379
S3150800B5B0ADF816300DF11603009306ABFFF754FEEF
S3150800B5C0044618B120460BB0BDE8F08F8DF81C5024
S3150800B5D09DF850308DF81D309DF854308DF81E308A
S3150800B5E09DF858308DF81F30BDF85C30ADF8203026
S3150800B5F0ADF8228007AB082220213046FFF7ACFEC3
S3150800B600BDF816304A4610213046FFF72DFD044690
S3150800B6100028D7D16DB21A9B002B62D0002D4CDAC8
S3150800B620069A937843F002039370B8F1000F42D05C
S3150800B63045464FF0000ACDF80C90B9461B9F15E019
S3150800B640F8213046FFF7E6FC069B80F02000C0F3A1
S3150800B65040109A7860F341029A7005E0BDF81430FC
S3150800B660ED1AADB24B4524D3002D46D0ADF8149053
S3150800B670BDF81620CDF804A01A9B009305AB0699D1
S3150800B6803046FFF73FFD04460628D9D0002899D151
S3150800B690002FE3D03B68D3F800B0BDF81410A8EB30
S3150800B6A00503ADF826300DF126031A9A3846D84711
S3150800B6B0D4E7DDF80C90A02117E0069A937843F0BA
S3150800B6C001039370BDF816201A9B00933B46069912
S3150800B6D03046FFF76DFE044600287FF473AF8021DD
S3150800B6E003E0002DB4BFA0218021BDF816304A46DC
S3150800B6F03046FFF7B9FC044664E7DDF80C90002CE9
S3150800B7007FF460AFA021F0E730B589B00024079434
S3150800B7100C9D0695059304930394012302930194C3
S3150800B720062300938023FFF737FF09B030BD30B5F5
S3150800B73089B0002407940D9D0695059304930394F8
S3150800B740022302939DF83030019306230093802349
S3150800B750FFF722FF09B030BDF0B599B005460E4691
S3150800B76017461C4608AB019300940923FFF7DFFF31
S3150800B770034610B1184619B0F0BD1E9B079308ABD7
S3150800B780069340230593BDF82230049300230393C0
S3150800B7900223029301940623009380233A463146F6
S3150800B7A02846FFF7F9FE0346E4E710B588B00024FB
S3150800B7B0079406940594049403940294019305232C
S3150800B7C000932346FFF7E8FE04464FF4967003F00D
S3150800B7D053FF204608B010BD10B588B00024079462
S3150800B7E00694059404940394029401930923009300
S3150800B7F02346FFF7D1FE08B010BD002900F0E78206
S3150800B8002DE9F04F91B002918346C1EBC103034481
S3150800B8101B7B13F0400F19D0C1EBC10303441B7BFC
S3150800B82003F007084FF0010ACDF810A0CDF800A0E4
S3150800B830C346D046824639E0D846D3469BF80730F9
S3150800B840434504BF03F1FF338BF80730029BC3EB74
S3150800B850C3035B4400221A73012159739A730BF1CF
S3150800B8600400986011B0BDE8F08FD846D346E5E7E6
S3150800B8704FF0010867E1DDF81480BA465F46DDF847
S3150800B88018B09AF80730BB4204BF03F1FF338AF8B1
S3150800B8900730019BC3EBC303534400221A734FF0CE
S3150800B8A0010159739A730AF104029A6008F1FF3389
S3150800B8B0DBB20E2B00F22881B8F10F0F00F22181BE
S3150800B8C0C8EBC80353441B7BC3F3C2035B4540F074
S3150800B8D0248134E1DDF81480BA465F46DDF818B0F5
S3150800B8E0CFE7DDF810A066E1DDF824A04F46D9467B
S3150800B8F0DDF820B0FB794B4504BF03F1FF33FB713C
S3150800B900039BC3EBC3033B4400221A734FF00101A8
S3150800B91059739A733A1D9A600AF1FF33DBB20E2BFC
S3150800B92000F22B81BAF10F0F00F2E480CAEBCA03CA
S3150800B9303B441B7BC3F3C2035B4540F0268136E1DB
S3150800B940DDF824A04F46D946DDF820B0D2E7DDF869
S3150800B95000A069E1DDF830A05E46DDF82CB099F864
S3150800B9600730B34204BF03F1FF3389F80730079B5A
S3150800B970C3EBC3034B4400221A734FF001015973FA
S3150800B9809A7309F104029A600AF1FF33DBB20E2BAF
S3150800B99000F22B81BAF10F0F00F2A580CAEBCA0399
S3150800B9A04B441B7BC3F3C2035B4540F0278137E159
S3150800B9B0DDF830A05E46DDF82CB0D0E7DDF800A053
S3150800B9C06AE1DDF838B0DDF83CA099F80730434560
S3150800B9D004BF03F1FF3389F807300A9BC3EBC3039F
S3150800B9E04B4400221A734FF0010159739A7309F1F7
S3150800B9F004029A600AF1FF33DBB20E2B00F22D81A6
S3150800BA00BAF10F0F69D8CAEBCA034B441B7BC3F3C1
S3150800BA10C2035B4540F02A813AE1DDF838B0DDF82B
S3150800BA203CA0D2E7009F67E1009C90E1009DBAE147
S3150800BA3099F807305B4504BF03F1FF3389F80730EF
S3150800BA40CAEBCA0ACA444FF000038AF80C304FF012
S3150800BA5001028AF80D208AF80E3009F10403CAF8A3
S3150800BA600830631EDBB20E2B00F257810F2C09D863
S3150800BA70C4EBC4034B441B7BC3F3C203B34240F07D
S3150800BA80548161E199F80730B34204BF03F1FF33EB
S3150800BA9089F807300D9BC3EBC3034B4400221A7386
S3150800BAA04FF0010159739A7309F104029A607B1EDB
S3150800BAB0DBB20E2B00F206810F2F09D8C7EBC7039E
S3150800BAC04B441B7BC3F3C203434540F0038110E19B
S3150800BAD0DDF838B0DDF83CA077E7DDF830A05E4643
S3150800BAE0DDF82CB03BE7DDF824A04F46D946DDF853
S3150800BAF020B0FFE6DDF81480BA465F46DDF818B0D8
S3150800BB00BFE6D846D34699E69AF81330C3F3C2037C
S3150800BB105B453FF4ADAE4FF0010808F10103DBB217
S3150800BB205FFA83F8B8F10F0F3FF686AEC3EBC30290
S3150800BB305244127BC2F3C20201339345F0D1B8F1E5
S3150800BB40000F3FF492AECDF80480C8EBC803534407
S3150800BB501B7B13F0400F3FF49CAEC8EBC80353445D
S3150800BB601B7B03F007074FF00109CDF81480CDF8C9
S3150800BB7018B0BB465746CA46CEE6FB7CC3F3C2039B
S3150800BB805B453FF4AEAEDDF810A00AF10103DBB267
S3150800BB905FFA83FABAF10F0F3FF66DAEC3EBC30235
S3150800BBA03A44127BC2F3C20201339345F0D1BAF18B
S3150800BBB0000F3FF48FAECDF80CA0CAEBCA033B4486
S3150800BBC01B7B13F0400F3FF49BAECAEBCA033B4402
S3150800BBD01B7B03F00709DDF81080CDF820B0CDF8FF
S3150800BBE024A0CB46C246B946CEE699F81330C3F32D
S3150800BBF0C2035B453FF4ABAEDDF800A00AF10103D2
S3150800BC00DBB25FFA83FABAF10F0F3FF66DAEC3EBFC
S3150800BC10C3024A44127BC2F3C20201339345F0D1F0
S3150800BC20BAF1000F3FF48CAECDF81CA0CAEBCA03DC
S3150800BC304B441B7B13F0400F3FF499AECAEBCA0383
S3150800BC404B441B7B03F00706DDF80080CDF82CB0CB
S3150800BC50CDF830A0B346C246CCE699F81330C3F304
S3150800BC60C2035B453FF4AAAEDDF800A00AF1010362
S3150800BC70DBB25FFA83FABAF10F0F3FF66BAEC3EB8E
S3150800BC80C3024A44127BC2F3C20201339345F0D180
S3150800BC90BAF1000F3FF48CAECDF828A0CAEBCA0360
S3150800BCA04B441B7B13F0400F3FF497AECAEBCA0315
S3150800BCB04B441B7B03F00708009FCDF838B0CDF83E
S3150800BCC03CA0F4E699F81330C3F3C20343453FF4A6
S3150800BCD0A9AE009F0137FBB2DFB20F2F3FF671AE58
S3150800BCE0C3EBC3024A44127BC2F3C2020133904536
S3150800BCF0F2D1002F3FF491AE0D97C7EBC7034B4423
S3150800BD001B7B13F0400F3FF4C5AEC7EBC7034B448C
S3150800BD101E7B06F00706009CA3E699F81330C3F3CA
S3150800BD20C203B3423FF480AE009C631CDBB2DCB2B4
S3150800BD300F2C3FF6A7AEC3EBC3024A44127BC2F3ED
S3150800BD40C20201339642F2D1002C3FF49BAEA246C2
S3150800BD50C4EBC4034B441B7B13F0400F3FF470AE97
S3150800BD60C4EBC4034B4493F80CB00BF0070B009DCF
S3150800BD701DE099F81330C3F3C2035B453FF456AE92
S3150800BD80009D6B1CDBB2DDB20F2D3FF651AEC3EB47
S3150800BD90C3024A44127BC2F3C20201339345F2D16D
S3150800BDA0002D3FF445AE29464846FFF726FD6B1E93
S3150800BDB0DBB20E2BDDD80F2D3FF63AAEC5EBC50329
S3150800BDC04B441B7BC3F3C2035B45DAD1E8E77047F4
S3150800BDD02DE9F04F8BB041290DD0C37C8B4238D06A
S3150800BDE002460223DDB2947E8C421BD00133073211
S3150800BDF0102BF7D113E0034600F16907012200244E
S3150800BE001646051DDC741E755C75C2EBC20101443D
S3150800BE108D6001320733BB42F4D10023C3710BB0E6
S3150800BE20BDE8F08F002DFAD083460195C5EBC50312
S3150800BE3003441B7B13F0400F17D003F0070A4FF09B
S3150800BE400109CDF81090CDF80890D346CA46814628
S3150800BE5038E00125E8E7DA46CB469BF80730534534
S3150800BE6004BF03F1FF338BF80730019BC3EBC30311
S3150800BE705B4400221A73012159739A730BF104006B
S3150800BE809860CCE7DA46CB46E7E74FF0010AEAE0E6
S3150800BE90DDF818A0D846DDF814B099F80730434500
S3150800BEA004BF03F1FF3389F80730009BC3EBC303D4
S3150800BEB04B4400221A734FF0010159739A7309F122
S3150800BEC004029A600AF1FF33DBB20E2B00F2AC8053
S3150800BED0BAF10F0F00F2A580CAEBCA034B441B7BCD
S3150800BEE0C3F3C2035B4540F0A880B8E0DDF818A0AC
S3150800BEF0D846DDF814B0D0E7DDF810A0EAE0DDF8A2
S3150800BF0020B0DDF824A099F80730434504BF03F1B3
S3150800BF10FF3389F80730039BC3EBC3034B44002266
S3150800BF201A734FF0010159739A7309F104029A6062
S3150800BF300AF1FF33DBB20E2B00F2AD80BAF10F0F18
S3150800BF4069D8CAEBCA034B441B7BC3F3C2035B45E0
S3150800BF5040F0AA80BAE0DDF820B0DDF824A0D2E7E8
S3150800BF60029FE7E0029C10E1029D3AE199F807304A
S3150800BF705B4504BF03F1FF3389F80730CAEBCA0AE9
S3150800BF80CA444FF000038AF80C304FF001028AF8D1
S3150800BF900D208AF80E3009F10403CAF80830631E2A
S3150800BFA0DBB20E2B00F2D7800F2C09D8C4EBC403E2
S3150800BFB04B441B7BC3F3C203B34240F0D480E1E099
S3150800BFC099F80730B34204BF03F1FF3389F8073005
S3150800BFD0079BC3EBC3034B4400221A734FF00101BE
S3150800BFE059739A7309F104029A607B1EDBB20E2B11
S3150800BFF000F286800F2F09D8C7EBC7034B441B7B7B
S3150800C000C3F3C203434540F0838090E0DDF820B0D7
S3150800C010DDF824A077E7DDF818A0D846DDF814B0D7
S3150800C0203BE7DA46CB4618E799F81330C3F3C20361
S3150800C0305B453FF42AAF4FF0010A0AF10103DBB270
S3150800C0405FFA83FABAF10F0F3FF605AFC3EBC302E7
S3150800C0504A44127BC2F3C20201339345F0D1BAF1C6
S3150800C060000F3FF40FAFCDF800A0CAEBCA034B444C
S3150800C0701B7B13F0400F3FF418AFCAEBCA034B44BF
S3150800C0801B7B03F007080126CDF814B0CDF818A0DD
S3150800C090C346B2464CE799F81330C3F3C2035B456F
S3150800C0A03FF42AAFDDF810A00AF10103DBB25FFA0C
S3150800C0B083FABAF10F0F3FF6EBAEC3EBC3024A445D
S3150800C0C0127BC2F3C20201339345F0D1BAF1000FD5
S3150800C0D03FF40CAFCDF80CA0CAEBCA034B441B7B4C
S3150800C0E013F0400F3FF417AFCAEBCA034B441B7B50
S3150800C0F003F00708049FCDF820B0CDF824A074E714
S3150800C10099F81330C3F3C20343453FF429AF029F9E
S3150800C1100137FBB2DFB20F2F3FF6F1AEC3EBC30216
S3150800C1204A44127BC2F3C20201339045F2D1002F72
S3150800C1303FF411AF0797C7EBC7034B441B7B13F0BC
S3150800C140400F3FF445AFC7EBC7034B441E7B06F0D1
S3150800C1500706029C23E799F81330C3F3C203B342D8
S3150800C1603FF400AF029C631CDBB2DCB20F2C3FF637
S3150800C17027AFC3EBC3024A44127BC2F3C2020133A0
S3150800C1809642F2D1002C3FF41BAFA246C4EBC4037F
S3150800C1904B441B7B13F0400F3FF4F0AEC4EBC403D3
S3150800C1A04B4493F80CB00BF0070B029D1DE099F871
S3150800C1B01330C3F3C2035B453FF4D6AE029D013587
S3150800C1C0EBB2DDB20F2D3FF6D1AEC3EBC3024A4444
S3150800C1D0127BC2F3C20201339345F2D1002D3FF41C
S3150800C1E0C5AE29464846FFF708FB6B1EDBB20E2B89
S3150800C1F0DDD80F2D3FF6BAAEC5EBC5034B441B7B06
S3150800C200C3F3C2035B45DAD1E8E72DE9F04F95B0F1
S3150800C21010F1080C00F047828468002C00F0468272
S3150800C220837311F0800F40F04A82072A00F2478292
S3150800C230C47C24B305460224E6B2AF7E37B1013486
S3150800C2400735102CF8D14FF0D40B3AE2002E00F047
S3150800C2503682B1B9C6EBC606064401253573C27CDB
S3150800C260AA4247D001460222D6B28C7EAC421CD0E6
S3150800C27001320731102AF7D14FF0D60B21E20126F9
S3150800C280E7E700242546C1F3020161F3C50564F317
S3150800C290861562F30205C6EBC60682191573EDB25A
S3150800C2A0002DDCD14FF0D40B0BE2002E00F00182FA
S3150800C2B0C6EBC6061CEB060600F0FE818046B37187
S3150800C2C02B4600221146FFF770FA8346002800F035
S3150800C2D0F881412D10D098F81330AB423ED0424633
S3150800C2E00223D8B2917EA9421DD001330732102B02
S3150800C2F0F7D1E6E10126DBE7434608F169060122A4
S3150800C3000020154608F10404D8741D755875C2EB4B
S3150800C310C20141448C60013207339E42F4D10023A6
S3150800C32088F80730CDE1002800F0CB810190C0EBFA
S3150800C330C00343441B7B13F0400F1DD0C0EBC00065
S3150800C34008EB00031B7B03F0070A012703970097F6
S3150800C350CDF810B0D346C246B8463CE00120E5E722
S3150800C360D046DA46DDF810B098F80730534504BFD2
S3150800C37003F1FF3388F80730019BC3EBC30242443D
S3150800C3800023137301215173937308F10403936017
S3150800C39097E1D046DA46DDF810B0E5E74FF0010838
S3150800C3A0B2E1DDF81C805F46DDF818B09AF8073070
S3150800C3B0BB4204BF03F1FF338AF80730029BC3EB85
S3150800C3C0C303534400221A734FF0010159739A7339
S3150800C3D00AF104029A6008F1FF33DBB20E2B00F271
S3150800C3E07481B8F10F0F00F25981C8EBC8035344A2
S3150800C3F01B7BC3F3C2035B4540F0708180E1DDF827
S3150800C4001C805F46DDF818B0D0E7DDF80C80B3E194
S3150800C410DDF828805F46DDF824B0CA469AF807306A
S3150800C420BB4204BF03F1FF338AF80730059BC3EB11
S3150800C430C303534400221A734FF0010159739A73C8
S3150800C4400AF104029A6008F1FF33DBB20E2B00F200
S3150800C4507481B8F10F0F00F21B81C8EBC80353446F
S3150800C4601B7BC3F3C2035B4540F0708180E1DDF8B6
S3150800C47028805F46DDF824B0CA46CFE7DDF800A07D
S3150800C480B4E15F46DDF82CB0D146DDF830A099F866
S3150800C4900730BB4204BF03F1FF3389F80730089B16
S3150800C4A0C3EBC3034B4400221A734FF001015973BF
S3150800C4B09A7309F104029A600AF1FF33DBB20E2B74
S3150800C4C000F27581BAF10F0F00F2DB80CAEBCA03DE
S3150800C4D04B441B7BC3F3C2035B4540F0718181E18A
S3150800C4E05F46DDF82CB0D146DDF830A0CFE7009FD7
S3150800C4F0B0E10F9FD946DDF838B09AF807304B45BA
S3150800C50004BF03F1FF338AF807300D9BC3EBC3035F
S3150800C510534400221A734FF0010159739A730AF1B2
S3150800C52004029A607B1EDBB20E2B00F279810F2F74
S3150800C53000F2A080C7EBC70353441B7BC3F3C203B7
S3150800C5405B4540F0758182E10F9FD946DDF838B02A
S3150800C550D3E7DDF80080B2E1DDF840B0DDF84480CD
S3150800C5609AF807304B4504BF03F1FF338AF80730C2
S3150800C570129BC3EBC303534400221A734FF0010105
S3150800C58059739A730AF104029A6008F1FF33DBB211
S3150800C5900E2B00F27581B8F10F0F66D8C8EBC803E9
S3150800C5A053441B7BC3F3C2035B4540F0728182E1AF
S3150800C5B0DDF840B0DDF84480D2E7009FAFE1009C8B
S3150800C5C0D8E1009D02E29AF80730434504BF03F11B
S3150800C5D0FF338AF80730CBEBCB0B0AEB0B034FF094
S3150800C5E000021A734FF0010159739A730AF1040293
S3150800C5F09A60631EDBB20E2B00F2A2810F2C09D8BB
S3150800C600C4EBC40353441B7BC3F3C203B34240F0D9
S3150800C6109F81ACE19AF80730B34204BF03F1FF33B8
S3150800C6208AF80730139BC3EBC303534400221A73DB
S3150800C6304FF0010159739A730AF104029A607B1E3E
S3150800C640DBB20E2B00F251810F2F09D8C7EBC703B7
S3150800C65053441B7BC3F3C2034B4540F04E815BE159
S3150800C660DDF840B0DDF844807AE70F9FD946DDF85B
S3150800C67038B042E75F46DDF82CB0D146DDF830A089
S3150800C68005E7DDF828805F46DDF824B0CA46C5E62A
S3150800C690DDF81C805F46DDF818B087E6D046DA4636
S3150800C6A0DDF810B060E64FF0D60B0AE04FF0D70B76
S3150800C6B007E04FF0D60B04E04FF0D60B01E04FF041
S3150800C6C0D40B584615B0BDE8F08F9AF81330C3F36B
S3150800C6D0C2035B453FF462AE4FF0010808F101035F
S3150800C6E0DBB25FFA83F8B8F10F0F3FF639AEC3EB4A
S3150800C6F0C3025244127BC2F3C20201339345F0D1FE
S3150800C700B8F1000F3FF445AECDF80880C8EBC80372
S3150800C71053441B7B13F0400F3FF450AEC8EBC803DD
S3150800C72053441B7B03F007074FF00109CDF818B0F7
S3150800C730CDF81C80BB46C84685E69AF81330C3F385
S3150800C740C2035B453FF461AEDDF80C8008F10103D6
S3150800C750DBB25FFA83F8B8F10F0F3FF622AEC3EBF0
S3150800C760C3025244127BC2F3C20201339345F0D18D
S3150800C770B8F1000F3FF443AECDF81480C8EBC803F8
S3150800C78053441B7B13F0400F3FF450AEC8EBC8036D
S3150800C79053441B7B03F00707DDF80C90CDF824B053
S3150800C7A0CDF82880BB465346CA46994684E699F88A
S3150800C7B01330C3F3C2035B453FF460AEDDF800A057
S3150800C7C00AF10103DBB25FFA83FABAF10F0F3FF6FB
S3150800C7D01FAEC3EBC3024A44127BC2F3C202013343
S3150800C7E09345F0D1BAF1000F3FF441AECDF820A041
S3150800C7F0CAEBCA034B441B7B13F0400F3FF44FAE02
S3150800C800CAEBCA034B441B7B03F00707DDF800801D
S3150800C810CDF82CB0CDF830A0BB464746CA4681E6CF
S3150800C8209AF81330C3F3C2035B453FF460AE009F2A
S3150800C8307B1CDBB2DFB20F2F3FF623AEC3EBC3027E
S3150800C8405244127BC2F3C20201339345F2D1002F40
S3150800C8503FF446AE0D97C7EBC70353441B7B13F053
S3150800C860400F3FF452AEC7EBC70353441B7B03F09C
S3150800C8700709DDF80080CDF838B00F97CB4684E677
S3150800C8809AF81330C3F3C2035B453FF462AEDDF892
S3150800C890008008F10103DBB25FFA83F8B8F10F0FE5
S3150800C8A03FF627AEC3EBC3025244127BC2F3C20261
S3150800C8B001339345F0D1B8F1000F3FF445AECDF8FA
S3150800C8C04880C8EBC80353441B7B13F0400F3FF462
S3150800C8D04FAEC8EBC80353441B7B03F00709009F00
S3150800C8E0CDF840B0CDF84480A9E69AF81330C3F3E2
S3150800C8F0C2034B453FF461AE009F7B1CDBB2DFB23F
S3150800C9000F2F3FF629AEC3EBC3025244127BC2F384
S3150800C910C20201339145F2D1002F3FF449AE139775
S3150800C920C7EBC70353441B7B13F0400F3FF47AAEA3
S3150800C930C7EBC70353441E7B06F00706009C58E660
S3150800C9409AF81330C3F3C203B3423FF438AE009CDF
S3150800C950631CDBB2DCB20F2C3FF65CAEC3EBC30242
S3150800C9605244127BC2F3C20201339642F2D1002C22
S3150800C9703FF450AEA346C4EBC40353441B7B13F0E9
S3150800C980400F3FF428AEC4EBC403534493F80C801D
S3150800C99008F00708009D1DE09AF81330C3F3C20398
S3150800C9A043453FF40EAE009D6B1CDBB2DDB20F2D86
S3150800C9B03FF609AEC3EBC3025244127BC2F3C2026E
S3150800C9C001339045F2D1002D3FF4FDAD294650467E
S3150800C9D0FEF713FF6B1EDBB20E2BDDD80F2D3FF6CD
S3150800C9E0F2ADC5EBC50353441B7BC3F3C2034345F2
S3150800C9F0DAD1E8E72DE9F04F8DB0064603910492A7
S3150800CA00984600218DF8181008238DF819300B4622
S3150800CA100F2262F387038DF81A3003681B6898475C
S3150800CA20002800F090800446056806AB036080F88D
S3150800CA30068007AB00931223002211463046FEF704
S3150800CA4063FE25600346002871D1BDF82490BDF821
S3150800CA5026A09DF8203005939DF8217000240CE04F
S3150800CA60CDF80080049B039A59463046FEF772FAC1
S3150800CA70D12825D10134102C26D05FFA84FB06EB89
S3150800CA808405A86F0028F5D003681B699847002815
S3150800CA90F0D1A86F03681B6A394698470028E9D081
S3150800CAA0A86F03689B695246494698470028D7D11C
S3150800CAB0A86F0368DB69059998470028DAD0CFE79D
S3150800CAC00346BBF10F0F32D9002402E00134102CC3
S3150800CAD031D05FFA84FB06EB8405A86F0028F5D0F1
S3150800CAE003681B6998470028F0D1A86F03681B6A7A
S3150800CAF03946984770B1A86F03689B6952464946FC
S3150800CB0098470028E2D1A86F0368DB69059998471A
S3150800CB100028DBD1CDF80080049B039A594630469D
S3150800CB20FEF718FA00F0F703D12BCFD003461846C4
S3150800CB300DB0BDE8F08F4346049A03993046FFF7D7
S3150800CB4064FB0346F3E7D623F1E7000010B5044675
S3150800CB50F821FEF75FFA00F0C00040282CD007D96C
S3150800CB60802810D0C02802D1204B01221A7010BD8F
S3150800CB700028FCD1D122D8212046FEF7C9F91B4B43
S3150800CB8000221A70F3E7D8212046FEF743FA10F080
S3150800CB90020F08D1C922D8212046FEF7B9F9134B4E
S3150800CBA002221A70E3E7CB22D8212046FEF7B0F915
S3150800CBB00E4B03221A70DAE7D8212046FEF72AFA26
S3150800CBC010F0020F08D1CB22D8212046FEF7A0F993
S3150800CBD0064B03221A70CAE7C922D8212046FEF757
S3150800CBE097F9024B02221A70C1E700BF20DB00202A
S3150800CBF02DE9F04107464FF40051684803F03EFC22
S3150800CC0038B1674B1B78032B41D8DFE803F01B15B7
S3150800CC102A270446C8213846FEF7FCF910F0200FEB
S3150800CC2005D12246C8213846FEF772F9E9E73846A3
S3150800CC30FFF78CFF2024F4E75A4B13221A704FF0A3
S3150800CC40000816E0574B1B7803F0F003102B21D091
S3150800CC50544B11221A704FF000080AE04FF00108F1
S3150800CC6001E04FF000084F4B1B7803F0F003102B40
S3150800CC7005D007F1740607F1B40534460FE002F053
S3150800CC80F5FC484BC830586020221A70F1E74FF07F
S3150800CC900008EEE74FF00008EBE7AC4207D054F87F
S3150800CCA0040F0028F9D00368DB689847F5E73D4B81
S3150800CCB01B78402B41D009D8202B2AD0302B32D0D4
S3150800CCC0112B38D1002387F8B83016E0512B4AD0FB
S3150800CCD0802B52D0502B2ED1C8213846FEF79AF910
S3150800CCE010F0400F27D02F4C5123237002F0BEFCC2
S3150800CCF0143060601FE0A64207D056F8040F0028DB
S3150800CD00F9D003689B689847F5E7264B12221A70F4
S3150800CD1011E002F0ABFC234B5B68C31A002B0ADB5D
S3150800CD20204B30221A700122E8213846FEF7F0F827
S3150800CD301C4B40221A70BDE8F081E8213846FEF700
S3150800CD4069F910F0010FF6D1D8213846FEF762F9D5
S3150800CD5040F00802D2B2D8213846FEF7D9F8114B6E
S3150800CD6050221A70E7E702F081FC0E4B5B68C31A83
S3150800CD70002BE0DB0B4B80221A704346002211463B
S3150800CD803846FFF737FE28B1D228D4D0054BA02263
S3150800CD901A70D0E7034B90221A70CCE700080240BD
S3150800CDA020DB0020140A00200368D3B130B40479CC
S3150800CDB0CCB113889BB10B681D7843791B1B04689B
S3150800CDC0E5540379013B03711388013B13800B6813
S3150800CDD001330B60047934B11388002BEBD10020A2
S3150800CDE004E00020704743790371012030BC704786
S3150800CDF07F281BD981B942F2AC03984213D00C4A5A
S3150800CE00012332F8021F814203D001339BB2802BE3
S3150800CE10F7D18033D8B27047FF2806D88038044B3C
S3150800CE2033F8100070470023F3E70020704700BF6F
S3150800CE30D03B0308612812D00A490122622398428E
S3150800CE4005D0013231F8023F002BF8D105E028B1B0
S3150800CE50054B03EB4202B2F8E00270477047002226
S3150800CE60F6E700BFD23C0308D03B030808B524F018
S3150800CE70D1FB08BD08B524F0D5FB08BD08B5044BA1
S3150800CE801A1803EB80035B685B68107A984708BD3D
S3150800CE903C0A002008B5084B1B5C53B9064B012217
S3150800CEA01A541A1803EB800043681B68107A9847CF
S3150800CEB008BD0020FCE700BF3C0A002038B5044C3A
S3150800CEC0251804EB800460688468287AA04738BD72
S3150800CED03C0A002038B5044C251804EB8004606829
S3150800CEE0C468287AA04738BD3C0A002010B5044B10
S3150800CEF01C1803EB80035B681B69207A984710BDF2
S3150800CF003C0A0020002070473AB101388A1811F807
S3150800CF10013B00F8013F9142F9D1704722B18218CE
S3150800CF2000F8011B8242FBD17047000010B4264B63
S3150800CF301B680BB3D0F8002293420DD00022224B77
S3150800CF40DB684BB3D0F80042A34217D032BB0229A4
S3150800CF500CBF0020122033E01B4B5A68D0F8083269
S3150800CF609A4201D00022EAE7174B1A89B0F806322E
S3150800CF709A4217D00022E2E70122E0E7124B1C6929
S3150800CF80D0F808329C42E1D10F4B9C8AB0F80632A1
S3150800CF909C42DBD1012206E00122D7E700200FE000
S3150800CFA010200DE000220029FAD153001A44064B3E
S3150800CFB003EB82035B89B3F5807F0CBF102000204A
S3150800CFC05DF8044B704700BF1C0A002070B4D0F807
S3150800CFD000222F4B1B689A420AD02D4CE4689442D3
S3150800CFE026D0002B34D02A4BDB687BB300201DE00B
S3150800CFF0274C6568D0F80842A542EED1244C25890D
S3150800D000B0F80642A542E8D10023002934D15A00D7
S3150800D010D1181F4A02EB81025089013080B25A00AA
S3150800D020D1181B4A02EB81025081581C70BC70470C
S3150800D030174C2569D0F80842A542D2D1144CA58AC6
S3150800D040B0F80642A542CCD10123DEE7012300E071
S3150800D05000230F4E5C001C44A40035193251D0F849
S3150800D06008226A60B0F806222A8100226A8100290D
S3150800D070CDD04FF48070D2E75A00D118044A02EB9B
S3150800D080810252890AB10020D0E74FF48070C6E7C2
S3150800D0901C0A00200138012814D800EB4003114A65
S3150800D0A002EB83035A8922F480739BB263B1013A77
S3150800D0B092B200EB40030B4901EB83035A8152B14C
S3150800D0C0002070470220704700EB4003054A02EB38
S3150800D0D0830300225A8100EB400083000020014AA6
S3150800D0E0D05070471C0A0020D0F82422131D490A84
S3150800D0F0D0F8000290F80202B1FBF0F1506848B18E
S3150800D100814205D3091A53F8080F20B18842F9D984
S3150800D1105868084470477047CA7E8B7E43EA0223E4
S3150800D12090F80022032A01D018467047487D0A7DE8
S3150800D13042EA002243EA0243F6E7024600F10B01FF
S3150800D1400020C30143EA500312F8010B50FA83F397
S3150800D150D8B28A42F5D170470168F1B110B40C789B
S3150800D1601F2C11D93A2C21D00A4612F8013F1F2B41
S3150800D1700CD93A2BF9D14B1C9A4211D1302C12D129
S3150800D18002310160002005E00A4623463A2B18BF03
S3150800D1900020F0D05DF8044B70474FF0FF30704721
S3150800D1A04FF0FF30F6E74FF0FF30F3E70A46E2E7C5
S3150800D1B090F804320BB9002070472DE9F041044677
S3150800D1C0D0F83052074601232A46014690F8010254
S3150800D1D0FFF780FEF0B9002384F80432D4F824322D
S3150800D1E0EB1AD4F81C22934217D294F80362012E44
S3150800D1F015D94FF00108D4F81C321D4443462A4677
S3150800D200394694F80102FFF765FE013E012EF2D178
S3150800D210002000E00120BDE8F0810020FBE70020A7
S3150800D220F9E770B5D0F830328B4214D004460D4673
S3150800D230FFF7BEFF064678B901232A46214694F829
S3150800D2400102FFF73BFE00281CBF01264FF0FF3501
S3150800D250C4F8305200E00026304670BD10B50446CA
S3150800D260002380F804324FF0FF33C0F83032FFF75E
S3150800D270D8FF80BB94F8FF2194F8FE3143EA0223D5
S3150800D2801BB2184A934228D194F8392094F83830BA
S3150800D2901B0443EA026394F83620134394F83720B4
S3150800D2A043EA022323F07F430F4A934217D094F8A8
S3150800D2B0553094F85400000440EA036094F852305C
S3150800D2C0184394F8533040EA032020F07F40801A30
S3150800D2D018BF012002E0032000E0022010BD002054
S3150800D2E0FCE700BF55AAFFFF46415400C8B108B580
S3150800D2F0D0F80032BBB193F80012B1B1B3F80612F8
S3150800D300B0F80422914201D0092008BD93F8010221
S3150800D310FFF7B4FD00F0010000280CBF002009202B
S3150800D320F3E7092070470920EFE70920EDE7000039
S3150800D3302DE9F04184B006461746002303600846E7
S3150800D340FFF70AFF051EC0F28581CD4B03EB850367
S3150800D3509C69002C00F08281346094F8003283B115
S3150800D36094F80102FFF78AFD10F0010F09D1002F8A
S3150800D37000F0768100F0040000280CBF00200A2087
S3150800D38069E1002384F80032E8B284F80102FFF765
S3150800D39081FD10F0010F40F065811FB110F0040FF8
S3150800D3A040F0628100212046FFF758FF0346012816
S3150800D3B000F0B7800026032B00F05881002B40F0C0
S3150800D3C05781227BE37A43EA02231BB2B3F5007F37
S3150800D3D040F05081E17DA37D53EA01210DD194F8F7
S3150800D3E0272094F826301B0443EA026394F8242085
S3150800D3F0134394F8251043EA0121C4F81C12227C31
S3150800D40084F80322531EDBB2012B00F23581657BBB
S3150800D41084F80252002D00F031816B1E2B4240F039
S3150800D4203781A37C607C40EA0320A4F8080210F048
S3150800D4300F0F40F02F81277DE37C53EA07230DD198
S3150800D44094F8237094F822301B0443EA076394F88F
S3150800D45020703B4394F8217043EA072394F80FC0E1
S3150800D460A77B57EA0C2C00F0178101FB02F20CEBA4
S3150800D47010171744BB42C0F01181DB1BB3FBF5F351
S3150800D480002B00F00D8140F6F575AB4294BF0125DF
S3150800D49002254FF6F57E734500F20C810233C4F877
S3150800D4A01832C4F82062B444C4F824C23744C4F815
S3150800D4B02C72032D00F00A81002800F0F7806244E0
S3150800D4C0C4F82822022D0FBF5B0003EB430203F0CA
S3150800D4D0010303EB520303F2FF13B1EB532FC0F022
S3150800D4E0E7804FF0FF33C4F81032C4F80C328023BB
S3150800D4F084F8053284F80052614A938B01339BB253
S3150800D5009383A4F806320023C4F8143213689C42A5
S3150800D51000F098805A4BDB689C4200F09780002008
S3150800D52099E023466D4604F140002946002705E0A8
S3150800D5303A4641F8042B1033834212D093F8C2219D
S3150800D540002AF5D093F8C96193F8C821120442EA73
S3150800D550066293F8C661324393F8C76142EA062227
S3150800D560E7E705F110074FF002080AE031462046C2
S3150800D570FFF774FE034600283FF423AFBD423FF48D
S3150800D5801AAF55F8046B002EF0D14346F6E7711C26
S3150800D5902046FFF746FE00284ED1002384F80532C0
S3150800D5A094F8FF2194F8FE3143EA02231BB2354A68
S3150800D5B0934201D003259DE7E278A3781B0443EA4A
S3150800D5C0026322781343627843EA02232E4A93427F
S3150800D5D034D194F8E72194F8E6311B0443EA026350
S3150800D5E094F8E421134394F8E52143EA0223274AF1
S3150800D5F0934225D194F8EB2194F8EA311B0443EAC7
S3150800D600026394F8E821134394F8E92143EA0223D4
S3150800D610C4F8103294F8EF2194F8EE311B0443EA6B
S3150800D620026394F8EC21134394F8ED2143EA0223AC
S3150800D630C4F80C3203255DE703255BE7032559E7A4
S3150800D640032557E7134600221A6063E70C4B0022AE
S3150800D650DA6064E70B2004B0BDE8F0810C20FAE735
S3150800D6600020F8E70320F6E70A20F4E70120F2E7AE
S3150800D6700D20F0E70D20EEE70D20ECE70D20EAE798
S3150800D6801C0A002055AAFFFF52526141727241617D
S3150800D6900D20E0E70D20DEE70D20DCE70D20DAE7B8
S3150800D6A00D20D8E70D20D6E70D20D4E70D20D2E7C8
S3150800D6B00D20D0E70233C4F81832C4F820620CEB08
S3150800D6C00602C4F824223744C4F82C720028E9D18B
S3150800D6D094F82F0094F82E20120442EA006294F877
S3150800D6E02C00024394F82D0042EA0022C4F82822AE
S3150800D6F09B0003F2FF13B1EB532FD5D34FF0FF3343
S3150800D700C4F81032C4F80C32802384F8053294F831
S3150800D710312094F8303043EA02231BB2012B3FF440
S3150800D72036AF0325E6E600BF2DE9F84F01F10905F6
S3150800D730D0F810328BB3D0F81462B64606F10B0C4B
S3150800D74032464FF02E094FF0E5084FF0100A63E015
S3150800D7506C1C85F80090A3F14105EDB2192D57D838
S3150800D76096F80CB055466DE02C4651E0F37A0B72EC
S3150800D770F27FB37F1B0443EA0263327F1343727F4F
S3150800D78043EA02230B60727E337E43EA02238B80D0
S3150800D790F27DB37D43EA0223CB8000232B708D698B
S3150800D7A035B3D0F8103203B3CC69FCB1B0F82422F3
S3150800D7B04FF6FF739A421DD0D0F820723888D8B138
S3150800D7C089466E1E0024A0464146FFF711FBA8B104
S3150800D7D0D9F81C30013BA34212D9013406F8010FCF
S3150800D7E037F814000028EFD100E0002400232B5559
S3150800D7F0BDE8F88F0024F9E70024F7E70024F5E7E9
S3150800D8000024F3E7A2EB0E03092B21D02C4643464E
S3150800D810651C23706245A9D012F8013B202BF9D06C
S3150800D820052BEFD0A2EB0E07092F91D0A3F14104E7
S3150800D830E4B2192C98D896F80CB02C46082F8CBF51
S3150800D8401025082515EA0B0FE2D02033DBB2DFE7F7
S3150800D8506C1C85F800904346DAE710B50446FFF7D6
S3150800D860A7FC034660B994F80032032B0AD00022BD
S3150800D870114694F80102FFF739FB031C18BF012370
S3150800D880184610BD94F80532012BF0D14FF40072FA
S3150800D89000212046FFF742FB552384F8FE31AA23D0
S3150800D8A084F8FF315223237063706123A3704122E9
S3150800D8B0E270722184F8E41184F8E51184F8E6210F
S3150800D8C084F8E731D4F8103284F8E831C3F3072234
S3150800D8D084F8E9211A0C84F8EA211B0E84F8EB3146
S3150800D8E0D4F80C3284F8EC31C3F3072284F8ED211E
S3150800D8F01A0C84F8EE211B0E84F8EF31D4F8202296
S3150800D9000132C4F830220123214694F80102FFF7B8
S3150800D910E1FA002384F80532A9E70239D0F818326B
S3150800D920023B8B4283BF90F80232D0F82C0201FBEF
S3150800D93003000020704701295BD9F8B5D0F81832E2
S3150800D9408B4258D90C46064690F80032022B28D04E
S3150800D950032B36D0012B01D001204DE001EB5105F8
S3150800D960D0F8241201EB5521FFF75BFC002844D1BF
S3150800D9706F1CC5F30805755DD6F8241201EB57210F
S3150800D9803046FFF74EFC00283AD1C7F30807F05D8A
S3150800D99045EA002014F0010F14BF0009C0F30B007C
S3150800D9A02AE0D0F8241201EB1421FFF73AFC50BB09
S3150800D9B0610001F4FF7173185B78705C40EA03201C
S3150800D9C01AE0D0F8241201EBD411FFF72AFCE8B9C3
S3150800D9D0A10001F4FE717218D07893781B0443EA0B
S3150800D9E00063705C1843537840EA032020F07040C7
S3150800D9F002E0012070470120F8BD4FF0FF30FBE739
S3150800DA004FF0FF30F8E74FF0FF30F5E74FF0FF3003
S3150800DA10F2E7F8B50646A0F80612D0F80842012C37
S3150800DA2046D00D46D0F80032D3F81822A24241D982
S3150800DA30FCB993F80022032A16D0B3F80822AA42A2
S3150800DA403AD9D3F82802C6F80C42E8B300EB151009
S3150800DA50C6F8100205F00F05D6F8003203EB451597
S3150800DA60C6F81452002026E0D3F82822002AE4D06B
S3150800DA70144693F802723F01BD4213D32146D6F8E5
S3150800DA800002FFF758FF0446B0F1FF3F16D0012801
S3150800DA9016D9D6F80032D3F81832834212D9ED1BBC
S3150800DAA0AF42EBD92146D6F80002FFF736FFCAE7A0
S3150800DAB0022000E00220F8BD0220FCE70120FAE778
S3150800DAC00220F8E70220F6E70220F4E72DE9F843FA
S3150800DAD0012940F28B80D0F818328B4240F28880B8
S3150800DAE016460C46054690F80032022B4DD0032BFD
S3150800DAF05FD0012B01D002277BE001EB5108D0F85B
S3150800DB00241201EB5821FFF78CFB0746002870D139
S3150800DB1008F10109C8F3080814F0010F1DD015F81B
S3150800DB20083003F00F0343EA061305F8083001230B
S3150800DB3085F80432D5F8241201EB59212846FFF757
S3150800DB4070FB002858D1C9F30809C6F3071605F86B
S3150800DB500960012385F804324BE005F808600123C3
S3150800DB6085F80432D5F8241201EB59212846FFF727
S3150800DB7058FB002842D1C9F3080915F8093023F0E3
S3150800DB800F03C6F303261E43E1E7D0F8241201EB80
S3150800DB901421FFF746FB074658BB610001F4FF71E5
S3150800DBA06E542944C6F307264E70012385F80432BD
S3150800DBB01FE0D0F8241201EBD411FFF732FB074619
S3150800DBC0B8B9A10001F4FE716B18DA78120602F0F2
S3150800DBD0704216436E54C6F307225A70320C9A7076
S3150800DBE0360EDE70012385F8043202E0022700E0D3
S3150800DBF002273846BDE8F8830746FAE70746F8E7F6
S3150800DC00F8B505460F4649B9D0F80C62A6B1D0F862
S3150800DC101832B34298BF012634461CE0FFF78BFE44
S3150800DC200346012849D9B0F1FF3F4BD0D5F8182251
S3150800DC30824247D83E46EFE70126EDE721462846C9
S3150800DC40FFF779FE034678B1B0F1FF3F3AD00128D5
S3150800DC5038D0B44235D00134D5F81832A342EDD8BD
S3150800DC60012E2CD90224E9E76FF070422146284696
S3150800DC70FFF72CFF0346D0B98FB9C5F80C42D5F883
S3150800DC801032B3F1FF3F1FD0013BC5F8103295F8AB
S3150800DC90053243F0010385F80532234612E0224691
S3150800DCA039462846FFF712FF03460028E5D0012B20
S3150800DCB00CBF4FF0FF33012304E0012302E00023E9
S3150800DCC000E000231846F8BD2346FBE72DE9F84394
S3150800DCD0B0F806526B1C9AB2002A00F08880D0F879
S3150800DCE01022002A00F085800F46044613F00F061E
S3150800DCF00BD10132C0F81022D0F80C1289B9D0F82D
S3150800DD000022B2F808229A4275D96B1CA4F806328A
S3150800DD10D4F8003203EB4613C4F814320020BDE8E9
S3150800DD20F883D0F8000290F80222013A12EA131892
S3150800DD30EBD1FFF700FE814601285ED9B0F1FF3F1F
S3150800DD405DD0D4F80002D0F818324B4545D8002FDC
S3150800DD5057D0D4F80C12FFF753FF8146002852D04B
S3150800DD60012852D0B0F1FF3F51D0D4F80002FFF796
S3150800DD701FFA08B10120D2E74FF400720021D4F847
S3150800DD800002FFF7CBF8D4F8007249463846FFF789
S3150800DD90C4FDC7F83002D4F8003293F80222B2B1B3
S3150800DDA0012783F80472D4F80002FFF701FA80BB52
S3150800DDB0D4F80022D2F830320133C2F8303208F1F2
S3150800DDC00108D4F8003293F802224245E9D8D3F87C
S3150800DDD03022A2EB0802C3F83022C4F80C92494656
S3150800DDE0D4F80002FFF799FDC4F810028DE7042065
S3150800DDF095E7042093E7042091E702208FE70120A6
S3150800DE008DE704208BE7072089E7022087E70120B2
S3150800DE1085E7012083E700002DE9F04F83B005462A
S3150800DE200021FFF7F6FD824600285BD14FF6FF7307
S3150800DE30A5F824324FF0FF09CB4698464F4609E02D
S3150800DE40A5F82482BB4600212846FFF73FFF8246F5
S3150800DE50002847D1D5F81012D5F80002FFF7E1F9E6
S3150800DE60824600283ED1D5F814422678002E00F0C6
S3150800DE708180E52EE4D0E37A03F03F0213F0080F21
S3150800DE8016D00F2ADCD1D5F820A2BAF1000FDAD0C5
S3150800DE9016F0400F2AD094F80D9006F0BF06B5F894
S3150800DEA00632A5F82432637B4B4524D0BB46CAE725
S3150800DEB00F2AE8D0BBF1000F04D12046FFF73DF941
S3150800DEC048450FD0D5F81832DA7A12F0010F4DD13D
S3150800DED004F10B0014F8011B13F8012B914245D1EC
S3150800DEE08442F7D1504603B0BDE8F08FB34518BF5A
S3150800DEF0BB46A8D1D7E7237823F04003013B03EBC1
S3150800DF00430203EB82030093DFF874B0012112E0A9
S3150800DF10FEF790FF0190009BFE2B17D85A1C009223
S3150800DF203AF81300FEF786FF0146019B83420DD19E
S3150800DF30124B9B450CD01BF8013BE2185278E35C68
S3150800DF4043EA02200029E3D14045F1D0BB467AE7EF
S3150800DF50237813F0400F05D021B1009B3AF813300F
S3150800DF60002BF3D1013E5FFA86FB6CE7A5F8248205
S3150800DF70BB4668E74FF0040AB4E700BF9D400308B4
S3150800DF80904003082DE9F04F83B005468A460B7882
S3150800DF902F2B08D05C2B06D0D0F80032D3F81432D9
S3150800DFA0C0F8083204E00AF1010A0023C5F808326D
S3150800DFB09AF800301F2B0BD800212846FFF729FDB9
S3150800DFC003460022C5F814225CE19A4600E09A4608
S3150800DFD0D046534613F8010B2F28F6D05C28F6D006
S3150800DFE0D5F8206280B21F2840F266812F2800F0FB
S3150800DFF069815C2800F07681B71E0124A1464FF09E
S3150800E0002A0B15E0002B40F0708127F8022F631CBD
S3150800E0101AF8010F1F2840F251812F2800F0548169
S3150800E0205C2800F05181B3F5807F00F05E811C46C4
S3150800E0304946FEF7DDFE0246002800F056817F2895
S3150800E040E3D8222800F01D815B46AA4998B290427F
S3150800E050D8D011F8013F002BF8D1D6E733882E2BFC
S3150800E06040F03D81002326F81430A34234BF2E2108
S3150800E0702021D5F81822D15401330B2BF5D1D5F828
S3150800E080183247F02007DF72A8E073882E2B40F07D
S3150800E090268133882E2B40F02281E3E7013C00F0ED
S3150800E0A0F08032F8023D202BF8D02E2BF6D0002C2B
S3150800E0B000F01B814FEA44084FF0000926F8149037
S3150800E0C00B222021D5F81802FEF728FFB11E4B4671
S3150800E0D000E0013331F8022F202AFAD02E2AF8D090
S3150800E0E00BB147F00307A8F1020806EB080236F859
S3150800E0F008102E2905D0013C03D032F8021D2E291E
S3150800E100F9D14FF0080B4FF00009CDF8049003F150
S3150800E110010836F8130000283CD020282ED02E28D7
S3150800E1201DD0D9452ED2A0451BD07F287BD82B28B9
S3150800E13000F088802C23704A99B2814200F08D80C5
S3150800E14012F8013F002BF7D1A0F141039BB2192B1E
S3150800E15000F28680019B43F00203019375E0A04517
S3150800E1600CD1BBF10B0F52D0019B9B00DBB2019384
S3150800E17023464FF00B0B4FF00809C8E747F0030793
S3150800E1804346C4E7BBF10B0F41D0A045ECD047F09E
S3150800E1900307E9D9D5F818321A78E52A40D0BBF131
S3150800E1A0080F69D0019A02F00C030C2B03D002F079
S3150800E1B00302032A01D147F0020717F0020F0AD11A
S3150800E1C0019A02F00302012A08BF47F01007042B40
S3150800E1D008BF47F00807D5F81832DF722846FFF758
S3150800E1E01BFED5F81832DA7A034600284ED112F00B
S3150800E1F0040F47D1D5F81412CB7A13F0100F59D063
S3150800E200D5F80002FEF788FFC5F80802E0E647F0F1
S3150800E2100307D5F818321A78E52AC3D14FF00B0B45
S3150800E22005221A70BBE70021FEF7E2FD0346002827
S3150800E2305DD0324A134413F8700C47F002070028E1
S3150800E2407FF475AF47F003075F20D5F8183203F857
S3150800E2500900434609F1010959E7002BF2D173E792
S3150800E260A0F161039BB2192BEFD8019B43F0010380
S3150800E2700193203880B2E8E7019B9B00DBB201934B
S3150800E28090E70623184603B0BDE8F08F042BF9D1B2
S3150800E29012F0200F08D00023C5F80832C5F814324A
S3150800E2A012F0040FEED193E602F00402002A08BF2A
S3150800E2B00523E7E70523E5E70123002408EB030A1E
S3150800E2C0042704E00123002408EB030A0027012C95
S3150800E2D03FF4C4AE022C3FF4D8AE002CD1D006EBE6
S3150800E2E04402DEE601230024EEE70623CAE747F0E8
S3150800E2F00207A7E741BB03084DBB03089040030884
S3150800E3002DE9F04F89B00446D0F81872D0F820925B
S3150800E3100C22394605A8FEF7F7FD9DF81F3013F0C5
S3150800E320200F40F0108113F0010F78D00023FB7204
S3150800E330C4F820320B2205A93846FEF7E5FD01256B
S3150800E3402B464FF07E0A4FF0200800E02B460DF1D1
S3150800E3501306072203F00F0000F13001392988BFA0
S3150800E36000F13701013A06F801191B09F2D108A98B
S3150800E370114401F814AC5AB1397820290BD0394622
S3150800E38001339A4206D011F8010F2028F8D102E08D
S3150800E390134600E01346591E394405E0404601334A
S3150800E3A001F8010F072B07D8072AF7D808A8104441
S3150800E3B010F8140C0132F2E72046FFF72DFD064649
S3150800E3C010BB0135642D1DD00B2205A93846FEF772
S3150800E3D09BFD052DBAD9A9F102062B4636F8022F60
S3150800E3E0002AB4D0102102F0010000EB43035208C2
S3150800E3F013F4803F1CBF83F4883383F0210301396B
S3150800E400F1D1EBE70726C1E0642D00F09E800428D1
S3150800E41040F0BC809DF81F30FB72C4F820929DF82E
S3150800E4201F3013F0020F1CD0B9F80030BBB100231F
S3150800E430013339F8022F002AFAD103F11905684B7E
S3150800E440A3FB0535AD0800212046FFF7E2FA06468C
S3150800E450002840F0988000274FF001080FE00023BD
S3150800E460EBE70125EFE70137BD4200F0938041460F
S3150800E4702046FFF72BFC0646002840F08480D4F897
S3150800E4801012D4F80002FEF7CCFE064600287AD110
S3150800E490D4F814321B78E52BE5D0002BE3D00027FF
S3150800E4A0E5E7B4F80612491B2046FFF7B2FA064616
S3150800E4B000286BD1D4F81802FEF73FFE009000271B
S3150800E4C001971AE0614649E04FF6FF72934202D07F
S3150800E4D038F811300BB94AF0400A80F800A0D4F891
S3150800E4E00032012283F8042239462046FFF7EEFB64
S3150800E4F0064600284AD1013D4ED0D4F81012D4F869
S3150800E5000002FEF78EFE064600283FD1D4F8208288
S3150800E510D4F814025FFA85FA009B43734FF00F0391
S3150800E520C37207738776C7760AF1FF3101EB410399
S3150800E53001EB83012B4A02F10D0E019B4FF6FF7684
S3150800E5404FF0FF090DE0062620E007261EE092F8A8
S3150800E55000C000F80C9084448CF801900132724592
S3150800E560B2D0B342F3D001F1010C38F8113011786A
S3150800E570435401444FEA132B81F801B0002BA1D173
S3150800E58061463346EAE7042E08BF0726304609B037
S3150800E590BDE8F08F013D84D1D4F81012D4F80002FA
S3150800E5A0FEF73FFE06460028F0D120220021D4F8C7
S3150800E5B01402FEF7B3FC0B22D4F81812D4F814028E
S3150800E5C0FEF7A2FCD4F81422D4F81832DB7A03F04A
S3150800E5D018031373D4F80032012283F80422D5E70E
S3150800E5E04FECC44E9040030801292ED9F8B50446CD
S3150800E5F00E46D0F818328B422AD900270DE001338F
S3150800E600C4F8103294F8053243F0010384F8053251
S3150800E6102E46D4F81832AB421BD931462046FFF7AE
S3150800E6208AF90546B8B1012817D0B0F1FF3F16D0D0
S3150800E6303A4631462046FFF749FA024648B9D4F821
S3150800E6401032B3F1FF3FDAD1E2E7022210467047F3
S3150800E65002221046F8BD0022FBE70222F9E7012252
S3150800E660F7E7000010B584B001900091144604A89D
S3150800E67040F8041DFEF770FD00282BDB194B03EB51
S3150800E68080039B6953B1174A1268934214D0154AFE
S3150800E690D268934214D0002283F80022019BDBB192
S3150800E6A0002283F800220F4A02EB80008361012CC6
S3150800E6B00AD0002004B010BD0A4A00211160E6E71E
S3150800E6C0084A0021D160E6E70022694601A8FEF75C
S3150800E6D02FFEEFE70B20EDE7024B03EB800300204C
S3150800E6E09861E7E71C0A00202DE9F047ADF5107D93
S3150800E6F00191002800F0BC80044615460023C0F8A6
S3150800E700003202F01E0201A986A8FEF711FE06468F
S3150800E71020B130460DF5107DBDE8F0874FF4007046
S3150800E720FEF7A4FB8146002800F0A48005F01F0828
S3150800E7308E9003AB8C93019906A8FFF723FC8B9F59
S3150800E7408246002840F09880002F00F0C58038F0F7
S3150800E750010314BF0121002106A8FEF7E7FB824644
S3150800E76015F01C0F5CD048B9FB7A13F0110F40F076
S3150800E770C68015F0040F0AD00826B6E0BAF1040FD1
S3150800E78030D048F008088B9FBAF1000F38D118F03E
S3150800E790080F56D0FEF7B6FBB873C0F30723FB7312
S3150800E7A0030C3B74000E78740025FD723D777D7767
S3150800E7B0BD77FD7739468698FEF7AEFCBD76FD76C1
S3150800E7C03D757D75869B012283F80422054600283F
S3150800E7D035D0D3F830A201461846FFF705FF88B1B1
S3150800E7E0064691E04B4B1B682BB14A4BDB684FF052
S3150800E7F0120A002BC5D106A8FFF782FD8246C0E79C
S3150800E800564681E08698013DC0F80C525146FEF7FF
S3150800E81008FD054698B14846FEF72CFB2E4678E7D4
S3150800E82000286ED1FB7A13F0100F6CD115F0020F89
S3150800E83002D013F0010F6BD115F0080F01D048F084
S3150800E8402008869BD3F83032C4F81C32C4F82072EC
S3150800E85038F0010314BF0121002106A8FEF7B6FB14
S3150800E860C4F8280200283FD04846FEF703FB0DE00F
S3150800E87009264EE711264CE715F01C0F7FF47EAFEC
S3150800E8804846FEF7F7FABAF1000F2BD184F806824C
S3150800E890002584F80752DDF8188239464046FEF707
S3150800E8A03BFCC4F81002FA7FBB7F1B0443EA0263F1
S3150800E8B03A7F13437A7F43EA0223C4F80C32C4F83A
S3150800E8C00852C4F81852C4F82452C4F80082B8F89A
S3150800E8D00632A4F804321CE715F01C0F09D14FF0D4
S3150800E8E0060ACDE7564614E702264846FEF7C2FA58
S3150800E8F00FE748F008088B9F4FF0060AC0E707267F
S3150800E900F3E7064600E004264846FEF7B3FA00E7B2
S3150800E9100726F9E71C0A00202DE9F04F83B00446C4
S3150800E9208846164699460023C9F80030FEF7DEFCED
S3150800E9300190002840F0F98094F80732002B40F047
S3150800E940F38094F8063213F0020F00F0F280D4F840
S3150800E9500832F34202D2002E40F0BB80D4F80832C7
S3150800E960D4F80C22934288BFC4F80C3294F80632C5
S3150800E97043F0200384F80632D7E0D4F82432C3B330
S3150800E9802046FEF7B1FB0028E8D0012837D0B0F1C1
S3150800E990FF3F39D0C4F81402D4F810320BB9C4F8C2
S3150800E9A0100294F8063213F0400F32D1D4F800A2C0
S3150800E9B0D4F814125046FEF7B0FF054600283FD09B
S3150800E9C03D445FEA562B56D09AF8023207EB0B0203
S3150800E9D09A4288BFA3EB070B5B462A4641469AF83C
S3150800E9E00102FEF777FA80B3012384F80732019310
S3150800E9F09BE0D4F814121046FFF702F9C3E7022386
S3150800EA0084F80732019390E0012384F807320193D2
S3150800EA108BE0D4F800020123D4F81822214690F896
S3150800EA200102FEF757FA30B994F8063223F040038C
S3150800EA3084F80632BAE7012384F80732019374E0B2
S3150800EA40022384F8073201936FE0D4F81812491BA1
S3150800EA50594502D34FEA4B252DE04FF4007208EBD7
S3150800EA6041212046FEF750FA94F8063223F0400377
S3150800EA7084F80632EEE7D4F81832AB4205D0D4F85B
S3150800EA800822D4F80C329A4240D3C4F81852D4F863
S3150800EA900802C0F30800C0F50075B54228BF354620
S3150800EAA02A4641462044FEF72FFA94F8063243F0E8
S3150800EAB0400384F80632A844D4F808322B44C4F834
S3150800EAC00832D9F800302B44C9F80030761B3FF4D9
S3150800EAD045AFD4F80812C1F30803002BD7D1D4F8F0
S3150800EAE0002292F80232013B03EA512313F0FF0792
S3150800EAF07FF457AF00297FF440AFD4F810020028FE
S3150800EB007FF443AF1046FFF77BF83CE701232A461C
S3150800EB1021469AF80102FEF7D1F90028B5D001235B
S3150800EB2084F80732019300E00193019803B0BDE829
S3150800EB30F08F07230193F8E738B50446FEF7D6FBAE
S3150800EB40034608BB94F8062212F0200F1CD012F0D8
S3150800EB50400F11D0D4F800020123D4F81822214618
S3150800EB6090F80102FEF7B6F900284AD194F8063261
S3150800EB7023F0400384F80632D4F81C12D4F80002B5
S3150800EB80FEF74FFB034608B1184638BDD4F82052A5
S3150800EB90EB7A43F02003EB72D4F80C322B77B4F8F7
S3150800EBA00C321B0A6B77B4F80E32AB7794F80F3237
S3150800EBB0EB77D4F81032AB76C3F30722EA761B0C50
S3150800EBC02B751B0A6B75FEF79DF9A875C0F307230D
S3150800EBD0EB75030C2B76000E68760023AB74EB748A
S3150800EBE094F8063223F0200384F80632D4F800326B
S3150800EBF0012283F80422D4F80002FEF72EFE03460B
S3150800EC00C2E70123C0E710B50446FFF795FF0346A0
S3150800EC1008B1184610BD2046FEF768FB03460028D3
S3150800EC20F7D1D4F82802FEF735FA03460028F0D1C2
S3150800EC300022C4F80022ECE770B5ADF5107D01900E
S3150800EC400D46002201A986A8FEF772FB044618B1F4
S3150800EC5020460DF5107D70BD4FF40070FEF706F9DD
S3150800EC600646A8B18E9003AB8C93019906A8FFF7C8
S3150800EC7089F9044630B98B9B43B11DB1294606A8CC
S3150800EC80FEF752FD3046FEF7F5F8E1E70624F9E708
S3150800EC901124DDE72DE9F04FADF5117D0190FEF762
S3150800ECA031F90546012201A986A8FEF741FB04466B
S3150800ECB020B120460DF5117DBDE8F08F4FF40070A8
S3150800ECC0FEF7D4F80646002800F0CA808E9003ABFB
S3150800ECD08C93019906A8FFF755F90446002800F019
S3150800ECE0C180042840F0BF808C9BDB7A13F0200F8C
S3150800ECF040F0B48000218698FEF782FF0746002878
S3150800ED0000F0A680012F1ED10224002C40F0A1801D
S3150800ED108B9B1022DA729D75C5F30722DA752A0CC9
S3150800ED201A762D0E5D769F76C7F30722DA763F0CA4
S3150800ED301F753F0A5F758698012380F80432FEF72F
S3150800ED408CFD04468FE0B7F1FF3F01D1012480E036
S3150800ED508698FEF72DFA044600287AD1DDF818823F
S3150800ED6039464046FEF7D9FD0446CDF800804FF4F3
S3150800ED70007200214046FEF7D1F80B2220214046BA
S3150800ED80FEF7CCF84FF02E0988F80090102388F883
S3150800ED900B3088F81650C5F3072388F817302B0C64
S3150800EDA088F818302B0E88F8193088F81A70C7F3C7
S3150800EDB0072388F81B303B0C88F814301B0A88F8A0
S3150800EDC015302022414608EB0200FEF79DF888F828
S3150800EDD02190889B869A92F80012032932D088F8E7
S3150800EDE03A30C3F3072288F83B201B0C88F83430E6
S3150800EDF01B0A88F83530869B93F80232EBB103F18B
S3150800EE00FF395FFA89F909F10109A1444FF0010AAE
S3150800EE104FF4007B04F101088698C0F8304280F868
S3150800EE2004A2FEF7C5F9044698B95A460021009887
S3150800EE30FEF774F84446C145ECD106A8FFF760FA18
S3150800EE40044662E7D2F828229A4208BF0023C6E79A
S3150800EE50072439468698FFF7C7FB04E0062402E034
S3150800EE60112426E708243046FEF704F821E70000B7
S3150800EE702DE9F04F89B00590012903D9132009B06F
S3150800EE80BDE8F08F0C46164605A8FEF765F900287A
S3150800EE90C0F26382D04B03EB80039F69002F00F01A
S3150800EEA05E82002387F80032C5B22846FDF7F2FFD6
S3150800EEB010F0010F40F0558210F0040F40F0538215
S3150800EEC006AA01212846FEF711F8002840F04D82CF
S3150800EED0069A7F2A40F24B82002C14BF4FF0000A94
S3150800EEE04FF03F0AA2EB0A020692731E334202D182
S3150800EEF0002E40F04E82B948A0FB0230C009B0F59A
S3150800EF00806F14D2B6490023013331F8026FB0423C
S3150800EF10FAD3B44901EB4303B3F8A860B6F5007F0A
S3150800EF2000D3760A002E40F03882012638E24FF4E4
S3150800EF300046F6E703EB430303F101084FEA5808D6
S3150800EF4008F10308012300938AE29B44039A1A44B2
S3150800EF500392069BA3EB0B03A3EB0803019A9B1AE8
S3150800EF60B3FBF6F31A4604934FF6F5739A4240F24A
S3150800EF7002824FF00C090BE040F6F573994240F215
S3150800EF80FC81B2F5803F34BF4FF004094FF0060903
S3150800EF90002C48D14FF4007200213846FDF7BEFF19
S3150800EFA0012387F8BF3187F8C031002287F8C121CD
S3150800EFB087F8C291FE2187F8C31106980AEB000468
S3150800EFC08949A1FB04C1641A01EB54014C0B07944F
S3150800EFD0C90B41F03F0187F8C41187F8C5413F21A5
S3150800EFE087F8C61187F8C72187F8C82187F8C92185
S3150800EFF087F8CA01C0F3072187F8CB11010C87F8F7
S3150800F000CC11000E87F8CD01552187F8FE11AA21EB
S3150800F01087F8FF1139462846FDF75CFF002840F0BF
S3150800F020AE81F82400E0F02402974FF40072002124
S3150800F0303846FDF773FF0B226C493846FDF764FF27
S3150800F0400023FB7202233B737E7387F80EB0CBF363
S3150800F050072B87F80FB001233B74009B032B4FF057
S3150800F06000037B7418BF0223BB74069BB3F5803F6D
S3150800F07080F0A580FB74C3F307233B757C753F239B
S3150800F0803B7600237B76FF22BA76FB7687F81CA0B0
S3150800F0907B77BB77FB77FDF735FF0790009B032B44
S3150800F0A000F0AA8087F82700C0F3072387F82830DE
S3150800F0B0030C87F82930000E87F82A0087F816808F
S3150800F0C0C8F30723FB75802387F82430292387F89C
S3150800F0D026301322464907F12B00FDF715FF552365
S3150800F0E087F8FE31AA2387F8FF31012352463946AD
S3150800F0F02846FDF7EFFE002840F043814FF40072E2
S3150800F10000213846FDF70AFF009B012B394B18BF33
S3150800F1106FF0FF031C4307943C70BDF81C301B0AB4
S3150800F1207B70BDF81E30BB709DF81F30FB70039ACC
S3150800F130541C012339462846FDF7CCFE002840F02A
S3150800F14022814FF4007200213846FDF7E7FE0123BD
S3150800F1500793984540F2C0809B46224602F1010972
S3150800F1605B4602992846FDF7B5FE002840F00D815A
S3150800F170079B013307934A464345EFD3019B009A01
S3150800F180032A18BF1E4601244A4602F101082346EF
S3150800F19002992846FDF79EFE002840F0F880424670
S3150800F1A0013EF2D1009B032B00F098800022114605
S3150800F1B02846FDF79BFE003018BF01205FE687F85A
S3150800F1C02030C3F3072287F821201A0C87F822205B
S3150800F1D01B0E87F8233051E71C0A0020D34D621016
S3150800F1E020410308904003085B56150554BB0308E5
S3150800F1F074BB030800FFFF0087F84300C0F307232A
S3150800F20087F84430030C87F84530000E87F8460027
S3150800F21087F82480C8F3072387F825304FEA184370
S3150800F22087F826304FEA186387F82730022387F8CD
S3150800F2302C30002387F82D3087F82E3087F82F30AA
S3150800F2404FF0010987F8309087F83130062287F8A1
S3150800F250322087F83330802387F84030292387F80F
S3150800F26042301322834907F14700FDF74DFE552327
S3150800F27087F8FE31AA2387F8FF314B4652463946AE
S3150800F2802846FDF727FE08B10120F8E501230AF113
S3150800F290060239462846FDF71DFE4FF40072002186
S3150800F2A03846FDF73BFE64F0FF0407943C70BDF852
S3150800F2B01C301B0A7B70BDF81E30BB709DF81F30D2
S3150800F2C0FB70FF233B717B71BB71FB713B727B72D9
S3150800F2D0BB720F23FB722AE7A1464FE752233B7006
S3150800F2E07B706123BB704122FA70722187F8E411A2
S3150800F2F087F8E51187F8E62187F8E731049A531E5F
S3150800F30087F8E831531EC3F3072387F8E931531EFC
S3150800F3101A0C87F8EA211B0E87F8EB31022387F8C7
S3150800F320EC31002387F8ED3187F8EE3187F8EF31B5
S3150800F330552387F8FE31AA2387F8FF3101230AEB04
S3150800F340030239462846FDF7C5FD01230AF10702DF
S3150800F35039462846FDF7BEFD28E70B208FE50C2029
S3150800F3608DE503208BE50A2089E5012087E5012044
S3150800F37085E50E2083E50E2081E50E207FE5012038
S3150800F3807DE501207BE5012079E5012077E501206F
S3150800F39075E5B6F5007FBFF4C4AD802E28BF80267C
S3150800F3A0B2FBF6F340F6F5718B424FD84FF6F5717E
S3150800F3B08B427FF6BFAD4FEA830808F207284FEA6B
S3150800F3C0582803230093002301934FF0200B0BEBDF
S3150800F3D00A030393019908EB01099944A6EB0A036A
S3150800F3E04B449A42C5D307AA03212846FDF77EFD5A
S3150800F3F020B9079B013BB3F5004F01D301230793BF
S3150800F400079A531E4B4452421340A3EB0903079332
S3150800F410009A032A3FF499AD9844069AA2EB0B0387
S3150800F420A3EB080301995B1AB3FBF6F10491009B61
S3150800F430022B3FF4A1AD009B012B7FF4A2ADB2F5E0
S3150800F440803F34BF99464FF00609A1E54FF6F5719E
S3150800F4508B42B0D803F102084FEA4808022300930A
S3150800F46008F2FF184FEA5828202301934FF0010BA2
S3150800F470ADE700BF60BB0308114B5B7ADBB2012B1B
S3150800F48001D90120704730B40D4C657AEDB20023DE
S3150800F4906355657A04EB85056860607A20440272D4
S3150800F4A0627AD2B2501CC0B2607230320A703A2206
S3150800F4B04A702F228A70CB70184630BC704700BF3E
S3150800F4C03C0A002008B50022FFF7D6FF08BD000059
S3150800F4D00D4B5B7A9BB10378303BDBB20A4A02EBF1
S3150800F4E0830252686AB1084A02EB83010020486029
S3150800F4F013441872537A013BDBB2537270470120EA
S3150800F50070470120704700BF3C0A002008B500215B
S3150800F510FFF7DEFF08BD000008B5074B01221A7089
S3150800F52006F0DEFC20B9044A137803F0FE031370D4
S3150800F530014B187808BD00BF0000002008B5074B2E
S3150800F54001221A7006F012FD20B9044A137803F056
S3150800F550FE031370014B187808BD00BF0000002099
S3150800F56000B583B001934FF4007300935202002351
S3150800F570084606F0A7FB003018BF012003B05DF867
S3150800F58004FB00B583B001934FF400730093520255
S3150800F5900023084606F0A8FB003018BF012003B078
S3150800F5A05DF804FB144B1B7813F0010F20D10329D7
S3150800F5B003D8DFE801F01F0413180420704710B5BC
S3150800F5C096B01446684606F0D9FC129B5B0A139A55
S3150800F5D043EAC2532360002016B010BD4FF40073EF
S3150800F5E01380002070474FF40073136001207047A2
S3150800F5F003207047002070470000002010B504461D
S3150800F600074B1868074BA3FB0030800900F00EFB78
S3150800F610002221464FF0FF3000F0BCFA002010BD52
S3150800F62004000020D34D621008B50B4B1A6842F44B
S3150800F63000721A601A6842F480621A601A6842F404
S3150800F64080721A60032000F093FA0020FFF7D6FFB5
S3150800F65020F0B0F9002008BD003C0240024A1368B9
S3150800F66001331360704700BF54DB0020014B186854
S3150800F670704700BF54DB002010B582B00190FFF739
S3150800F680F5FF0446FFF7F2FF019B001B9842F9D3EA
S3150800F69002B010BD70470000002800F0BC8010B50D
S3150800F6A00446036C43B1236C13F0100F0AD00120F3
S3150800F6B0002384F83C3010BD436480F83C30FFF7E3
S3150800F6C0E9FFF0E7236C23F4885323F0020343F0A1
S3150800F6D002032364514B5A6822F440325A605A682E
S3150800F6E061680A435A602268536823F4807353603A
S3150800F6F022685368216943EA0123536022685368E4
S3150800F70023F04073536022685368A1680B43536023
S3150800F7102268936823F40063936022689368E1681B
S3150800F7200B439360A26A3E4B9A4251D02268936873
S3150800F73023F07063936022689368A16A0B43936011
S3150800F7402268936823F04053936022689368E16ABD
S3150800F7500B4393602268936823F002039360226840
S3150800F7609368A16943EA41039360236A002B3AD15F
S3150800F7702268536823F4006353602268D36A23F42B
S3150800F7807003D3622168CB6AE269013A43EA0253FD
S3150800F790CB622268936823F40073936022689368A7
S3150800F7A0216B43EA412393602268936823F48063BC
S3150800F7B0936022689368616943EA81239360002015
S3150800F7C06064236C23F0030343F0010323646FE7AB
S3150800F7D02268936823F0706393602268936823F025
S3150800F7E040539360B6E72268536843F40063536056
S3150800F7F02268536823F4604353604FF4604393FAD6
S3150800F800A3F3B3FA83F221684868636A013B93401D
S3150800F81003434B60B1E70120704700BF0023014056
S3150800F8200100000F82B00023019390F83C30012BB1
S3150800F83063D0012380F83C3003689A6812F0010F00
S3150800F84014D19A6842F001029A60304B1B68304A1C
S3150800F850A2FB03239B0C03EB43030193019B2BB1F0
S3150800F860019B013B0193019B002BF9D10268936828
S3150800F87013F0010F43D0036C23F4E06323F0010374
S3150800F88043F480730364536813F4806F05D0036CE4
S3150800F89023F4405343F480530364036C13F4805FEA
S3150800F8A01ABF436C23F0060300234364002380F841
S3150800F8B03C306FF022031360164B5B6813F01F0F82
S3150800F8C00AD103689A6812F0405F1BD19A6842F021
S3150800F8D080429A60002013E002680F4B9A4201D0DA
S3150800F8E000200DE09B6813F0405F0DD10A4A93682B
S3150800F8F043F080439360002002E0022000E00020ED
S3150800F90002B070470020FBE70020F9E7040000205A
S3150800F91083DE1B43002301400020014003689A68E8
S3150800F92012F4806F03D09B6813F4807F1CD170B5E6
S3150800F9300C460546FFF79AFE06462A68136813F032
S3150800F940020F1AD1B4F1FF3FF8D024B1FFF78EFEAB
S3150800F950801BA042F1D92B6C43F004032B640023CF
S3150800F96085F83C3003202DE0036C43F02003036444
S3150800F970002380F83C30012070476FF012031360B3
S3150800F9802B6C43F400732B642B689A6812F0405F63
S3150800F99017D1AA69BAB9DA6A12F4700F03D09B684C
S3150800F9A013F4806F11D12B6C23F480732B642B6CAA
S3150800F9B013F4805F0BD12B6C43F001032B640020FA
S3150800F9C000E0002070BD0020FCE70020FAE70020D8
S3150800F9D0F8E70368D86C704730B482B00023019307
S3150800F9E090F83C30012B00F0B680012380F83C30BB
S3150800F9F00B68092B3AD90568EA689BB203EB4303FF
S3150800FA001E3B072404FA03F322EA0303EB600468A7
S3150800FA10E5680B8803EB43031E3B8A6802FA03F387
S3150800FA202B43E3604B68062B35D805686A6B03EBF6
S3150800FA308303053B1F2404FA03F322EA03036B63DB
S3150800FA400468656B0A884B6803EB8303053B02FA77
S3150800FA5003F32B4363630268404B9A424BD000235F
S3150800FA6080F83C30184602B030BC704705682A69F1
S3150800FA709BB203EB4303072404FA03F322EA0303C6
S3150800FA802B61046825690B8803EB43028B68934056
S3150800FA902B432361C6E70C2B16D805682A6B03EBA4
S3150800FAA08303233B1F2404FA03F322EA03032B638D
S3150800FAB00468256B0A884B6803EB8303233B02FA29
S3150800FAC003F32B432363C6E70568EA6A03EB83035C
S3150800FAD0413B1F2404FA03F322EA0303EB6204689A
S3150800FAE0E56A0A884B6803EB8303413B02FA03F392
S3150800FAF02B43E362AFE70B68122B22D00B68184A38
S3150800FB00934201D0112BAAD1164A536843F4000335
S3150800FB1053600A68124B9A42A1D1134B1B68134AC9
S3150800FB20A2FB03239B0C03EB83035B000193019B5E
S3150800FB30002B94D0019B013B0193019B002BF9D12B
S3150800FB408DE7084A536843F4800353600268034B01
S3150800FB509A42D3D083E7022085E700BF0020014000
S3150800FB6012000010002301400400002083DE1B431E
S3150800FB70074AD36823F4E0631B041B0C43F0BF63F6
S3150800FB8043F40033000200F4E0600343D360704797
S3150800FB9000ED00E030B4164BDB68C3F30223C3F173
S3150800FBA00704042C28BF04241D1D062D8CBF033B07
S3150800FBB000234FF0FF3505FA04F421EA04019940C1
S3150800FBC005FA03F322EA03031943002809DB0901AE
S3150800FBD0C9B200F1604000F5614080F8001330BCFE
S3150800FBE0704700F00F000901C9B2024B1954F6E735
S3150800FBF000ED00E014ED00E0420900F01F000123CB
S3150800FC0003FA00F0014B43F82200704700E100E0D8
S3150800FC10430900F01F00012202FA00F02033024ACD
S3150800FC2042F82300704700BF00E100E00138B0F158
S3150800FC30807F0AD2064B5860064AF02182F82310C4
S3150800FC400020986007221A6070470120704700BF9D
S3150800FC5010E000E000ED00E0430900F01F0001227B
S3150800FC6002FA00F06033024A42F82300704700BFE8
S3150800FC7000E100E00428044A13680CBF43F00403BB
S3150800FC8023F004031360704710E000E0704708B5DE
S3150800FC90FFF7FCFF08BD00000268D3B2103B084915
S3150800FCA0A1FB03131B090749C95CC165032B22F491
S3150800FCB07F7222F0030288BF04328265806D704726
S3150800FCC0ABAAAAAA6441030838B50446FFF7CEFCD6
S3150800FCD0002C00F093800546002384F83430022374
S3150800FCE084F835302268136823F00103136023680B
S3150800FCF01A6812F0010F0AD0FFF7B8FC401B052856
S3150800FD00F5D920236365032084F8350038BD1A68C1
S3150800FD103B4810406168A2680A43E1680A432169C2
S3150800FD200A4361690A43A1690A43E1690A43216AE8
S3150800FD300A430243616A042912D01A6021684B6992
S3150800FD4023F00703626A1343042A15D1A26AA0693D
S3150800FD5060BB012A1ED042B1022A22D0002008E048
S3150800FD60E16A206B01430A43E7E794F82F0000F0A5
S3150800FD70010000283CD113434B612046FFF78CFF56
S3150800FD80E26D3F239340836000206065012384F879
S3150800FD903530BBE7E06AB0F1C07F14BF0020012010
S3150800FDA0E7E794F82F0000F00100E2E7B0F5005FFE
S3150800FDB008D0022A1CD9032A18D194F82F0000F07B
S3150800FDC00100D6E7032A0FD8DFE802F0120212076D
S3150800FDD094F82F0000F00100CBE7E06AB0F1C07F8D
S3150800FDE014BF00200120C4E70020C2E70020C0E7B6
S3150800FDF040236365012084F8350087E7012085E7FD
S3150800FE003F8010F030B338B5044690F83530DBB291
S3150800FE10022B21D00268136823F0010313600368DC
S3150800FE2000251D6003685D6003689D600368DD60EA
S3150800FE3003681D61036821225A61FFF72DFFE26DF1
S3150800FE403F2393408360656584F8355084F83450C1
S3150800FE50284638BD012070470220FAE770B490F8AA
S3150800FE603440012C42D0856D012480F8344090F846
S3150800FE703540E4B2012C05D0002380F83430022046
S3150800FE8070BC7047022480F8354000244465066833
S3150800FE90346824F480243460046863608368402BE3
S3150800FEA01FD0036899600368DA60C26D3F239340E8
S3150800FEB0AB600268136843F016031360026853695F
S3150800FEC043F080035361036C23B10268136843F05F
S3150800FED0080313600268136843F0010313600020E7
S3150800FEE0CEE703689A600368D960DEE70220C7E7B1
S3150800FEF070B50446866DFFF7B9FB94F83530DBB26A
S3150800FF00022B06D080236365002384F83430012051
S3150800FF1070BD05462268136823F01603136022682D
S3150800FF20536923F080035361236CE3B12268136895
S3150800FF3023F0080313602268136823F00103136093
S3150800FF4023681B6813F0010F11D0FFF78FFB401BC6
S3150800FF500528F5D920236365002384F83430032067
S3150800FF6084F83500D4E7A36C002BDFD1E3E7E26D14
S3150800FF703F239340B360002084F83400012384F8BB
S3150800FF803530C5E790F83530DBB2022B03D0802335
S3150800FF90436501207047052380F8353002681368E9
S3150800FFA023F001031360002070470000F0B583B00A
S3150800FFB0044600230193724B1E68876D3D68C26D27
S3150800FFC0082393402B4210D003681A6812F0040FD6
S3150800FFD00BD01A6822F004021A60C26D08239340F7
S3150800FFE0BB60436D43F001034365E26D654B934087
S3150800FFF02B4209D02268526912F0800F04D0BB60E8
S31508010000636D43F002036365E26D5F4B93402B42D8
S3150801001009D02268126812F0020F04D0BB60636D22
S3150801002043F004036365E26D102393402B4224D009
S315080100302268126812F0080F1FD0BB6023681A687D
S3150801004012F4802F0DD01B6813F4002F04D1236CF2
S315080100509BB12046984710E0A36C73B12046984798
S315080100600BE01A6812F4807F03D11A6822F008029D
S315080100701A60236C0BB120469847E26D2023934002
S315080100802B4255D02268126812F0100F50D0BB606F
S3150801009094F83530DBB2052B0ED023681A6812F4B2
S315080100A0802F33D01B6813F4002F2AD1636C002BE1
S315080100B03ED0204698473BE02268136823F0160392
S315080100C013602268536923F080035361236CA3B13B
S315080100D02268136823F008031360E26D3F239340F7
S315080100E0BB60002384F83430012384F83530236D4E
S315080100F0002B43D02046984740E0A36C002BE7D15C
S31508010100EBE7E36BA3B12046984711E01A6812F4AE
S31508010110807F09D11A6822F010021A60002384F838
S315080101203430012384F83530E36B0BB12046984708
S31508010130636D1BB3636D13F0010F1BD0052384F8A0
S3150801014035302268136823F0010313600F4BA3FBB4
S315080101500636B60A019B01330193B34204D82368D4
S315080101601B6813F0010FF5D1002384F834300123FD
S3150801017084F83530E36C0BB12046984703B0F0BDDF
S31508010180040000200100800004008000B5814E1B98
S315080101902DE9F04F83B00025664FDFF8A4C1664EFE
S315080101A0DFF8A091DFF8A0A142E0EC0800EB840497
S315080101B0D4F820E005F007024FEA820B0F2202FA73
S315080101C00BF22EEA020E0A6902FA0BF242EA0E0253
S315080101D0226239E00022A24042EA0E029A6033689E
S315080101E06FEA08044A6812F4803F0CBF234048EAC4
S315080101F00303336073684A6812F4003F0CBF234057
S3150801020048EA03037360B2684B6813F4801F0CBF96
S31508010210224048EA0202B260F3684A6812F4001FF3
S315080102200CBF234048EA0303F3600135102D7ED045
S315080102300123AB400A6803EA02084345F5D14A6837
S3150801024022F01002022AB0D004684FEA450E0322B2
S3150801025002FA0EF2D24302EA040B4C6804F00304D4
S3150801026004FA0EF444EA0B0404604C6824F0100402
S31508010270013C012C12D8846802EA040BCC6804FA02
S315080102800EF444EA0B048460446824EA030B4C68C0
S31508010290C4F30013AB4043EA0B034360C3681A4037
S315080102A08B6803FA0EF31343C3604B6813F0805F40
S315080102B0BBD0002301937B6C43F480437B647B6C46
S315080102C003F480430193019B25F0030303F1804363
S315080102D003F59C339A6805F00304A4004FF00F0E4A
S315080102E00EFA04FE22EA0E0E60453FF473AF484546
S315080102F013D0504513D0114A904212D002F58062AC
S31508010300904210D002F5806290420ED002F58062CA
S3150801031090420CBF062207225DE701225BE7022213
S3150801032059E7032257E7042255E7052253E703B0A5
S31508010330BDE8F08F00380240003C0140000C024045
S315080103400000024000040240000802402DE9F04F77
S3150801035000234FF00108DFF818A1DFF81891DFF83C
S3150801036018B108E04FF0000C0CFA04F4744560D09B
S315080103700133102B77D008FA03F404EA0105AC42DD
S31508010380F6D106685F000322BA40D24316400660DA
S315080103904FEAD30C00EB8C0CDCF820E003F00706DF
S315080103A0B6000F2707FA06F62EEA0606CCF82060ED
S315080103B0866816408660466826EA04044460C4686E
S315080103C02240C26023F0030202F1804202F59C3208
S315080103D0966803F00304A400A74006EA070E5045F1
S315080103E0C0D0584517D0214EB04216D006F58066C2
S315080103F0B04215D006F58066B04214D006F580667F
S31508010400B04213D006F58066B0420CBF4FF0060C19
S315080104104FF0070CA8E7C446A6E74FF0020CA3E77E
S315080104204FF0030CA0E74FF0040C9DE74FF0050CC5
S315080104309AE7946824EA07079760D9F80020ED43FC
S315080104402A40C9F80020D9F804202A40C9F804200E
S31508010450D9F808202A40C9F80820D9F80C201540EF
S31508010460C9F80C5084E7BDE8F08F00BF00080240C8
S3150801047000000240003C01400004024003691942A1
S3150801048014BF01200020704712B909048161704721
S31508010490816170477047000008B5054B5B690342E7
S315080104A000D108BD024B5861FFF7F4FFF9E700BF19
S315080104B0003C014003685A6912F4806F0DD06FF44D
S315080104C080625A610423036400230363202280F8AF
S315080104D03D2080F83C3001207047002070472DE907
S315080104E0F041064690461D46C1F307478CB2012FD7
S315080104F033680CBF5B699B6934EA03030CBF0123AC
S315080105000023984512D1B5F1FF3FF0D02DB1FFF781
S31508010510ADF8069BC01AA842E9D900233363202205
S3150801052086F83D2086F83C30032000E00020BDE82F
S31508010530F0812DE9F041044617469846C1F307466E
S315080105408DB2012E23680CBF5B699B6935EA0303EB
S3150801055014BF0123002353B323685A6912F4806F29
S3150801056012D1B7F1FF3FECD02FB1FFF77FF8A0EB1F
S315080105700800B842E5D900232363202284F83D20E8
S3150801058084F83C30032013E01A6842F400721A60BA
S3150801059023686FF480625A6104232364002323636A
S315080105A0202284F83D2084F83C30012000E0002018
S315080105B0BDE8F08170B504460D46164623685B69A9
S315080105C013F0800F19D12046FFF774FFB8B9B5F1BA
S315080105D0FF3FF3D025B1FFF749F8801BA842EDD9B3
S315080105E0236C43F02003236400232363202284F829
S315080105F03D2084F83C30032000E0002070BD012036
S31508010600FCE700002DE9F04184B004460E46174682
S3150801061098460B9D0268136843F48073136000952E
S315080106200A9B00224FF00111FFF759FF002848D114
S31508010630236806F0FE061E612B460A9A25492046BE
S31508010640FFF777FF28B1236C042B0CBF0123032383
S3150801065038E00023039323685A6903929B6903933D
S31508010660039B2A460A992046FFF7A4FF034648B189
S31508010670236C042B2AD12268136843F40073136090
S3150801068001231FE0B8F1010F13D023683A0A1A6152
S315080106902A460A992046FFF78DFF034668B1236C5F
S315080106A0042B15D12268136843F4007313600123E0
S315080106B008E02268FFB2176104E02268FFB21761F9
S315080106C000E00323184604B0BDE8F0810323F9E7E7
S315080106D00323F7E7020001002DE9F04184B004463F
S315080106E00E46174698460B9D0268136843F48063C5
S315080106F013600268136843F48073136000950A9BBC
S3150801070000224FF00111FFF7EAFE002876D1F6B272
S31508010710236806F0FE021A612B460A9A3E492046CC
S31508010720FFF707FF28B1236C042B0CBF0123032312
S3150801073065E00023039323685A6903929B6903932F
S31508010740039B2A460A992046FFF734FF48B1236CD2
S31508010750042B58D12268136843F4007313600123EC
S315080107604DE0B8F1010F12D12368FFB21F612A4685
S315080107700A992046FFF71EFF00B3236C042B46D1C6
S315080107802268136843F400731360012337E0236872
S315080107903A0A1A612A460A992046FFF70BFF48B119
S315080107A0236C042B31D12268136843F40073136058
S315080107B0012324E02368FFB21F61D8E72268136882
S315080107C043F48073136000950A9B00224FF00111D0
S315080107D02046FFF784FEE0B9236846F001061E614C
S315080107E02B460A9A0C492046FFF7A3FE034630B169
S315080107F0236C042B0CBF0123032300E003231846B3
S3150801080004B0BDE8F0810323F9E70323F7E70323DF
S31508010810F5E70323F3E700BF0200010070B50446BC
S315080108200D46164623685B6913F0040F19D1204655
S31508010830FFF740FEB8B9B5F1FF3FF3D025B1FEF792
S3150801084015FF801BA842EDD9236C43F020032364CE
S3150801085000232363202284F83D2084F83C300320BA
S3150801086000E0002070BD0120FCE770B505460C4686
S3150801087016462B685A6912F0400F22D15A6912F0AE
S31508010880100F11D124B1FEF7F1FE801BA042F0D959
S315080108902B6C43F020032B64202385F83D3000237D
S315080108A085F83C30032070BD6FF010025A610023B1
S315080108B02B642B63202285F83D2085F83C300120E6
S315080108C0F1E70020EFE70000002872D010B50446D2
S315080108D090F83D30002B41D0242384F83D3022681E
S315080108E0136823F00103136000F0A4FB324BA3FB4A
S315080108F000239B0C226853606168304A914232D8C2
S3150801090001332268136263682C4A934235D85B0027
S31508010910B0FBF3F0C0F30B03032B98BF0420236845
S31508010920D8612268E369216A0B4313602268236947
S31508010930E1680B43936022686369A1690B43D3603D
S315080109402268136843F00103136000202064202302
S3150801095084F83D30206384F83E0010BD80F83C30B1
S315080109601FF058F8B8E74FF4967202FB03F3144ADE
S31508010970A2FB03239B090133C3E7A26842B903EB30
S315080109804303B0FBF3F0C0F30B036BB90120C6E7D1
S3150801099003EB830303EB8303B0FBF3F0C0F30B0311
S315080109A02BB140F44040BAE740F40040B7E70120D4
S315080109B0B5E70120704700BF83DE1B43A08601000F
S315080109C0D34D62102DE9F04782B004468846914618
S315080109D09A460A9EBDF82C50FEF748FE94F83D301B
S315080109E0DBB2202B04D00223184602B0BDE8F087FB
S315080109F0074600901923012240492046FFF76FFD5B
S31508010A00002873D194F83C30012B71D0012384F866
S31508010A103C302268136823F400631360212384F8A9
S31508010A203D30402384F83E3000232364A3F5803308
S31508010A30E36201970C9B009353464A46414620467A
S31508010A40FFF7E0FD98B9002D2ED13A460C992046BC
S31508010A50FFF7E4FE034600283AD0236C042B4BD15A
S31508010A602268136843F4007313600123BCE7236CFF
S31508010A70042B4FF0000384F83C300CBF01230323F9
S31508010A80B2E7236C042B35D12268136843F400734B
S31508010A9013600123A8E7002BD7D073781361023DB1
S31508010AA0ADB20236002DD0D03A460C992046FFF752
S31508010AB081FD0028E5D1236832781A616B1E9BB245
S31508010AC02268516911F0040FE5D101361D46E9E79F
S31508010AD021680A6842F400720A60202284F83D20DF
S31508010AE0002284F83E2084F83C207DE702237BE738
S31508010AF0022379E7032377E7032375E7020010004A
S31508010B002DE9F04786B00446884691469A460E9ED8
S31508010B10BDF83C50FEF7AAFD94F83D30DBB2202B18
S31508010B2005D04FF00208404606B0BDE8F0870746F3
S31508010B3000901923012283492046FFF7D0FC00289B
S31508010B4040F0F18094F83C30012B00F0EF8001234E
S31508010B5084F83C302268136823F400631360222367
S31508010B6084F83D30402384F83E3000232364A3F5FE
S31508010B708033E3620197109B009353464A464146E8
S31508010B802046FFF7A9FD804658B1236C042B4FF088
S31508010B90000384F83C300CBF4FF001084FF00308FE
S31508010BA0C1E765B90023029323685A6902929A69D3
S31508010BB00292029A1A6842F400721A6052E0012DF2
S31508010BC00ED0022D28D00023059323685A69059271
S31508010BD09B690593059BDFF870A14FF0000966E054
S31508010BE02268136823F48063136000230393236840
S31508010BF05A6903929A690392039A1A6842F400722F
S31508010C001A603A4610992046FFF72FFE002832D17E
S31508010C1023681B69337025E02268136823F480630F
S31508010C2013602268136843F4006313600023049376
S31508010C3023685A6904929B690493049B0097109B45
S31508010C40002241492046FFF74AFC002871D1226853
S31508010C50136843F40073136023681B6933702368B0
S31508010C601B697370202384F83D30002384F83E30D5
S31508010C7084F83C3057E7236C202B0CBF4FF0030850
S31508010C804FF001084FE73A4610992046FFF7EDFD68
S31508010C9000283AD123681B69337023685A6912F010
S31508010CA0040F3AD10136013DADB2002DDAD0032D3C
S31508010CB0E9D8012DA5D0022DC0D00097109B4A4630
S31508010CC051462046FFF70BFC002835D122681368E8
S31508010CD023F48063136023681B6933700097109BA4
S31508010CE04A4651462046FFF7FAFB40BB226813687D
S31508010CF043F40073136023681B69737023681B69C7
S31508010D00B370033DADB20336CFE7236C202B0CBF7E
S31508010D104FF003084FF0010805E71B697370023DA0
S31508010D20ADB20236C1E74FF00208FCE64FF0020801
S31508010D30F9E64FF00308F6E64FF00308F3E64FF03D
S31508010D400308F0E6020010000400010030B583B084
S31508010D5000230193234B1A6C42F080521A641B6CD0
S31508010D6003F080530193019B4FF4803393FAA3F365
S31508010D70B3FA83F303F1845303F560339B0001222D
S31508010D801A60FEF773FC0546174C636813F4803F37
S31508010D9008D1FEF76BFC401BB0F57A7FF5D9032025
S31508010DA003B030BD4FF4003393FAA3F3B3FA83F3D8
S31508010DB003F1845303F560339B0001221A60FEF7A1
S31508010DC055FC0546084C636813F4003F07D1FEF746
S31508010DD04DFC401BB0F57A7FF5D90320E0E70020EA
S31508010DE0DEE700BF003802400070004070B588B0E9
S31508010DF00E46154608B300230293204C226B42F097
S31508010E0004022263226B02F004020292029A4FF450
S31508010E100072039202220492032206920593079313
S31508010E2003A91748FFF7B4F9A26822F078423243BA
S31508010E3042EAC502A26008B070BD002301930F4CB7
S31508010E40226B42F001022263226B02F00102019237
S31508010E50019A4FF4807203920222049203220692A7
S31508010E600593079303A90748FFF792F9A26822F0A9
S31508010E70EC6232432A43A260DDE700BF0038024034
S31508010E800008024000000240634B1B6803F00F0391
S31508010E908B4209D2CBB2604A1370136803F00F0371
S31508010EA08B4201D0012070472DE9F041036813F008
S31508010EB0020F06D0594A936823F0F0038468234346
S31508010EC093600C460546036813F0010F64D0426827
S31508010ED0012A26D0931E012B2AD9504B1B6813F0E1
S31508010EE0020F00F097804D498B6823F003031343E3
S31508010EF08B60FEF7BBFB06466B68012B1FD0022BE6
S31508010F002CD0032B39D0454F41F28838BB6813F0F2
S31508010F100C0F41D0FEF7AAFB801B4045F6D90320EA
S31508010F2076E03E4B1B6813F4003FDCD101206FE0ED
S31508010F303A4B1B6813F0007FD5D1012068E0374F83
S31508010F4041F28838BB6803F00C03042B24D0FEF762
S31508010F508DFB801B4045F5D9032059E02F4F41F2FF
S31508010F608838BB6803F00C03082B15D0FEF77EFB07
S31508010F70801B4045F5D903204AE0284F41F28838BD
S31508010F80BB6803F00C030C2B06D0FEF76FFB801B26
S31508010F904045F5D903203BE01F4B1B6803F00F03BF
S31508010FA0A34209D9E2B21C4B1A701B6803F00F035E
S31508010FB0A34201D001202BE02B6813F0040F06D0C1
S31508010FC0164A936823F4E053E9680B4393602B6848
S31508010FD013F0080F07D0114A9368296923F460436F
S31508010FE043EAC103936000F02FFD0C4B9B68F02286
S31508010FF092FAA2F2B2FA82F203F0F003D340084A57
S31508011000D35CD840074B18600020FEF7F7FA00209A
S31508011010BDE8F0810120FBE7003C024000380240B0
S315080110206C41030804000020014B1868704700BF93
S3150801103004000020084B9B684FF4E05292FAA2F292
S31508011040B2FA82F203F4E053D340044AD35C044A69
S315080110501068D840704700BF003802406C41030849
S3150801106004000020084B9B684FF4604292FAA2F2F2
S31508011070B2FA82F203F46043D340044AD35C044AC9
S315080110801068D840704700BF003802406C41030819
S31508011090040000202DE9F04782B00446036813F0E6
S315080110A0010F00F0AB80964AD2F88C3023F0C0636A
S315080110B0816B0B43C2F88C30856BB5FA85F56D09E2
S315080110C0236813F0020F0CD08D4AD2F88C3023F026
S315080110D0C053E16B0B43C2F88C30E36B002B08BF9E
S315080110E00125236813F0040F00F08A80844AD2F898
S315080110F08C3023F44013216B0B43C2F88C30266BDA
S31508011100B6F5801F08BF0125B6FA86F67609236863
S3150801111013F0080F0FD07A4AD2F88C3023F4400323
S31508011120616B0B43C2F88C30636BB3F5800F69D0E2
S31508011130002B08BF0126236813F0200F64D123680A
S3150801114013F0100F03D094F858206E4B1A602368D9
S3150801115013F0800F08D06A4AD2F8943023F440037A
S31508011160E16C0B43C2F89430236813F0400F08D0A2
S31508011170634AD2F8943023F08063A16C0B43C2F81A
S315080111809430236813F4807F0DD05D4AD2F89430E9
S3150801119023F00063616D0B43C2F89430636DB3F1BC
S315080111A0006F08BF0126236813F4007F08D0544A4C
S315080111B0D2F8943023F08053616C0B43C2F8943013
S315080111C0236813F4806F0CD04D4AD2F8943023F07B
S315080111D00053216D0B43C2F89430236DB3F1005FC0
S315080111E07BD0012D79D02368B3F5006F75D0012E18
S315080111F000F0C681002002B0BDE8F08700255FE750
S31508011200002684E7012596E7002301933C4B1A6CD7
S3150801121042F080521A641B6C03F080530193019BC0
S31508011220394A136843F480731360FEF71FFA804640
S31508011230354F3B6813F4807F07D1FEF717FAA0EB09
S3150801124008000228F5D90320D5E72D4B1B6F13F4A7
S31508011250407312D0226C02F440729A420DD0284B88
S315080112601A6F22F44072294901200860002008609B
S315080112701A671B6F13F0010F12D1236C03F4407226
S31508011280B2F5407F1ED01E4A936823F4F813936083
S315080112901B4A116F236CC3F30B030B4313674EE70A
S315080112A0FEF7E4F98146164F41F288383B6F13F091
S315080112B0020FE2D1FEF7DAF9A0EB09004045F5D9AC
S315080112C0032098E70E498A6822F4F81223F070433E
S315080112D023F4407313438B60DAE70D4B00221A603F
S315080112E0FEF7C4F90746064D2B6813F0006F11D0B7
S315080112F0FEF7BCF9C01B0228F6D903207BE700BF1D
S3150801130000380240E011474200700040400E474253
S3150801131068004742236813F0010F01D0A26B2AB176
S3150801132013F0020F43D0E36B002B40D1CA49D1F821
S3150801133084304FF4403090FAA0FCBCFA8CFCD1F80A
S3150801134084504FF0706E9EFAAEF8B8FA88F847F6F0
S31508011350C07292FAA2F2B2FA82F790FAA0F0B0FA43
S3150801136080F09EFAAEFEBEFA8EFE4FF0E04999FA7B
S31508011370A9F9B9FA89F9A268BA40676907FA09F7B2
S315080113803A4367683A4305F0706525FA08F808FA9A
S315080113900EFE42EA0E0203F4403323FA0CF301333C
S315080113A023F00043013B83401343C1F8843023688B
S315080113B013F0040F03D0226BB2F5801F06D013F089
S315080113C0080F4ED0636BB3F5800F4AD1A249D1F805
S315080113D084304FF4403090FAA0FCBCFA8CFCD1F86A
S315080113E084504FF0E04E9EFAAEF8B8FA88F847F600
S315080113F0C07292FAA2F2B2FA82FA90FAA0F0B0FAA0
S3150801140080F04FF0706999FAA9F9B9FA89F99EFA43
S31508011410AEFEBEFA8EFEA26802FA0AF2276907FA3A
S3150801142009F73A4367683A4305F0E04525FA08F8AB
S3150801143008FA0EFE42EA0E0203F4403323FA0CF3CD
S31508011440013323F00043013B83401343C1F8843041
S31508011450D1F88C20A36A013B22F01F021343C1F87D
S315080114608C30236813F4806F03D0236DB3F1005FCA
S3150801147043D0236813F4006F2CD047F6C07090FA56
S31508011480A0F0B0FA80F04FF4403393FAA3F3B3FA1D
S3150801149083F54FF0706191FAA1F1B1FA81F14FF03C
S315080114A0E04292FAA2F2B2FA82F2E3685B08013BE1
S315080114B0AB40A56805FA00F0034360680343206959
S315080114C000FA01F10B43616901FA02F21343624A18
S315080114D0C2F88430614B01221A60FEF7C7F8074645
S315080114E05D4D2B6813F0006F7FF481AEFEF7BEF8F1
S315080114F0C01B0228F5D903207DE6DFF85CC1DCF8BC
S3150801150084204FF4403393FAA3FEBEFA8EFEDCF82C
S3150801151084104FF0E04090FAA0F8B8FA88F847F638
S31508011520C07999FAA9F9B9FA89F993FAA3F3B3FA39
S3150801153083F74FF0706595FAA5F5B5FA85F590FA32
S31508011540A0F0B0FA80F0E3685B08013BBB40A768EE
S3150801155007FA09F73B4367683B4301F0E04121FA83
S3150801156008F808FA00F0034302F4403222FA0EF2B0
S315080115700132520002FA05F52B43CCF8843078E79C
S31508011580374B00221A60FEF771F80646324D2B6872
S3150801159013F0005F06D0FEF769F8801B0228F6D91A
S315080115A0032028E6236813F0040F01D0226B22B129
S315080115B013F0080F36D0636BA3BB2749D1F88830DF
S315080115C04FF4403292FAA2F6B6FA86F647F6C0709A
S315080115D090FAA0F0B0FA80F092FAA2F2B2FA82F288
S315080115E04FF0706595FAA5F5B5FA85F503F440331C
S315080115F0F340013323F00043013B9340E269824003
S31508011600606AA8400243A06902431343C1F88830BF
S31508011610D1F88C30E26A013A23F4F85343EA0223FB
S31508011620C1F88C30236813F4807F03D0636DB3F15E
S31508011630006F17D00A4B01221A60FEF717F8054604
S31508011640054C236813F0005F37D1FEF70FF8401BEE
S315080116500228F6D90320CEE5003802406800474241
S31508011660700047421648D0F888204FF0706191FA09
S31508011670A1F7B7FA87F747F6C07595FAA5F5B5FA4A
S3150801168085F54FF4403393FAA3F3B3FA83F691FA47
S31508011690A1F1B1FA81F1236A5B08013BB340E6691E
S315080116A006FA05F52B43A469234302F07062FA4052
S315080116B08A401343C0F88830BCE700209BE500BF89
S315080116C000380240F0B583B00446036813F0010FF1
S315080116D034D0AE4B9B6803F00C03042B25D0AB4BDF
S315080116E09B6803F00C03082B1AD0A84B9B6803F0E0
S315080116F00C030C2B4CD02279A54B1A706368002B6E
S315080117004CD0FDF7B3FF0646A04D2B6813F4003FF6
S3150801171014D1FDF7ABFF801B6428F6D903208AE1B3
S315080117209A4B5B6813F4800FDFD0984B1B6813F450
S31508011730003F03D06368002B00F07A81236813F019
S31508011740020F5CD0914B9B6813F00C0F3AD08F4B6C
S315080117509B6803F00C03082B2FD08C4B9B6803F076
S315080117600C030C2B38D0E368002B6ED0894B012271
S315080117701A60FDF77BFF0646844D2B6813F0020FAE
S3150801178055D1FDF773FF801B0228F6D9032052E1D4
S315080117907E4B5B6813F4800FADD0C6E7FDF766FF95
S315080117A006467A4D2B6813F4003FC7D0FDF75EFF56
S315080117B0801B6428F6D903203DE1744B5B6813F45A
S315080117C0800FCAD1714B1B6813F0020F0AD0E36868
S315080117D0012B07D001202EE16C4B5B6813F4800FB7
S315080117E0C1D1EFE769480168F82393FAA3F3B3FA7D
S315080117F083F22369934021F0F802134303602368B7
S3150801180013F0080F45D063698BB3634B01221A6045
S31508011810FDF72CFF06465D4D6B6F13F0020F38D1AD
S31508011820FDF724FF801B0228F6D9032003E1574858
S315080118300168F82393FAA3F3B3FA83F22369934071
S3150801184021F0F80213430360D9E7524B00221A60CC
S31508011850FDF70CFF06464D4D2B6813F0020FCED04F
S31508011860FDF704FF801B0228F6D90320E3E04A4B63
S3150801187000221A60FDF7FAFE0646444D6B6F13F017
S31508011880020F06D0FDF7F2FE801B0228F6D90320C7
S31508011890D1E0236813F0040F1FD1A369002B00F0D0
S315080118A0C9803A4A926802F00C02082A00F0C580FB
S315080118B0022B59D0394B00221A60FDF7D7FE05468F
S315080118C0324C236813F0007F00F0B080FDF7CEFE9E
S315080118D0401B0228F5D90320ADE0002301932B4BC9
S315080118E01A6C42F080521A641B6C03F08053019300
S315080118F0019B2B4A136843F480731360FDF7B6FE08
S315080119000646274D2B6813F4807F06D1FDF7AEFEF8
S31508011910801B0228F6D903208DE0227A214B1A7002
S31508011920A36883B1FDF7A2FE0746184D41F2883632
S315080119302B6F13F0020FB0D1FDF798FEC01BB04212
S31508011940F6D9032077E0FDF791FE07460F4D41F2E0
S3150801195088362B6F13F0020F9FD0FDF787FEC01B49
S31508011960B042F6D9032066E00C4B00221A60FDF757
S315080119707DFE0646054D2B6813F0007F14D0FDF752
S3150801198075FE801B0228F6D9032054E00038024070
S315080119900238024000004742800E47426000474233
S315080119A0007000407038024047F6C07696FAA6F6EF
S315080119B0B6FA86F64FF4403292FAA2F2B2FA82F5F4
S315080119C04FF0706090FAA0F0B0FA80F04FF0E04165
S315080119D091FAA1F1B1FA81F1E369226A1343626AC4
S315080119E002FA06F63343A26A5208013AAA40134399
S315080119F0E26A02FA00F00343226B02FA01F10B4391
S31508011A000F4A53600F4B01221A60FDF72FFE054658
S31508011A100B4C236813F0007F06D1FDF727FE401B08
S31508011A200228F6D9032006E0002004E0002002E09F
S31508011A30012000E0002003B0F0BD0120FBE700BF54
S31508011A400038024060004742274B9B6803F00C03AD
S31508011A50082B03D00C2B25D024487047224B5A68F3
S31508011A6002F03F025B68204B5B6847F6C07191FA4A
S31508011A70A1F0B0FA80F00B40C3401C48B0FBF2F06D
S31508011A8000FB03F0184B5B684FF4403292FAA2F25E
S31508011A90B2FA82F203F44033D34001335B00B0FB60
S31508011AA0F3F07047104B5A6802F03F025B680E4B21
S31508011AB05B6847F6C07191FAA1F0B0FA80F00B4065
S31508011AC0C3400A48B0FBF2F000FB03F0064B5B6823
S31508011AD04FF0E04292FAA2F2B2FA82F203F0E04340
S31508011AE0D340B0FBF3F07047003802400024F400FD
S31508011AF00268536B13F0450FFBD0536B13F0040FB9
S31508011B0008D1536B13F0010F08D140F2FF539363C9
S31508011B1000207047042393630320704701209063D4
S31508011B207047000038B50268536B13F0450FFBD0B8
S31508011B30536B13F0040F06D1536B13F0010F06D044
S31508011B400120906338BD042393630320FAE70D4609
S31508011B500446104602F03DFAA84201D01020F1E7EA
S31508011B60236840F2FF529A63002002F035FA324B9D
S31508011B700340DBB300283BDB10F0804F3AD110F06D
S31508011B80005F39D110F0805F38D110F0006F37D17E
S31508011B9010F0806F36D110F0807F35D110F4000F28
S31508011BA034D110F4800F33D110F4001F32D110F460
S31508011BB0801F31D110F4002F30D110F4802F2FD18E
S31508011BC010F4003F2ED110F4803F2DD110F4004FB0
S31508011BD02CD110F4804F2BD110F4005F2AD100F0DC
S31508011BE00800002814BF1A200020ABE70020A9E747
S31508011BF01C20A7E70920A5E70A20A3E70B20A1E7F0
S31508011C000C209FE70D209DE70E209BE70F2099E703
S31508011C10102097E7112095E7122093E7132091E703
S31508011C2014208FE715208DE716208BE7172089E703
S31508011C30182087E7192085E708E0FFFD30B587B04A
S31508011C4004460D4600220092436A1B0401930D23A4
S31508011C5002934023039304924FF48063059301A9E9
S31508011C60006802F0A1F92068436B13F0450FFBD019
S31508011C70436B13F0040F08D1436B13F0010F08D01F
S31508011C8001238363184607B030BD04238363032009
S31508011C90F9E702F09EF90D2801D01020F3E7236831
S31508011CA040F2FF529A63002002F096F90090009BD9
S31508011CB0C3F343232B70009A3C4B1340002B4ED0A1
S31508011CC0009B002B4DDB009B13F0804F4BD1009BF3
S31508011CD013F0005F49D1009B13F0805F47D1009B49
S31508011CE013F0006F45D1009B13F0806F43D1009B21
S31508011CF013F0807F41D1009B13F4000F3FD1009B65
S31508011D0013F4800F3DD1009B13F4001F3BD1009BB8
S31508011D1013F4801F39D1009B13F4002F37D1009B90
S31508011D2013F4802F35D1009B13F4003F33D1009B68
S31508011D3013F4803F31D1009B13F4004F2FD1009B40
S31508011D4013F4804F2DD1009B13F4005F2BD1009B18
S31508011D5003F00803002B14BF1A20002093E7002084
S31508011D6091E71C208FE709208DE70A208BE70B20D6
S31508011D7089E70C2087E70D2085E70E2083E70F20EA
S31508011D8081E710207FE711207DE712207BE71320EA
S31508011D9079E7142077E7152075E7162073E71720EA
S31508011DA071E718206FE719206DE700BF08E0FFFD0E
S31508011DB02DE9F0418EB004460E46002301930293A5
S31508011DC00822099210250A9540220B920C934FF48A
S31508011DD080630D9309A9006802F0E6F829462046B2
S31508011DE0FFF7A0FE054618B128460EB0BDE8F081FA
S31508011DF0636A1B04099337250A9509A9206802F025
S31508011E00D3F829462046FFF78DFE05460028EBD173
S31508011E104FF0FF33039308230493302305930223DA
S31508011E200693002507950123089303A9206802F064
S31508011E30DFF8099533250A9509A9206802F0B4F84F
S31508011E4029462046FFF76EFE05460028CCD10DF13E
S31508011E50040840F22A472068436B3B4208D1436B8A
S31508011E6013F4001FF8D002F08FF848F8040BF2E7D4
S31508011E70436B13F0080F25D1436B13F0020F25D1DD
S31508011E80436B13F0200F24D140F2FF538363019B68
S31508011E901A0E42EA0362190201F47F010A431B0A78
S31508011EA003F47F4313437360029B1A0E42EA0362EB
S31508011EB0190201F47F010A431B0A03F47F43134302
S31508011EC0336091E70823836304258DE7022585633B
S31508011ED08AE720238363062586E77047704770479C
S31508011EE010B5044603685A6B12F4807F16D15A6BF3
S31508011EF012F0020F23D15A6B12F0080F25D15A6B33
S31508011F0012F0200F28D15A6B12F0100F0FD01022A1
S31508011F109A630523C364FFF7E2FF08E04FF4807272
S31508011F209A63012383640023C364FFF7D7FF2268FA
S31508011F30D36B23F4414323F03A03D36310BD022242
S31508011F409A63C264FFF7CBFFF1E708229A63042379
S31508011F50C364FFF7C4FFEAE720229A630623C36432
S31508011F60FFF7BDFFE3E72DE970030346026A81F82F
S31508011F705620426AA1F85420826A900F0870C2F36B
S31508011F8083604870C2F301628A7093F82A20CA7086
S31508011F9093F829200A7193F828204A7193F82F207B
S31508011FA01201CA80DA6ACC88C2F303502043C8807A
S31508011FB0C2F303420A7293F82D20D0094872C2F37C
S31508011FC080108872C2F34010C872C2F300100873F9
S31508011FD000204873186A012840F2D080022840F090
S31508011FE00B81DA6A120402F47C120A610A6993F80F
S31508011FF0330042EA00220A61086993F83220024353
S315080120000A6193F831200C69002514F1010845F19C
S3150801201000094FEAC94040EA58304FEAC8448C647F
S31508012020C8644FF4007008650020C2F380144C762A
S31508012030520002F07E028A761A6B8C7EC2F3C015B4
S315080120402C438C7602F07F02CA765A6BD40F0C7732
S31508012050C2F341744C77C2F382648C77920D02F015
S315080120600C02CA775A6BCC7FC2F381552C43CC77C5
S31508012070C2F3405481F82040002481F82140C2F37C
S31508012080004281F822205A6BC2F3C03481F82340FA
S31508012090C2F3803481F82440C2F3403481F82540E4
S315080120A0C2F3003481F82640C2F3812481F827401F
S315080120B0C2F3012281F828205A6BC2F3460281F83D
S315080120C02920012481F82A4093F83B2081F82C2005
S315080120D093F83A201202CA85CD8D93F839202A43FE
S315080120E0CA859A6B12060A630A6B93F83F5042EA4D
S315080120F005420A630D6BDA8F120292B22A430A630A
S315080121000D6B93F83D202A430A6393F83C2081F826
S31508012110342093F8432081F83520B3F8422012067B
S315080121208A638D6B1A6C120202F47F022A438A6350
S315080121308D6B1A6C120292B22A438A638D6B93F8DD
S3150801214047202A438A635A6C91F83C50C2F30356D6
S31508012150354381F83C50120A02F47062CA87CD8F62
S3150801216093F845202A43CA875B6CC3F3460381F873
S31508012170403081F84140BDE870037047920202F48D
S3150801218040620A610869DA6A920002F47F720243C0
S315080121900A611A6B086940EA92700861C2F3C26063
S315080121A00875C2F302624A751A6BC2F34250887502
S315080121B0C2F38240C875D20B02F006020A76186B82
S315080121C0C0F307220C7EC0F3C030204308760C69A1
S315080121D00D7E087AC0B2012606FA00F008650235B6
S315080121E0AE400134A4FB0045A6FB048906FB05990C
S315080121F0C1E91289002018E7292016E72DE9F043DD
S3150801220093B00446894600258DF847500577FFF7B0
S3150801221064FE0B950C950D950E950F9576231093E7
S315080122200EAB93E807008DE807000BAB0ECB2068D1
S3150801223001F08EFE8DF81750AA4F3D60206801F017
S31508012240ABFE0120FDF718FA01233B6006950795B9
S31508012250089509954FF480630A9306A9206801F049
S31508012260A3FE21684B6B13F0800F40F099814B6BED
S31508012270C3F3C0134FF6FF72002B40F091814B6BED
S31508012280C3F3C013013AF7D103238DE14FF4D57394
S315080122900693082307934023089306A9206801F0AB
S315080122A083FE21684B6B13F0450F40F094814FF480
S315080122B080334A6B013B12F0450F0FD1002BF8D141
S315080122C04B6B04238B6303238DF817309DF8173066
S315080122D0A3B9012323624FF0804610E04A6B002B15
S315080122E0EFD002F00402002AEBD14B6B13F0400F3A
S315080122F01DBF40238B6300232923E5E7002600231E
S3150801230006933725079506A9206801F04DFE29464B
S315080123102046FFF707FC8DF817009DF81730002BAC
S315080123205ED14FF00008454646F0004646F4801651
S3150801233017E09DF81730DBB240E1042393630323CA
S315080123408DF817309DF81730002B3CD1284601F03F
S3150801235043FE08F10108002839DB4FF6FF7398455B
S3150801236042D00695372707974023089309954FF4D6
S3150801237080630A9306A9206801F016FE39462046AD
S31508012380FFF7D0FB8DF817009DF81730002BD0D139
S315080123900696292307934023089309954FF48063EA
S315080123A00A9306A9206801F0FFFD2268536B13F012
S315080123B0450FFBD0536B13F0040FBED140F2FF5308
S315080123C093632B46BCE79DF81730DBB2F6E04FF670
S315080123D0FE73984508D810F0804F1CBF022323626C
S315080123E09DF81730DBB2E9E01B238DF817309DF80D
S315080123F01730DBB2E2E0206801F0D2FD002800F0D8
S315080124009B80236A042B0BD100258DF847509DF834
S315080124104730002B00F092809DF84700C0B2D7E004
S315080124200023069302220792C022089209934FF4C9
S3150801243080630A9306A9206801F0B6FD2046FFF7D6
S3150801244057FB05460028E0D101F0C6FDA06304202C
S3150801245001F0C2FDE063082001F0BEFD20640C20F6
S3150801246001F0BAFD6064236A022B01D9062B61D1FA
S31508012470032307934023089306A9206801F094FDD6
S315080124802068436B13F0450FFBD0436B13F0040F21
S3150801249006D1436B13F0010F06D001258563B4E716
S315080124A0042383630325B0E701F093FD032801D0D4
S315080124B01025AAE7236840F2FF529A63002001F02B
S315080124C08BFD10F4604F0FD010F4005F40F0878049
S315080124D010F4804F40F0858010F4004F40F083805F
S315080124E0012302E0A0802542030C226A042A8CD02B
S315080124F063621B04069309230793C023089306A95D
S31508012500206801F051FD2046FFF7F2FA054600283A
S315080125107FF47BAF01F060FDA062042001F05CFD51
S31508012520E062082001F058FD20630C2001F054FDFB
S3150801253060636AE70123D8E7252566E74946204609
S31508012540FFF711FD8DF847009DF8473083B1234603
S3150801255053F8105B93E807008DE80700043494E804
S315080125600E00284601F0F4FC9DF84700C0B22FE0A2
S31508012570B9F854301B040693072507954023089399
S31508012580002309934FF480630A9306A9206801F092
S315080125900BFD29462046FFF7C5FA8DF84700D6E711
S315080125A040F2FF538B6300238DF817309DF81730DF
S315080125B0002B3FF46BAE9DF81730DBB28DF8473030
S315080125C09DF84730002B3FF416AF9DF84700C0B27F
S315080125D013B0BDE8F0834A6B02F0040283E61325C3
S315080125E013E7102511E70F250FE700BF70B592B065
S315080125F0036A032B00F09C80022B00F29B80B1F545
S31508012600805F00F09B800D460446B1F5006F3AD015
S31508012610002940F0958000200590069001F0DCFC29
S3150801262010F0007F69D105A92046FFF7C1FB0646D0
S31508012630002863D1069B13F4803F77D0636A1B0495
S315080126400793372608964023099300230A934FF4E4
S3150801265080630B9307A9206801F0A6FC3146204642
S31508012660FFF760FA0646002848D100230793062695
S31508012670089607A9206801F097FC31462046FFF71E
S3150801268051FA06463AE000200590069001F0A4FCAE
S3150801269010F0007F2DD105A92046FFF789FB0646D4
S315080126A060BB069B13F4802F25D0636A1B0407932E
S315080126B0372608964023099300230A934FF480632B
S315080126C00B9307A9206801F06FFC31462046FFF7F6
S315080126D029FA064690B9022307930626089607A9FA
S315080126E0206801F061FC31462046FFF71BFA0646D1
S315080126F004E00E2602E0252600E00E26DEB9636810
S315080127000C93A3680D93E3680E930F956369109371
S31508012710A3691193246812AB13E907008DE8070032
S315080127200CAB0ECB204601F013FC04E02526E5E7A9
S31508012730272600E00026304612B070BD2726FAE7A4
S315080127402626F8E730B587B00446002301930C2501
S3150801275002954022039204934FF48063059301A9DD
S31508012760006801F021FC29462046FFF7DBF907B08E
S3150801277030BD2DE9F0438DB004460E469046149DB2
S3150801278002680021D162026A022A17D0079510272A
S3150801279008974023099300230A934FF480630B9308
S315080127A007A9206801F000FC39462046FFF7BAF967
S315080127B0074650B138460DB0BDE8F0834FEA5828B0
S315080127C048EAC3584FF40075E0E74FF0FF33019329
S315080127D0159B03FB05F502959023039302230493A6
S315080127E0002305930123069301A9206801F000FC43
S315080127F0159B012B23D9122508950CA941F8148D8F
S31508012800206801F0D1FB29462046FFF78BF90746D8
S315080128100028CFD123685A6B12F4957F40D15A6BA1
S3150801282012F4004FF7D0351F06F11C08206801F095
S31508012830ABFB45F8040FA845F8D12036EAE7112580
S3150801284008950CA941F8148D206801F0ADFB2946BD
S315080128502046FFF767F907460028ABD140F22A4818
S3150801286023685A6B12EA080F26D15A6B12F4004FE5
S31508012870F7D0351F06F11C09206801F085FB45F8DC
S31508012880040FA945F8D12036EAE70823836304270C
S3150801289090E7022787638DE720238363062789E765
S315080128A05B6B13F4807F08D0236A022B05D8204678
S315080128B0FFF748FF074600E05B6B2068436B13F0A0
S315080128C0080FE2D1436B13F0020FE2D1436B13F009
S315080128D0200FE1D1436B13F4001F18BF4FF0FF35EA
S315080128E00AD001F051FB46F8040B2068436B13F438
S315080128F0001F01D0013DF4D140F2FF53836359E72C
S315080129002DE9F04F8DB004460F469046169D0022DC
S315080129108DF803200168CA62026A022A29D007953E
S31508012920102608964023099300230A934FF48063DF
S315080129300B9307A9206801F037FB31462046FFF7BC
S31508012940F1F8034688B9179B012B8CBF192618265F
S3150801295008960CA941F8148D206801F025FB31462B
S315080129602046FFF7DFF8034650B118460DB0BDE81B
S31508012970F08F4FEA582848EAC3584FF40075CEE756
S31508012980179B03FB05F54FF0FF330193029590233F
S3150801299003930023049305930123069301A9206851
S315080129A001F026FB179B012B29D94FF00008236854
S315080129B05A6B12F48D7F40F0A8805A6B12F4804F3F
S315080129C0F6D0A5EB080ABAF11F0F45D81AF0030F7E
S315080129D04FEA9A0A18BF0AF1010ABAF1000FE6D0BE
S315080129E0B94600264946206801F0D1FA09F10409D9
S315080129F00136B245F6D1B6003744B044D7E74FF0B1
S31508012A00000840F21A4623685A6B32424CD15A6B77
S31508012A1012F4804FF8D0A5EB080BBBF11F0F29D88C
S31508012A201BF0030F4FEA9B0B18BF0BF1010BBBF110
S31508012A30000FE8D0BA464FF000095146206801F068
S31508012A40A6FA0AF1040A09F10109CB45F5D14FEABB
S31508012A5089094F44C844D6E73E4607F1200931465D
S31508012A60206801F094FA04364E45F8D1203708F16A
S31508012A7020089CE7B94607F1200A4946206801F073
S31508012A8086FA09F10409CA45F7D1203708F1200861
S31508012A90B9E708239363042367E70223936364E78B
S31508012AA010239363052360E75B6B2268536B13F06E
S31508012AB0080FEED1536B13F0020FEED1536B13F0DF
S31508012AC0100FEDD140F2FF5393630DF10301204638
S31508012AD0FFF7B4F8034600287FF447AF9DF80320B3
S31508012AE0063AD2B2012A3FF640AF0DF1030120465C
S31508012AF0FFF7A4F8034600287FF437AF9DF80320B3
S31508012B00063AD2B2012AF0D92FE75B6B13F4807F1C
S31508012B10CBD0236A022BC8D82046FFF713FEC4E799
S31508012B2030B587B00446436A1B0401930D25029507
S31508012B3040230393002304934FF48063059301A96B
S31508012B40006801F031FA29462046FEF7EBFF08B185
S31508012B50022006E001F040FAC0F34320043818BF0A
S31508012B60012007B030BDF8B507460E4615461C4686
S31508012B703A68936836EA03030CBF012300239D4292
S31508012B8038D0B4F1FF3FF4D02CB1FCF76FFD069BAA
S31508012B90C01AA042ECD33A68536823F0E0035360A5
S31508012BA07B68B3F5827F0BD0BB6AB3F5005F14D09F
S31508012BB0012387F85130002387F8503003201AE0A3
S31508012BC0BB68B3F5004F02D0B3F5806FECD13A6814
S31508012BD0136823F040031360E6E73A68136823F4A1
S31508012BE000531B041B0C13603A68136843F4005323
S31508012BF01360DDE70020F8BD10B582B004460092E7
S31508012C000B4600228021FFF7AEFF034610B918468E
S31508012C1002B010BD636D43F0200363650323F6E735
S31508012C2000283BD010B504460023836290F8513042
S31508012C30002B2ED0022384F851302268136823F022
S31508012C404003136022686368A1680B43E1680B437C
S31508012C5021690B4361690B43E1690B43216A0B4304
S31508012C60A16A0B43A16901F400710B431360226841
S31508012C70638B03F00403616A0B4353602268D369CB
S31508012C8023F40063D36100206065012384F8513081
S31508012C9010BD80F850301CF0E9FECBE701207047E3
S31508012CA02DE9F04184B01E4690F85030012B00F012
S31508012CB0C58004460D469046012380F85030FCF73E
S31508012CC0D5FC074694F85130DBB2012B09D0022016
S31508012CD0012384F85130002384F8503004B0BDE84C
S31508012CE0F081002D00F0A280B8F1000F00F0A0805D
S31508012CF0032384F85130002363652563A4F83480DF
S31508012D00A4F83680A363A387E38763642364A3686F
S31508012D10B3F5004F1BD023681A6812F0400F03D190
S31508012D201A6842F040021A60E368B3F5006F14D0DE
S31508012D3063681BB1E38E9BB2012B3ED1236815F85C
S31508012D40012B1A73E38E013B9BB2E38635E02268B9
S31508012D50136843F480431360DDE763681BB1E38EB0
S31508012D609BB2012B0DD1236835F8022BDA60E38E6D
S31508012D70013B9BB2E38604E0002E5BD0B6F1FF3F30
S31508012D800FD1E38E9BB27BB323689A6812F0020FC8
S31508012D90F2D035F8022BDA60E38E013B9BB2E3866B
S31508012DA0EFE7FCF763FCC01BB042EAD303208FE7C9
S31508012DB0002E41D0B6F1FF3F0FD1E38E9BB29BB1F6
S31508012DC023689A6812F0020FF2D015F8012B1A73CC
S31508012DD0E38E013B9BB2E386EFE7FCF747FCC01B9A
S31508012DE0B042EAD3032073E7009733460122022152
S31508012DF02046FFF7B8FE08B1032069E73A4631468F
S31508012E002046FFF7F9FE18B12023636501205FE725
S31508012E10A36833B903932368DA6803929B6803931B
S31508012E20039B606D003018BF012051E701204FE771
S31508012E3001204DE703204BE7032049E702204DE730
S31508012E402DE9F04F85B099460E9D90F85030012B2B
S31508012E5000F0118104460F461646012380F85030CA
S31508012E60FCF704FC804694F85130DBB2012B16D0EE
S31508012E706268B2F5827F0AD00223012284F85120C2
S31508012E80002284F85020184605B0BDE8F08FA268E4
S31508012E90002A40F0E880042B01D00223EDE7002F39
S31508012EA000F0E380002E00F0E280B9F1000F00F097
S31508012EB0E08094F85130DBB2012B04BF052384F876
S31508012EC0513000236365A663A4F83E90A4F83C90AC
S31508012ED02763A4F83690A4F83490236463642368BE
S31508012EE01A6812F0400F03D11A6842F040021A60BC
S31508012EF0E368B3F5006F13D063681BB1E38E9BB229
S31508012F00012B07D1236817F8012B1A73E38E013BAE
S31508012F109BB2E3864FF001094FF0000BCA465DE00C
S31508012F2063681BB1E38E9BB2012B07D1236837F87F
S31508012F30022BDA60E38E013B9BB2E3864FF001096F
S31508012F404FF0000BCA4612E0E38F9BB263B12368C8
S31508012F509A6812F0010F07D0DB6826F8023BE38F67
S31508012F60013B9BB2E387D146B5F1FF3F1BD1E38E07
S31508012F709BB21BB9E38F9BB2002B52D0B9F1000F5C
S31508012F80E2D0E38E9BB2002BDED023689A6812F05A
S31508012F90020FD9D037F8022BDA60E38E013B9BB2D8
S31508012FA0E386D946D0E7FCF761FBA0EB0800A84207
S31508012FB0DDD3032361E7E38F9BB263B123689A6884
S31508012FC012F0010F07D0DB683370E38F013B9BB228
S31508012FD0E3870136D146B5F1FF3F1AD1E38E9BB29D
S31508012FE013B9E38F9BB2E3B1B9F1000FE3D0E38ED6
S31508012FF09BB2002BDFD023689A6812F0020FDAD051
S315080130003A781A73E38E013B9BB2E3860137D946B8
S31508013010D1E7FCF72BFBA0EB0800A842DED303237C
S315080130202BE7CDF800802B46012202212046FFF727
S315080130309AFD08B1032320E7424629462046FFF7B1
S31508013040DBFD034618B120236365012315E7A26852
S31508013050002A7FF412AF03922268D168039192681D
S315080130600392039A09E7022307E7012305E70123E8
S3150801307003E7012301E7022305E72DE9F04182B0C1
S3150801308004460D4617461E464368B3F5827F19D096
S3150801309094F85030012B00F0A180012384F85030B8
S315080130A0FCF7E4FA804694F85130DBB2012B15D0CF
S315080130B00220012384F85130002384F8503002B0ED
S315080130C0BDE8F0818368002BE2D1042380F85130F2
S315080130D0009613460A46FFF7B3FEF0E7002D75D0B2
S315080130E0002F75D0042384F8513000236365A56346
S315080130F0A787E7872363A386E38623646364A368B4
S31508013100B3F5004F0BD023681A6812F0400F03D1AC
S315080131101A6842F040021A60E3685BB128E0226847
S31508013120136823F480431360EDE7002E52D0B6F1FD
S31508013130FF3F10D1E38F9BB2002B31D023689A68E9
S3150801314012F0010FF1D01B7B05F8013BE38F013B20
S315080131509BB2E387EEE7FCF789FAA0EB0800B042D9
S31508013160E8D30320A5E7002E36D0B6F1FF3F0FD1ED
S31508013170E38F9BB2A3B123689A6812F0010FF2D0CC
S31508013180DB6825F8023BE38F013B9BB2E387EFE758
S31508013190FCF76CFAA0EB0800B042E9D3032088E7F4
S315080131A06368B3F5827F04D0606D003018BF0120D3
S315080131B07FE7A368B3F5004F02D0B3F5806FF3D16B
S315080131C02268136823F040031360EDE7012070E7D6
S315080131D001206EE703206CE703206AE702206EE709
S315080131E07047022380F839300268136843F00103F7
S315080131F01360012380F83930002070477047704703
S3150801320070477047704710B5044603681A6912F08B
S31508013210020F11D0DA6812F0020F0DD06FF0020218
S315080132201A610123037603689B6913F0030F70D0B3
S31508013230FFF7E6FF0023237623681A6912F0040FC5
S3150801324012D0DA6812F0040F0ED06FF004021A6178
S315080132500223237623689B6913F4407F5FD02046B7
S31508013260FFF7CEFF0023237623681A6912F0080FA9
S3150801327012D0DA6812F0080F0ED06FF008021A6140
S31508013280042323762368DB6913F0030F4ED0204607
S31508013290FFF7B6FF0023237623681A6912F0100F89
S315080132A012D0DA6812F0100F0ED06FF010021A6100
S315080132B0082323762368DB6913F4407F3DD0204633
S315080132C0FFF79EFF0023237623681A6912F0010F80
S315080132D003D0DA6812F0010F36D123681A6912F0A1
S315080132E0800F03D0DA6812F0800F34D123681A6987
S315080132F012F0400F03D0DA6812F0400F32D123687A
S315080133001A6912F0200F03D0DA6812F0200F30D1B3
S3150801331010BDFFF774FF2046FFF773FF8AE72046C3
S31508013320FFF76DFF2046FFF76CFF9BE72046FFF787
S3150801333066FF2046FFF765FFACE72046FFF75FFF0C
S315080133402046FFF75EFFBDE76FF001021A612046CE
S31508013350FFF754FFC1E76FF080021A61204600F0BB
S315080133609DF8C3E76FF040021A612046FFF74AFF4E
S31508013370C5E76FF020021A61204600F08EF8C7E70C
S315080133800368384A904249D0B0F1804F2DD0A2F552
S315080133907C4290422ED002F5806290422FD002F5EF
S315080133A08062904230D002F57842904231D002F5DF
S315080133B0705290424BD002F58062904247D002F596
S315080133C08062904243D0A2F5983290423FD002F5EE
S315080133D0806290423BD002F58062904237D003600A
S315080133E08B68C3620B6883622EE023F070034A6818
S315080133F0134317E023F070034A68134312E023F0DE
S3150801340070034A6813430DE023F070034A681343B7
S3150801341008E023F070034A68134303E023F07003BE
S315080134204A68134323F44073CA68134303608B68DD
S31508013430C3620B6883620B4B984203D003F5806322
S31508013440984201D10B69036301234361704723F451
S315080134504073CA68134303608B68C3620B6883624F
S31508013460F2E700BF00000140A8B110B5044690F884
S3150801347039305BB1022384F83930211D2068FFF702
S315080134807FFF012384F83930002010BD80F83830D9
S31508013490FFF7A6FEEEE701207047704770470268FE
S315080134A0D36823F49073D3600268536923F0010348
S315080134B05361202380F83A30704700002DE9F8431C
S315080134C004460268136923F44053C1680B43136128
S315080134D00168CA6822F4164222F00C028368006960
S315080134E0034360690343E06903431343CB602268DE
S315080134F0536923F44073A1690B435361E369B3F537
S31508013500004F5ED02368B34A934200F00C8102F55E
S315080135108062934200F00781FDF78CFD00EB800085
S3150801352000EB800063689B00B0FBF3F3AA4FA7FB8F
S3150801353003235B091D01FDF77DFD00EB800000EB10
S31508013540800063689B00B0FBF3F6FDF773FD00EBA3
S31508013550800000EB800063689B00B0FBF3F3A7FBD8
S3150801356003235B094FF0640909FB13631B0132331B
S31508013570A7FB03235B0903F0F006FDF75BFD00EBF0
S31508013580800000EB800063689B00B0FBF3F8FDF751
S3150801359051FD226800EB800000EB800063689B0008
S315080135A0B0FBF3F3A7FB03135B0909FB13831B01A9
S315080135B03233A7FB0313C3F3431333432B449360FB
S315080135C005E12368834A934258D002F58062934203
S315080135D054D0FDF72FFD00EB800000EB80006368F7
S315080135E05B00B0FBF3F37C4FA7FB03235B091E01CA
S315080135F0FDF720FD00EB800000EB800063685B00AF
S31508013600B0FBF3F5FDF716FD00EB800000EB80003B
S3150801361063685B00B0FBF3F3A7FB03235B094FF079
S31508013620640909FB1353DB003233A7FB03231B0988
S3150801363003F4F875FDF7FEFC00EB800000EB800053
S3150801364063685B00B0FBF3F8FDF7F4FC226800EB56
S31508013650800000EB800063685B00B0FBF3F3A7FB17
S3150801366003135B0909FB1383DB003233A7FB03133F
S31508013670C3F3421333442B449360A8E0FDF7F2FCED
S3150801368000EB800000EB800063685B00B0FBF3F39E
S31508013690514FA7FB03235B091E01FDF7E3FC00EB72
S315080136A0800000EB800063685B00B0FBF3F5FDF773
S315080136B0D9FC00EB800000EB800063685B00B0FB7F
S315080136C0F3F3A7FB03235B094FF0640909FB1353C3
S315080136D0DB003233A7FB03231B0903F4F875FDF757
S315080136E0C1FC00EB800000EB800063685B00B0FB67
S315080136F0F3F8FDF7B7FC226800EB800000EB8000C9
S3150801370063685B00B0FBF3F3A7FB03135B0909FBD3
S315080137101383DB003233A7FB0313C3F3421333448A
S315080137202B44936053E0FDF79DFC00EB800000EB12
S31508013730800063689B00B0FBF3F3274FA7FB0323C5
S315080137405B091D01FDF78EFC00EB800000EB800094
S3150801375063689B00B0FBF3F6FDF784FC00EB800081
S3150801376000EB800063689B00B0FBF3F3A7FB032320
S315080137705B094FF0640909FB13631B013233A7FB8D
S3150801378003235B0903F0F006FDF76CFC00EB8000F0
S3150801379000EB800063689B00B0FBF3F8FDF762FC61
S315080137A0226800EB800000EB800063689B00B0FB99
S315080137B0F3F3A7FB03135B0909FB13831B013233DD
S315080137C0A7FB0313C3F3431333432B449360BDE8A9
S315080137D0F88300BF001001401F85EB512DE9F04128
S315080137E007460E4615469846069C3A68136836EA11
S315080137F003030CBF01230023AB421DD1B4F1FF3FE4
S31508013800F4D02CB1FBF732FFA0EB0800A042ECD9AB
S315080138103A68D36823F4D073D3603A68536923F0BE
S3150801382001035361202387F8393087F83A3000239A
S3150801383087F83830032000E00020BDE8F08158B34E
S3150801384010B5044690F839300BB3242384F839307F
S315080138502268D36823F40053D3602046FFF72EFE6F
S315080138602268136923F4904313612268536923F08C
S315080138702A0353612268D36843F40053D3600020B6
S31508013880E063202384F8393084F83A3010BD80F893
S3150801389038301CF06FF9D8E70120704778B110B5B8
S315080138A00446242380F839301CF064FA0020E063CA
S315080138B084F8390084F83A0084F8380010BD0120EC
S315080138C070472DE9F04782B01F4690F83930DBB2D0
S315080138D0202B53D104460E461546002953D0002AFB
S315080138E053D090F83830012B51D0012380F8383065
S315080138F00023C363212380F83930FBF7B7FE8046DE
S31508013900A5844FF0000A4FF0800912E0009743465C
S31508013910524649462046FFF761FF002839D12268F9
S315080139203388C3F3080353602369ABB90236E58CC0
S31508013930A5B1013DE584A368B3F5805FE6D000979C
S315080139404346524649462046FFF748FF18BB2368B7
S3150801395032785A600136EAE70136E8E700974346C6
S31508013960002240212046FFF739FF0346A8B9202245
S3150801397084F83920002284F8382000E0022318460A
S3150801398002B0BDE8F0870123F9E70123F7E702232F
S31508013990F5E70323F3E70323F1E70323EFE72DE92C
S315080139A0F04782B01F4690F83A30DBB2202B58D147
S315080139B004460E461546002957D0002A57D090F8D6
S315080139C03830012B55D0012380F838300023C363E2
S315080139D0222380F83A30FBF749FE8246A5854FF047
S315080139E000094FF020081FE0009753464A46414612
S315080139F02046FFF7F3FE00283DD1236933B9236832
S31508013A005B68C3F3080326F8023B0BE023685B688F
S31508013A10DBB226F8013B05E023685B6803F07F0308
S31508013A2033700136E58DADB1013DE585A368B3F582
S31508013A30805FD9D0009753464A4641462046FFF74C
S31508013A40CDFED0B92369002BE6D123685B683370B4
S31508013A500136E7E7202384F83A30002084F8380055
S31508013A6000E0022002B0BDE8F0870120FAE7012054
S31508013A70F8E70220F6E70320F4E70320F2E700005F
S31508013A8038B590F83940E4B2202C31D1002931D02B
S31508013A90002A31D090F83830012B2FD0134604462E
S31508013AA0012280F8382001628384C3840025C56316
S31508013AB0212280F83920026B1148D063226B114804
S31508013AC01064226B1048D064226B15652268043293
S31508013AD0206BFCF7C3F923686FF040021A6084F87B
S31508013AE038502268536943F080035361284600E041
S31508013AF0022038BD0120FCE70120FAE70220F8E799
S31508013B000F3C0108473C01082F3D010838B590F8DC
S31508013B103A40E4B2202C37D1002937D0002A37D0D1
S31508013B2090F83830012B35D013460A46054601214F
S31508013B3080F83810826283850024C463222180F8C4
S31508013B403A10416B1448C863696B14480864696B79
S31508013B501348C864696B0C6529680431686BFCF7FE
S31508013B607DF92A68D36843F48073D3602A68536958
S31508013B7043F0010353612A68536943F040035361D3
S31508013B8085F83840204600E0022038BD0120FCE7D0
S31508013B900120FAE70220F8E7513C0108233D010814
S31508013BA02F3D010810B504460268516990F839306D
S31508013BB0DBB2212B08D02268516994F83A30DBB27E
S31508013BC0222B15D0002010BD11F0800FF3D05369B8
S31508013BD023F080035361006B08B1FCF789F9226869
S31508013BE0D36823F0C003D360202384F83930E2E791
S31508013BF011F0400FE6D0536923F040035361606B1F
S31508013C0008B1FCF775F92046FFF749FCDAE708B56C
S31508013C10836B0268126812F4807F0FD10022DA845E
S31508013C2019684A6922F080024A611968CA6842F02D
S31508013C304002CA60202283F8392008BD184612F0CE
S31508013C402BFFFAE7704708B5806BFFF7FBFF08BD46
S31508013C5008B5836B0268126812F4807F13D10022BB
S31508013C60DA851968CA6822F48072CA6019684A69CD
S31508013C7022F001024A6119684A6922F040024A6142
S31508013C80202283F83A20184618F0C4FC08BD08B566
S31508013C9090F83A30DBB2222B40D18368B3F5805FC6
S31508013CA00ED0036903BB03685A68836A591C81628B
S31508013CB01A70C38D013B9BB2C385F3B100202EE078
S31508013CC0826A036943B903685B68C3F3080313800F
S31508013CD0836A02338362ECE703685B68DBB21380AD
S31508013CE0836A01338362E4E703685B68826A511C6D
S31508013CF0816203F07F031370DBE70268D36823F45C
S31508013D009073D3600268536923F00103536120233A
S31508013D1080F83A3018F07EFC002000E0022008BD49
S31508013D20704708B5806BFFF7FBFF08BD704710B5F4
S31508013D30846B2268516994F83930DBB2212B0ED095
S31508013D4023685A6994F83A30DBB2222B14D0E36B14
S31508013D5043F01003E3632046FFF7E8FF10BD11F0B7
S31508013D60800FEDD00023E384D36823F0C003D3602A
S31508013D70202384F83930E3E712F0400FE7D0002317
S31508013D80E3852046FFF78BFBE1E7000010B5044603
S31508013D9002681368D068516913F00F0F17D113F031
S31508013DA0200F02D010F0200F0DD113F0800F02D092
S31508013DB010F0800F77D113F0400F03D010F0400FA9
S31508013DC040F0A08010BD2046FFF761FFFAE711F029
S31508013DD0010102D110F4907FE7D013F0010F06D04C
S31508013DE010F4807F03D0E26B42F00102E26313F024
S31508013DF0040F40D0002900F09080E26B42F00202E5
S31508013E00E26313F0020F00F09480E26B42F00402C1
S31508013E10E26313F0080F03D0E26B42F00802E26393
S31508013E20E26B002ACED013F0200F02D010F0200F3B
S31508013E3027D123685A69E36B13F0080F02D112F0F0
S31508013E40400F2AD02046FFF72AFB23685A6912F049
S31508013E50400F1ED05A6922F040025A61636BA3B122
S31508013E60364A1A65606BFCF78DF80028AAD0606B94
S31508013E70036D9847A6E713F0020F52D00029C4D163
S31508013E80CEE72046FFF703FFD3E72046FFF74EFFAD
S31508013E9098E72046FFF74AFF94E72046FFF746FFD3
S31508013EA00023E3638EE794F83930DBB2212B89D1FD
S31508013EB0A368B3F5805F16D0236A591C21621B7863
S31508013EC05360E38C013B9BB2E384002B7FF47AAF0A
S31508013ED02268D36823F08003D3602268D36843F04D
S31508013EE04003D3606EE7236A1B88C3F30803536054
S31508013EF023691BB9236A02332362E2E7236A013382
S31508013F002362DEE7D36823F04003D360202384F8D5
S31508013F103930204612F0C0FD54E713F0020F7FF442
S31508013F207FAF13F0080F3FF47BAF00293FF478AF5A
S31508013F3072E713F0080F7FF46FAF71E7413F01088D
S31508013F4008B5806B0023C385C384FFF7EFFE08BD60
S31508013F5084B010B402AC84E80E0042680B4603999B
S31508013F600B4304990B4305990B4306990B43079990
S31508013F700B4322F4FD4222F07F02134343600020E3
S31508013F805DF8044B04B07047D0F8800070470B68A1
S31508013F90C0F8803000207047032303600020704773
S31508013FA0006800F00300704710B40B688360C268AC
S31508013FB04B688C682343CC68234309690B4322F475
S31508013FC07F6222F00F021343C36000205DF8044BA1
S31508013FD070470069C0B2704782B000230193034B52
S31508013FE003440193019B186802B07047142C0140E1
S31508013FF010B40B6843624B688362C26A8B68CC68EB
S3150801400023430C69234349690B4322F0F7021343FF
S31508014010C36200205DF8044B704700000E49D1F8D1
S31508014020883043F47003C1F888300C4B1A6842F0A3
S3150801403001021A60002098601A6822F0847222F43C
S3150801404080321A60064A5A601A6822F480221A6077
S31508014050D860044B8B60704700ED00E000380240E1
S31508014060103000240080000810B582B002AB03F8B6
S31508014070011D0268546801221946A04702B010BD05
S315080140804FF0FF3070474FF0FF307047704710B55B
S3150801409014464FF0FF3392B20069FFF712FC20462F
S315080140A010BD00B583B04FF0FF3301220DF10701B2
S315080140B00069FFF774FC9DF8070003B05DF804FB7F
S315080140C0FEE7012070470000024B16221A604FF0E6
S315080140D0FF307047A0DB002010B51446012807D031
S315080140E002280DD00A4B09221A604FF0FF3006E06C
S315080140F04FF0FF3392B20748FFF7E3FB204610BDA6
S315080141004FF0FF3392B20348FFF7DBFB2046F6E791
S31508014110A0DB0020EC20002008B503460A4A1068F7
S31508014120EFF308820344934202D8074A136008BD95
S31508014130192206490220FFF7CFFF054B0C221A6008
S315080141404FF0FF30F3E700BF0800002088BB0308E3
S31508014150A0DB002010B50446FCF766FF054BA3FB60
S315080141600030000D04FB00F00A380138B0F1FF3FBA
S31508014170FBD110BD83DE1B4308B5FBF77DFA08BDED
S3150801418008B50120FFF7E6FF08BD08B50A20FFF7C5
S31508014190E1FF08BD10B582B018468DF80720013930
S315080141A0062919D8DFE801F0041B2A3B4C565600AC
S315080141B02D4C002210212046FCF766F90120FBF759
S315080141C05BFA012210212046FCF75EF901224FF421
S315080141D000412648FCF758F9012002B010BD9DF8A8
S315080141E007302BB9002220211F48FCF74DF9F3E7C8
S315080141F0012220211C48FCF747F9EDE79DF8073015
S3150801420033B901224FF400411848FCF73DF9E3E7B9
S3150801421000224FF400411548FCF736F9DCE79DF812
S3150801422007303BB9002210210F48FCF72DF9FFF79B
S31508014230ACFFD1E7012210210B48FCF725F9F6E777
S315080142404FF47A7301220DF1070109480068FEF758
S3150801425027FDC1E74FF47A739DF807200146044804
S315080142600068FEF71DFDB7E70004024000000240A2
S315080142704C0A002008B5084B186001224FF400418A
S315080142800648FCF701F90A20FBF7F6F9044A05493D
S31508014290054800F0BDFC08BD4C0A0020000002409C
S315080142A0954101081000002058DB00202DE9F04F48
S315080142B089B003908B4616469A46BDF84840DDF804
S315080142C04C90009400F059F8002853D0002C51D096
S315080142D03444A3B20593AAF108039BB2DA08013262
S315080142E006920AF10702C2F3CC02049223F00703ED
S315080142F00BF10F021344079317E053464D4630E07E
S315080143000135ADB27F08AC4208D017F0010FF7D0DE
S3150801431032462946039800F0C8FCF1E7049B994404
S315080143200136B6B2059B9E4224D00BF10704A4B20E
S31508014330BAF1070FE1D9069B09EB03084D46022797
S3150801434015F8013B00933B4632462146039800F097
S31508014350B3FC0834A4B24545F2D10AF00703BDF807
S315080143601C40002BDAD02F78E51FADB21C44073C60
S31508014370A4B2CAE709B0BDE8F08F70B4BDF80C4025
S31508014380013C1444A4B2C58FB0F84260964205D3E5
S31508014390A54207D9A24205D800201AE0A54217D896
S315080143A0A24218D9013B0B449BB2828FB0F8400058
S315080143B0884206D39A4210D9994294BF0020012017
S315080143C007E09A420BD8994294BF0020012000E0E9
S315080143D0002070BC70470020FBE70120F9E70020A8
S315080143E0F7E710B58C6800230121A04710BD10B569
S315080143F08C6800230321A04710BD10B58C680023E3
S315080144001A460421A04710BD10B58C680023012265
S315080144100421A04710BD10B58C6800230221A047CE
S3150801442010BD10B58C6800230521A04710BD2DE9E4
S31508014430F84F07468B46551E0026B0464FF0FF0A31
S315080144404FF0010906E0224659463846FFF7E9FFCB
S3150801445000284BD015F8014F1EB9FF2CF3D14E4653
S31508014460F8E7FF2C0ED0FE2C41D0EF2C3CD8DF2CE0
S3150801447011D8CF2C17D8BF2C1DD814F0800F2ED0E9
S315080144804646E7E7524659463846FFF7CAFF064603
S3150801449068B34646DEE704F00F0259463846FFF789
S315080144A0BAFF4646D6E704F00F0259463846FFF7E3
S315080144B09EFF4646CEE759463846FFF79EFF24013A
S315080144C0023404F0FE042046FFF756FE59463846E4
S315080144D0FFF79AFF2046FFF74FFE4646BAE7204602
S315080144E0FFF74AFE4646B5E74646B3E7064630466F
S315080144F0BDE8F88F2DE9F04102F1FF3E5FFA8EFE25
S315080145000EF1010E9E440022DFF844C00E4F13F847
S31508014510014B551C0CEB020804F00F063E44367D90
S3150801452088F808600232D2B25CFA85F507EB1414F2
S31508014530247D2C727345EAD18C68044B80220621AE
S31508014540A0470120BDE8F0819C410308580A0020D4
S31508014550500A002001207047F8B506460D464B68FB
S315080145601F7A1C8807FB042404F0FF040E4AFFF790
S315080145705EFF224629463046FFF753FF621CD2B238
S3150801458029463046FFF74DFF002229463046FFF7F8
S3150801459042FF5C2229463046FFF743FF012229469E
S315080145A03046FFF738FFF8BDC04103082DE9F04F43
S315080145B083B005460C4690469946A2F10A030B2B91
S315080145C00FD8DFE803F0060E0E0E0E4162670E0ED7
S315080145D00E170222FFF705FF314A21462846FFF743
S315080145E026FF4B4642462146284600F05DFD03B0AC
S315080145F0BDE8F08FD1F804A0DAF80C70BAF80AB061
S315080146004FEA9B0BBAF80030002BEAD000265FFA76
S315080146108BF30193324621462846FFF79DFF3B4619
S31508014620019A21462846FFF765FFFFF7A9FD0022F3
S3150801463021462846FFF7DBFE5F440136F6B2BAF893
S315080146400030B342E6D8CCE70122FFF7D0FE0022BC
S3150801465021462846FFF7DFFEC12221462846FFF7F5
S31508014660E0FE012221462846FFF7D5FE99F80020EB
S31508014670520821462846FFF7D4FEFFF781FD00229E
S3150801468021462846FFF7B3FEABE7064AFFF7CFFEFA
S315080146900120ACE7044AFFF7CAFE0120A7E700BFDD
S315080146A0D0410308504203085C4203082DE9F04F44
S315080146B083B005460C4690469946A2F10A030B2B90
S315080146C00FD8DFE803F0060E0E0E0E3F5E630E0EE0
S315080146D00E170222FFF785FE2F4A21462846FFF7C5
S315080146E0A6FE4B4642462146284600F015FC03B075
S315080146F0BDE8F08FD1F804A0DAF80C70BAF80AB060
S315080147004FEA9B0BBAF80030002BEAD000265FFA75
S315080147108BF30193324621462846FFF71DFF3B4698
S31508014720019A21462846FFF7E5FE0022214628463A
S31508014730FFF75DFE5F440136F6B2BAF80030B342C0
S31508014740E8D8CEE70122FFF752FE00222146284685
S31508014750FFF761FEC12221462846FFF762FE0122C4
S3150801476021462846FFF757FE99F8002052082146A8
S315080147702846FFF756FE002221462846FFF737FE50
S31508014780AFE7064AFFF753FE0120B0E7044AFFF7F1
S315080147904EFE0120ABE700BFD04103085042030893
S315080147A05C4203084218435C507800EB032080B250
S315080147B070470078704708B5FFF7FBFF18B1022864
S315080147C001D0032008BD0620FCE70020704790F9B8
S315080147D02900013080B2704708B50621FFF7E2FFCC
S315080147E008BD08B50821FFF7DDFF08BD807A7047C7
S315080147F0C07A70472DE9F84F07460E46D0F808B03B
S315080148005846FFF7D6FF82465846FFF7D4FF81463A
S31508014810BAF1010F14BF4FF0FF084FF00F085846C1
S31508014820FFF7E4FF04465846FFF7E2FF05465846F8
S31508014830FFF7D7FF602E03D910B1584461240AE067
S315080148405846FFF7C9FF402E03D910B158444124F1
S3150801485001E00BF11100B5420AD3AC4215D900208B
S315080148603877F87787F820007877B877BDE8F88F32
S3150801487000203877F87787F820007877B877F5E752
S315080148800130AC42EBD00134E4B20378FF2BF7D008
S31508014890B44205D0837808EA03034B441844F0E789
S315080148A0BAF1000F13D0BAF1020F10D003F00F02BC
S315080148B0023ABA771B097B77437803F00F0287F828
S315080148C020201B09FB7783781B093B77CEE7FB770B
S315080148D0437887F82030C3783B7703797B77437928
S315080148E0BB77C3E72DE9F04F85B0074689461646DB
S315080148F01946FFF77FFF002851D00546B868FFF72C
S315080149005AFF804697F81FB097F8204097F91D304F
S3150801491099441FFA89F10391A2B297F91E301344FB
S31508014920F61AB6B200925B4632463846FFF725FDBF
S31508014930A8B10BF1070BCBF3C40B6CB3454404F1D7
S31508014940FF3A5FFA8AFA0AF1010AB2441FFA8AFAA9
S315080149500BF1FF33DBB203F10108029717E097F970
S315080149601C001DE005EB0809039C002715F8013B0F
S3150801497000933B4632462146029800F09DF90834D9
S31508014980A4B2A945F2D10136B6B2B24503D0BBF1FC
S31508014990000FE7D1F7E7029F97F91C0000E0002016
S315080149A005B0BDE8F08F2DE9F04180460C46174663
S315080149B01E46436A98470744337893B1BFB2002528
S315080149C03A4621464046FFF78DFF80B20444A4B219
S315080149D00544ADB216F8013F002BF1D12846BDE8D2
S315080149E0F0810025FAE78368C3B190F82820B2B9A7
S315080149F05A7980F829201B7B80F82A3090F92930CA
S31508014A0090F92A209B1A9BB290F82B20402A03D0B2
S31508014A10DBB202FB03F39B0980F82C307047012AAD
S31508014A2006D05A7B80F829209B7B80F82A30E5E757
S31508014A30DA7B80F829201B7C80F82A30DEE708B566
S31508014A40002280F82820FFF7CEFF08BD08B501230C
S31508014A5080F82830FFF7C7FF08BD0000014B436205
S31508014A60704700BFCB470108014B4362704700BF3F
S31508014A70CF47010870B50D46097871B1064600247D
S31508014A803046FFF7B7FE96F91C301C44A4B215F858
S31508014A90011F0029F4D1204670BD0024FBE7000060
S31508014AA083688B4207D010B504468160FFF79BFFE8
S31508014AB0014B636210BD7047CB47010810B50C68FE
S31508014AC0A04710BD38B504460D46836B02209847AA
S31508014AD000230A2229462046FFF7F0FF0546A36B65
S31508014AE003209847A36B00209847284638BD38B558
S31508014AF004460D46836B02209847A36B012098470D
S31508014B000023142229462046FFF7D8FF04F13C0367
S31508014B10172229462046FFF7D1FFA36B00209847A5
S31508014B2038BD70B504460D46836B02209847A36BC2
S31508014B30012098470023152229462046FFF7BEFF84
S31508014B40064620B9A36B00209847304670BD04F18C
S31508014B503C03172229462046FFF7B0FFF2E700B5C6
S31508014B6083B002AB03F8012D0F22FFF7A7FF03B0AD
S31508014B705DF804FB10B5C285038600F12E033222C7
S31508014B80FFF79CFF10BD00B583B00DF10603462261
S31508014B90FFF794FFBDF8060003B05DF804FB00B506
S31508014BA083B00DF106034722FFF788FFBDF806001B
S31508014BB003B05DF804FB08B500234822FFF77EFF22
S31508014BC008BD10B504464168FFF7DDFF208061681E
S31508014BD02046FFF7E4FF608061682046FFF7EBFF98
S31508014BE0E07404F13C03172261682046FFF766FF6B
S31508014BF010BD10B504464168FFF764FF034608B9BE
S31508014C00184610BD2046FFF7DCFF0123F8E7000030
S31508014C102DE9F04104460F46904600258560C5609A
S31508014C2045740126067422238374856180F83460ED
S31508014C30FFF714FF84F8286084F8295084F82A506D
S31508014C40402384F82B3084F82C50054BA363676006
S31508014C50C7F808802046FFF7CCFFBDE8F08100BF02
S31508014C608154010808B54168FFF741FF08BD10B531
S31508014C700446836903B1984761682046FFF751FFE7
S31508014C8010BD08B50A464168FFF769FF08BD08B5B2
S31508014C90002310224168FFF711FF08BD08B500235C
S31508014CA011224168FFF70AFF08BD08B513460A46EF
S31508014CB04168FFF75FFF08BD38B54568C1850286BB
S31508014CC080F833309DF8103080F8323000F12E0329
S31508014CD03B222946FFF7F2FE38BD80F834107047AB
S31508014CE0C37C282B04D0022B0CBF0320012070475C
S31508014CF0FF207047C37C302B06D010B50446FFF75A
S31508014D00EFFF84F8340010BDFF2380F8343080F8B3
S31508014D1035307047002282800388013BC3800272C6
S31508014D2070470288838813449BB2838041888B42EB
S31508014D300DD2037A01330372C3881A4492B291429F
S31508014D409CBF01F1FF3292B2C28001207047002058
S31508014D507047C36842891A44002103F8011B9A4225
S31508014D60FBD1704710B4C3888B4234BF002301239B
S31508014D70914294BF00210121848843EA01009442AB
S31508014D808CBF002000F001000B4018435DF8044B6E
S31508014D90704700230B8083884B804389013B8B80B6
S31508014DA0C388CB80704708B54B884A79012A03D056
S31508014DB0032A08D01A4602E003F1080292B21946FC
S31508014DC0FFF7D0FF08BDA3F108011A468BB2F6E733
S31508014DD070B49DF80C60C4684589AD088088121ABC
S31508014DE0D2B212FB05F2880810FA82F2490001F0E4
S31508014DF0060136B903208840C0B2A55C25EA000041
S31508014E00A05403F0030303FA01F1A35C1943A15467
S31508014E1070BC7047C368428903EB4202002103F85C
S31508014E20011B9A42FBD1704730B583B04C88838801
S31508014E30A34206D8C388A34203D30D884389AB424C
S31508014E4001D803B030BD8B79009222462946FFF777
S31508014E50BFFFF6E7F8B507460D460C7900260CE0C4
S31508014E60324629463846FFF7DFFF09E02B8801332A
S31508014E702B80640014F0FF041CD014F0800FEFD1CE
S31508014E806B79032BF5D801A252F823F06D4E010870
S31508014E909D4E0108A54E0108AD4E01086B880133E8
S31508014EA06B80E6E72B88013B2B80E2E76B88013BA9
S31508014EB06B80DEE7F8BD00BFF8B507460D460C79ED
S31508014EC0012606E02B8801332B80A40014F0FF0489
S31508014ED020D0A309AB71324629463846FFF7A4FF0D
S31508014EE06B79032BF1D801A252F823F0C54E0108BC
S31508014EF0FD4E0108054F01080D4F01086B88013366
S31508014F006B80E2E72B88013B2B80DEE76B88013B50
S31508014F106B80DAE7F8BD00BF38B51D464C68143A10
S31508014F20342A1CD8DFE802F03E461B501B1B1B1B0C
S31508014F301B1B1B1B1B1B1B1B1B1B1B1B1B1B1B1BB2
S31508014F4037311B1B1B1B2A1B1B1B1B1B1B1B1B1D5F
S31508014F501B1B1B1B1B1B1B1B1B1B565A5E00012302
S31508014F6041E029462046FFF71EFF08B901233AE02A
S31508014F7029462046FFF76EFF012334E00022294621
S31508014F802046FFF751FF01232DE029462046FFF76A
S31508014F9093FF012327E0012229462046FFF744FF14
S31508014FA0012320E02046FFF7B5FE2046FFF732FF32
S31508014FB0012318E02046FFF7B4FE034698B12046C0
S31508014FC0FFF728FF01230EE029462046FFF7E1FEF9
S31508014FD0012308E063892B80012304E063882B8081
S31508014FE0012300E00223184638BD30B4C468458958
S31508014FF0AD088088121AD2B212FB05F2880810FA97
S3150801500082F2490001F0060103208840C0B203F08C
S3150801501003038B40A15C21EA00011943A15430BC6A
S3150801502070474A88838893420DD8C38893420AD326
S3150801503010B50C884389A34200D810BD8B79214647
S31508015040FFF7D3FFF9E7704770B506460D460C79A9
S315080150500BE029463046FFF7E4FF09E02B880133C8
S315080150602B80640014F0FF041CD014F0800FF0D1DB
S315080150706B79032BF5D801A252F823F05D5001088C
S315080150808D500108955001089D5001086B88013320
S315080150906B80E6E72B88013B2B80E2E76B88013BB7
S315080150A06B80DEE770BD00BF38B51D464C68143A03
S315080150B0342A1CD8DFE802F030381B421B1B1B1BA5
S315080150C01B1B1B1B1B1B1B1B1B1B1B1B1B1B1B1B21
S315080150D01B1B1B1B1B1B2A1B1B1B1B1B1B1B1B1D00
S315080150E01B1B1B1B1B1B1B1B1B1B484C500001239B
S315080150F033E029462046FFF756FE08B901232CE07E
S3150801510029462046FFF7A0FF012326E02946204627
S31508015110FFF787FF012320E02046FFF71AFE204606
S31508015120FFF7F8FD012318E02046FFF7FAFD0346CD
S3150801513098B12046FFF70DFE01230EE029462046C9
S31508015140FFF727FE012308E063892B80012304E08A
S3150801515063882B80012300E00223184638BD2DE918
S31508015160F04782B082460C4690461E46072B17D951
S31508015170A3F1080525F0070501F108031D44ADB2A1
S31508015180FF274FF0000900974B46424621465046F5
S31508015190FFF792FD0834A4B2AC42F4D106F0070633
S315080151A016B902B0BDE8F08786F00703013303F0AC
S315080151B00703FF2202FA03F3DBB2009300234246F8
S315080151C021465046FFF778FDEBE72DE9F04782B017
S315080151D08246884614461E46072B17D9A3F10805A9
S315080151E025F0070502F108031D44ADB2FF274FF06C
S315080151F0010900974B46224641465046FFF75CFD9A
S315080152000834A4B2AC42F4D106F0070616B902B0C6
S31508015210BDE8F08786F00703013303F00703FF2291
S3150801522002FA03F3DBB200930123224641465046B4
S31508015230FFF742FDEBE72DE9F04182B006460F463E
S3150801524015469846BDF820400094FFF796F810B920
S3150801525002B0BDE8F08143462A4639463046FFF793
S315080152607EFF23462A4639463046FFF7AEFF08F148
S31508015270FF31394423462A4689B23046FFF7A5FF4E
S31508015280013C2C444346A2B239463046FFF767FF34
S31508015290DEE72DE9F04180460F4614461E46BDF865
S315080152A018501544ADB23346224639464046FFF7F3
S315080152B056FF0134A4B2AC42F5D1BDE8F0812DE91F
S315080152C0F04182B005460E4617469846BDF820407D
S315080152D00094FFF752F810B902B0BDE8F0810094C6
S315080152E043463A4631462846FFF7D3FFF4E70020FE
S315080152F070472DE9F843054617461C464E68A2F144
S315080153001703302B1AD8DFE803F0201919191919D0
S315080153101919191919191919191919191919195EA9
S315080153207A191919195E19191919191919197A19D7
S3150801533019191919191919191952580023463A46EA
S315080153403146FFF7BBFBBDE8F883234617223146F2
S31508015350FFF7B4FB31462846FFF715FCB4F804906D
S315080153606FEA090981441FFA89F931462846FFF788
S315080153700AFC2788FF430744BFB231462846FFF790
S315080153800EFCB4F806806FEA080880441FFA88F80C
S3150801539031462846FFF703FC6388DB431844A4F823
S315080153A00090A4F80280A780E0800120CBE731466F
S315080153B0FFF7E9FB20800120C5E73146FFF7EFFB40
S315080153C020800120BFE73146FFF7E9FBB4F80280E8
S315080153D06FEA080880441FFA88F831462846FFF71D
S315080153E0D2FB2388DB4318442080A4F80280234695
S315080153F03A4631462846FFF761FB0120A3E73146C5
S31508015400FFF7CDFBB4F802806FEA080880441FFA5B
S3150801541088F831462846FFF7B6FB2388DB4318444C
S315080154202080A4F802806379023303F003036371D1
S3150801543023463A4631462846FFF740FB012082E7D4
S3150801544008B54268044B9A4200D008BD5B684360C0
S31508015450FFF7B7FBF9E700BF8C00002008B54368E2
S31508015460054A93421CBF53604260034B034A1A60C4
S31508015470FFF7A7FB08BD00BF8C000020F352010807
S315080154807047FF2808D9B0F5007F07D3B0F5407FEC
S3150801549034BFA520A7207047A1207047A3207047D5
S315080154A070B584B0841840F2FE339C4202DD0020B8
S315080154B004B070BD15460E460446FFF7E2FF0E23FB
S315080154C00293019500960123E2B2C1B20248FBF7A5
S315080154D017FB0120ECE700BFF01F002070B586B06E
S315080154E0841840F2FE339C4202DD002006B070BDEE
S315080154F015460E460446FFF7C4FF0E23029301958F
S3150801550005AB00930123E2B2C1B20648FBF7F8FAEC
S315080155109DF814209DF8153043EA022333800120B3
S31508015520E4E700BFF01F002070B584B0841840F28C
S31508015530FE339C4202DD002004B070BD15460E46BE
S315080155400446FFF79EFF0E23029301950096012359
S31508015550E2B2C1B20248FBF7D3FA0120ECE700BF79
S31508015560F01F0020FF2808D9B0F5007F07D3B0F552
S31508015570407F34BFA420A6207047A0207047A220F0
S315080155807047000070B584B0841840F2FE339C421F
S3150801559002DD002004B070BD15460E460446FFF72D
S315080155A0E1FF0E230293019500960123E2B2C1B2EF
S315080155B00348FBF707FA0420FAF75EF80120E9E742
S315080155C0F01F002070B584B0841840F2FE339C4267
S315080155D002DD002004B070BD15460E460446FFF7ED
S315080155E0C1FF0E230293019500960123E2B2C1B2CF
S315080155F00348FBF7E7F90520FAF73EF80120E9E742
S31508015600F01F002030B587B00B8819128DF81410D9
S315080156108DF81530811840F2FE33994202DD0020DB
S3150801562007B030BD15460446FFF79CFF0E230293CB
S31508015630019505AB00930123E2B2C1B20348FBF71A
S31508015640C1F90520FAF718F80120E9E7F01F00204B
S315080156500170002242708270C2704260C2600261AB
S315080156600D4941610D498161C26102624262028549
S315080156704285C26240F6B83101860949416341F261
S3150801568088310187428702218187C287082180F8EC
S31508015690401080F841207047006CCA88009435771D
S315080156A0801A060070B582B0047861F07F018DF822
S315080156B000108DF801208DF802309DF818308DF80C
S315080156C003309DF81C308DF80430032C01DD02B03F
S315080156D070BD0B4E0B4D002236F814102846FAF70A
S315080156E0D3FE4FF47A73052269460748FDF7D8FABF
S315080156F0012236F814102846FAF7C6FEE7E700BF76
S31508015700A0000020000C02406C1D002000B583B0EB
S31508015710CBB20193C1F307230093C1F307430A0EE2
S315080157202D21FFF7BFFF03B05DF804FB00B583B079
S31508015730084A8A42A8BF0A46D3B20193C2F307238D
S315080157400093C2F30743120E2721FFF7ABFF03B0FD
S315080157505DF804FB00FE7F0000B583B04FF6FF72CB
S315080157608A42A8BF0A46D3B20193C2F3072300931C
S31508015770C2F30743120E2821FFF794FF03B05DF821
S3150801578004FB30B583B005460C464FF6FF728A42D4
S31508015790A8BF0A46D3B20193C2F307230093C2F303
S315080157A00743120E2621FFF77DFF21462846FFF7FC
S315080157B0D3FF03B030BD2DE9F04383B006460D464D
S315080157C00423019300240094234622462021FFF74F
S315080157D069FF2F0EC5F30748C5F30729EDB20195F1
S315080157E0CDF8009043463A4621213046FFF75AFF45
S315080157F00195CDF8009043463A462D213046FFF7EC
S3150801580051FF019400942346224620213046FFF792
S3150801581049FF03B0BDE8F08300B583B0019200915A
S3150801582000221021FFF73EFF03B05DF804FB0000DC
S31508015830042B00D970472DE9F0411C4616460D4642
S31508015840DFF834800A4F002238F813103846FAF781
S315080158501BFEC823B2B229460648FDF721FA0122E2
S3150801586038F814103846FAF70FFEBDE8F08100BF84
S31508015870000C02406C1D0020A0000020F0B587B086
S315080158800546274B93E8030004908DF81410C823A6
S31508015890052204A92348FDF703FA29780122224B98
S315080158A033F811102148FAF7EFFD214F2B78214ED5
S315080158B0012237F813103046FAF7E6FD0A20F9F700
S315080158C0DBFEA1238DF8083000248DF809408DF8F8
S315080158D00A408DF80B408DF80C402B78052202A959
S315080158E02846FFF7A5FF0A20F9F7C6FEAD238DF86E
S315080158F000308DF801408DF802408DF803408DF88F
S3150801590004402B78052269462846FFF791FF2B7834
S31508015910224637F813103046FAF7B6FD07B0F0BD40
S315080159204CB703086C1D0020A0000020000C0240A3
S31508015930A80000200008024030B591B00446057859
S315080159403A4B03F1280292E803000E908DF83C10B9
S3150801595003F1380292E803000C908DF8341003F134
S31508015960400292E803000A908DF82C1093228DF8D4
S31508015970202000228DF821208DF822208DF8232061
S315080159808DF8242003F1480292E8030006908DF869
S315080159901C1003F1500292E8030004908DF81410CC
S315080159A003F1580292E8030002908DF80C10603357
S315080159B093E8030000908DF804102B4605220EA9E2
S315080159C02046FFF735FF2B4605220EA92046FFF78D
S315080159D02FFF2B4605220CA92046FFF729FF2B4648
S315080159E005220AA92046FFF723FF2B46052208A907
S315080159F02046FFF71DFF2B46052206A92046FFF77D
S31508015A0017FF2B46052204A92046FFF711FF2B464F
S31508015A10052202A92046FFF70BFF2B4605226946F8
S31508015A202046FFF705FF11B030BD00BF4CB703088C
S31508015A3030B58BB004460578264B03F1080292E887
S31508015A40030008908DF8241003F1100292E8030070
S31508015A5006908DF81C1003F1680292E80300049081
S31508015A608DF81410203393E8030002908DF80C107A
S31508015A7080238DF8003000238DF801308DF802302F
S31508015A808DF803308DF804302B46052208A92046E7
S31508015A90FFF7CEFE2B46052208A92046FFF7C8FECA
S31508015AA02B46052206A92046FFF7C2FE2B460522EC
S31508015AB004A92046FFF7BCFE2B46052202A920466B
S31508015AC0FFF7B6FE2B46052269462046FFF7B0FECC
S31508015AD00BB030BD4CB7030830B587B0044605781E
S31508015AE01B4B93E8030004908DF81410AD238DF831
S31508015AF0083000238DF809308DF80A308DF80B30FF
S31508015B008DF80C30A1228DF800208DF801308DF822
S31508015B1002308DF803308DF804302B46052204A98E
S31508015B202046FFF785FE2B46052204A92046FFF7E6
S31508015B307FFE2B46052202A92046FFF779FE2B4652
S31508015B40052269462046FFF773FE07B030BD00BF40
S31508015B5054B7030830B593B0044605783D4B03F1B5
S31508015B60700292E8030010908DF84410A5228DF872
S31508015B70382000228DF839208DF83A208DF83B20FF
S31508015B808DF83C2003F1780103C90C908DF8341087
S31508015B9003F1800103C90A908DF82C1003F18801DD
S31508015BA003C908908DF8241003F1900103C90690E2
S31508015BB08DF81C1003F1980103C904908DF814108F
S31508015BC0A0218DF808108DF809208DF80A208DF886
S31508015BD00B208DF80C200B4493E8030000908DF8F8
S31508015BE004102B46052210A92046FFF721FE2B4655
S31508015BF005220EA92046FFF71BFE2B4605220CA9F6
S31508015C002046FFF715FE2B4605220AA92046FFF76F
S31508015C100FFE2B46052208A92046FFF709FE2B464B
S31508015C20052206A92046FFF703FE2B46052204A9ED
S31508015C302046FFF7FDFD2B46052202A92046FFF760
S31508015C40F7FD2B46052269462046FFF7F1FD13B0FD
S31508015C5030BD00BF4CB703082DE9F0410446904614
S31508015C601F469DF818509DF81C6001291CD0022971
S31508015C701DD02046FFF76EFFC4F834804146204602
S31508015C80FFF754FD278639462046FFF77AFD84F843
S31508015C90405084F841609DF8203032462946204616
S31508015CA0FFF7BAFDBDE8F081FFF7C2FEE1E7FFF7AE
S31508015CB043FEDEE782B001238DF807309DF8070021
S31508015CC002B0704700B583B0059901910499009116
S31508015CD001460448FCF74DFD003018BF012003B00A
S31508015CE05DF804FBD80F002000B583B00599019132
S31508015CF00499009101460448FCF702FE003018BFDA
S31508015D00012003B05DF804FBD80F00202DE9F04F00
S31508015D108BB00746002500956A4B5A6C42F400621F
S31508015D205A645A6C02F400620092009A01951A6B41
S31508015D3042F480021A631A6B02F480020192019AF4
S31508015D4002951A6B42F002021A631A6B02F00202FA
S31508015D500292029A03951A6B42F004021A631A6BAD
S31508015D6002F004020392039A04951A6B42F00802A0
S31508015D701A631B6B03F008030493049B072305931B
S31508015D804FF00209CDF818900795032608960C24BA
S31508015D90099405A94C48FAF7FBF94FF410630593E2
S31508015DA0CDF8189007950896099405A94748FAF772
S31508015DB0EFF94FF00408CDF81480CDF8189007953F
S31508015DC00896099405A94248FAF7E2F92A460521EF
S31508015DD03120F9F7DFFE3120F9F70EFF3D4C3E4B36
S31508015DE023664FF0006BC4F864B0A566E5664FF408
S31508015DF0806AC4F870A04FF4805363674FF48043F8
S31508015E00A3672023E3674FF44033C4F88030C4F80E
S31508015E108480C4F888604FF40003C4F88C304FF4CA
S31508015E200019C4F8909004F16003BB65C4F8987032
S31508015E301846F9F7E7FF04F16000F9F745FF274B24
S31508015E40C4F8C030C4F8C4B04023C4F8C830C4F894
S31508015E50CC50C4F8D0A04FF48053C4F8D4304FF4D2
S31508015E608043C4F8D8302023C4F8DC304FF44033DB
S31508015E70C4F8E030C4F8E480C4F8E8604FF40003DD
S31508015E80C4F8EC30C4F8F09004F1C006FE65C4F815
S31508015E90F8703046F9F7B6FF3046F9F715FF2A4686
S31508015EA006213B20F9F776FE3B20F9F7A5FE2A469F
S31508015EB006214520F9F76EFE4520F9F79DFE0BB040
S31508015EC0BDE8F08F00380240000402400008024095
S31508015ED0000C0240D80F002058640240A06402401A
S31508015EE010B5144B144A1A6000225A609A60DA6097
S31508015EF01A614FF4804159619A61FFF7DBFE012867
S31508015F0001D0022010BD0B4C00212046FFF7FEFEF2
S31508015F1004F590712046FCF771F908B10120F1E703
S31508015F204FF400612046FCF761FB003018BF0120E1
S31508015F30E8E700BFD80F0020002C014008B5024849
S31508015F40FBF7CEFF08BD00BFD80F002008B5024BEE
S31508015F50D86DFAF72BF808BDD80F002008B5024B03
S31508015F60986DFAF723F808BDD80F002008B502483E
S31508015F70FCF7D6FD08BD00BFD80F002008B50146BD
S31508015F800148FBF7F0FF08BDD80F0020000000000C
S31508015F9008B510EE100AF2F79FFA02460B460EA153
S31508015FA0D1E90001F2F71AFC0022094BF2F734F99C
S31508015FB0F2F7E2FD07EE900AFCEEE77A054B1A685E
S31508015FC0C2ED0B7AC3ED037A08BD00BFAFF30080BB
S31508015FD00000F03F10120020000000002A759541CC
S31508015FE070B582B000250195174B1A6C42F0010273
S31508015FF01A641B6C03F001030193019B134C4FF0C8
S31508016000804323600126DE606560A560DFED107AB6
S3150801601087EE800AF7EE007A30EE670ABCEEC00A10
S3150801602084ED030A256165612046FDF71DFA2046C0
S31508016030FDF7D7F82A4631461C20F9F7ABFD1C2097
S31508016040F9F7DAFD02B070BD0038024010120020DF
S3150801605050A9AB4CF0B5ADF5597D2C4A1378527859
S315080160602B49898F00912B4945A81BF01DFC0A2253
S3150801607045A94DA8F8F738FB18B100200DF5597D4B
S31508016080F0BD45AA244905A81BF00EFC05A8F2F7A0
S31508016090C3FD04AB024605A94DA8F8F73DFC002847
S315080160A030D11B4B1B6C002B1BDD1C4C00251C4ED9
S315080160B0174FE3680293A368019363680093236803
S315080160C02A46314605A81BF0EFFB04AB024605A993
S315080160D04DA8F8F721FCB8B9013510343B6CAB4231
S315080160E0E7DC4DA8F8F78FFD044609498B8F013384
S315080160F021F83C3F02220520FFF784FAB4FA84F01E
S315080161004009BBE70020B9E70020B7E7980000205F
S3150801611010120020DCBB0308F4BB03088C24002002
S31508016120F8BB03082DE9F041ADF5567D0A4A137807
S3150801613052780A49898F0091094943A81BF0B4FB93
S315080161400A2243A94BA8F8F7CFFA58B100200DF552
S31508016150567DBDE8F08100BF98000020101200208E
S315080161600CBC0308BE4E7278BE4D1346294603A8D9
S315080161701BF09AFB03A8F2F74FFD02AB024603A9EF
S315080161804BA8F8F7C9FB32781346294603A81BF032
S315080161908BFB03A8F2F740FD02AB024603A94BA805
S315080161A0F8F7BAFBB04CB4F844201346294603A8BD
S315080161B01BF07AFB03A8F2F72FFD02AB024603A9EF
S315080161C04BA8F8F7A9FBA28F1346294603A81BF08B
S315080161D06BFB03A8F2F720FD02AB024603A94BA805
S315080161E0F8F79AFB94F84620A04F1346394603A8B8
S315080161F01BF05AFB03A8F2F70FFD02AB024603A9EF
S315080162004BA8F8F789FB94F847201346294603A8B3
S315080162101BF04AFB03A8F2F7FFFC02AB024603A9EF
S315080162204BA8F8F779FBA36C1A46294603A81BF075
S315080162303BFB03A8F2F7F0FC02AB024603A94BA805
S31508016240F8F76AFBE36C1A46294603A81BF02CFBF0
S3150801625003A8F2F7E1FC02AB024603A94BA8F8F73B
S315080162605BFB94F850201346294603A81BF01CFB38
S3150801627003A8F2F7D1FC02AB024603A94BA8F8F72B
S315080162804BFBB4F8B8201346294603A81BF00CFBB0
S3150801629003A8F2F7C1FC02AB024603A94BA8F8F71B
S315080162A03BFB94F8B42094F8B4305BB252B2394649
S315080162B003A81BF0F9FA03A8F2F7AEFC02AB0246F3
S315080162C003A94BA8F8F728FBD4F8B8301A4629468B
S315080162D003A81BF0E9FA03A8F2F79EFC02AB0246F3
S315080162E003A94BA8F8F718FBB4F8BC2013462946AE
S315080162F003A81BF0D9FA03A8F2F78EFC02AB0246F3
S3150801630003A94BA8F8F708FBB4F8BE20134629469B
S3150801631003A81BF0C9FA03A8F2F77EFC02AB0246F2
S3150801632003A94BA8F8F7F8FAB4F8C020134629468A
S3150801633003A81BF0B9FA03A8F2F76EFC02AB0246F2
S3150801634003A94BA8F8F7E8FA94F8C2201346294698
S3150801635003A81BF0A9FA03A8F2F75EFC02AB0246F2
S3150801636003A94BA8F8F7D8FA94F8C3201346394677
S3150801637003A81BF099FA03A8F2F74EFC02AB0246F2
S3150801638003A94BA8F8F7C8FA94F8C4201346294676
S3150801639003A81BF089FA03A8F2F73EFC02AB0246F2
S315080163A003A94BA8F8F7B8FA94F8E024DFF8C080F7
S315080163B01346414603A81BF077FA03A8F2F72CFC0B
S315080163C002AB024603A94BA8F8F7A6FA94F84425A6
S315080163D01346414603A81BF067FA03A8F2F71CFC0B
S315080163E002AB024603A94BA8F8F796FA94F8442596
S315080163F01346294603A81BF057FA03A8F2F70CFC23
S3150801640002AB024603A94BA8F8F786FAB4F8462563
S31508016410B4F84635294603A81BF046FA03A8F2F74D
S31508016420FBFB02AB024603A94BA8F8F775FAB4F8C9
S3150801643048251346294603A81BF036FA03A8F2F79E
S31508016440EBFB02AB024603A94BA8F8F765FA94F8E9
S315080164504A2594F84A35294603A81BF025FA09E086
S315080164609800002024BC0308101200202CBC030845
S3150801647034BC030803A8F2F7CFFB02AB024603A913
S315080164804BA8F8F749FA94F84B2594F84B35294661
S3150801649003A81BF009FA03A8F2F7BEFB02AB0246F2
S315080164A003A94BA8F8F738FA94F84C2594F84C3513
S315080164B0294603A81BF0F8F903A8F2F7ADFB02ABCE
S315080164C0024603A94BA8F8F727FA73681A4629461C
S315080164D003A81BF0E9F903A8F2F79EFB02AB0246F3
S315080164E003A94BA8F8F718FAD4F850351A462946DD
S315080164F003A81BF0D9F903A8F2F78EFB02AB0246F3
S3150801650003A94BA8F8F708FAD4F854351A462946C8
S3150801651003A81BF0C9F903A8F2F77EFB02AB0246F2
S3150801652003A94BA8F8F7F8F9328A1346294603A8AE
S315080165301BF0BAF903A8F2F76FFB02AB024603A9EF
S315080165404BA8F8F7E9F9328B1346294603A81BF03D
S31508016550ABF903A8F2F760FB02AB024603A94BA805
S31508016560F8F7DAF994F858251346294603A81BF0D3
S315080165709BF903A8F2F750FB02AB024603A94BA805
S31508016580F8F7CAF9D4F85C351A46294603A81BF068
S315080165908BF903A8F2F740FB02AB024603A94BA805
S315080165A0F8F7BAF9327E1346394603A81BF07CF987
S315080165B003A8F2F731FB02AB024603A94BA8F8F789
S315080165C0ABF994F860251346294603A81BF06CF924
S315080165D003A8F2F721FB02AB024603A94BA8F8F779
S315080165E09BF994F861251346294603A81BF05CF923
S315080165F003A8F2F711FB02AB024603A94BA8F8F769
S315080166008BF994F862251346294603A81BF04CF921
S3150801661003A8F2F701FB02AB024603A94BA8F8F758
S315080166207BF994F863251346294603A81BF03CF920
S3150801663003A8F2F7F1FA02AB024603A94BA8F8F749
S315080166406BF994F864251346294603A81BF02CF91F
S3150801665003A8F2F7E1FA02AB024603A94BA8F8F739
S315080166605BF994F865251346294603A81BF01CF91E
S3150801667003A8F2F7D1FA02AB024603A94BA8F8F729
S315080166804BF994F86C251346394603A81BF00CF907
S3150801669003A8F2F7C1FA02AB024603A94BA8F8F719
S315080166A03BF994F86C251346294603A81BF0FCF818
S315080166B003A8F2F7B1FA02AB024603A94BA8F8F709
S315080166C02BF994F86D251346294603A81BF0ECF817
S315080166D003A8F2F7A1FA02AB024603A94BA8F8F7F9
S315080166E01BF994F86E251346294603A81BF0DCF816
S315080166F003A8F2F791FA02AB024603A94BA8F8F7E9
S315080167000BF9B4F870251346294603A81BF0CCF8F3
S3150801671003A8F2F781FA02AB024603A94BA8F8F7D8
S31508016720FBF8264694F872252C461346294603A8F3
S315080167301BF0BAF803A8F2F76FFA02AB024603A9EF
S315080167404BA8F8F7E9F8BE4D95F9202013463946C6
S3150801675003A81BF0A9F803A8F2F75EFA02AB0246F2
S3150801676003A94BA8F8F7D8F896F9782513463946B8
S3150801677003A81BF099F803A8F2F74EFA02AB0246F2
S3150801678003A94BA8F8F7C8F82A8C1346214603A88B
S315080167901BF08AF803A8F2F73FFA02AB024603A9EF
S315080167A04BA8F8F7B9F86A8C1346214603A81BF0DB
S315080167B07BF803A8F2F730FA02AB024603A94BA805
S315080167C0F8F7AAF8AA8C1346214603A81BF06CF819
S315080167D003A8F2F721FA02AB024603A94BA8F8F778
S315080167E09BF8EA8C1346214603A81BF05DF803A81B
S315080167F0F2F712FA02AB024603A94BA8F8F78CF88E
S315080168002A8D1346214603A81BF04EF803A8F2F772
S3150801681003FA02AB024603A94BA8F8F77DF86A8D7D
S315080168201346214603A81BF03FF803A8F2F7F4F92B
S3150801683002AB024603A94BA8F8F76EF8AA8D1346D0
S31508016840214603A81BF030F803A8F2F7E5F902ABD5
S31508016850024603A94BA8F8F75FF8EA8D13462146C5
S3150801686003A81BF021F803A8F2F7D6F902AB0246F2
S3150801687003A94BA8F8F750F895F830201346214696
S3150801688003A81BF011F803A8F2F7C6F902AB0246F2
S3150801689003A94BA8F8F740F895F831201346214685
S315080168A003A81BF001F803A8F2F7B6F902AB0246F2
S315080168B003A94BA8F8F730F895F832201346214674
S315080168C003A81AF0F1FF03A8F2F7A6F902AB0246EC
S315080168D003A94BA8F8F720F895F833201346214663
S315080168E003A81AF0E1FF03A8F2F796F902AB0246EC
S315080168F003A94BA8F8F710F895F834201346214652
S3150801690003A81AF0D1FF03A8F2F786F902AB0246EB
S3150801691003A94BA8F8F700F895F835201346214640
S3150801692003A81AF0C1FF03A8F2F776F902AB0246EB
S3150801693003A94BA8F7F7F0FF95F836201346214629
S3150801694003A81AF0B1FF03A8F2F766F902AB0246EB
S3150801695003A94BA8F7F7E0FF95F837201346214618
S3150801696003A81AF0A1FF03A8F2F756F902AB0246EB
S3150801697003A94BA8F7F7D0FF95F838201346214607
S3150801698003A81AF091FF03A8F2F746F902AB0246EB
S3150801699003A94BA8F7F7C0FF95F8392013462146F6
S315080169A003A81AF081FF03A8F2F736F902AB0246EB
S315080169B003A94BA8F7F7B0FF95F83A2013462146E5
S315080169C003A81AF071FF03A8F2F726F902AB0246EB
S315080169D003A94BA8F7F7A0FF95F83B2013462146D4
S315080169E003A81AF061FF03A8F2F716F902AB0246EB
S315080169F003A94BA8F7F790FFB6F878251346214661
S31508016A0003A81AF051FF03A8F2F706F902AB0246EA
S31508016A1003A94BA8F7F780FFB6F87A25134621464E
S31508016A2003A81AF041FF03A8F2F7F6F802AB0246EB
S31508016A3003A94BA8F7F770FFB6F87C2502E000BF5B
S31508016A40980000201346214603A81AF02DFF03A833
S31508016A50F2F7E2F802AB024603A94BA8F7F75CFF87
S31508016A60B6F87E251346214603A81AF01DFF03A88A
S31508016A70F2F7D2F802AB024603A94BA8F7F74CFF87
S31508016A80B6F880251346214603A81AF00DFF03A878
S31508016A90F2F7C2F802AB024603A94BA8F7F73CFF87
S31508016AA0B6F882251346214603A81AF0FDFE03A867
S31508016AB0F2F7B2F802AB024603A94BA8F7F72CFF87
S31508016AC0B6F884251346214603A81AF0EDFE03A855
S31508016AD0F2F7A2F802AB024603A94BA8F7F71CFF87
S31508016AE0B6F886251346214603A81AF0DDFE03A843
S31508016AF0F2F792F802AB024603A94BA8F7F70CFF87
S31508016B00B6F888251346214603A81AF0CDFE03A830
S31508016B10F2F782F802AB024603A94BA8F7F7FCFE87
S31508016B20B6F88A251346214603A81AF0BDFE03A81E
S31508016B30F2F772F802AB024603A94BA8F7F7ECFE87
S31508016B4095F83C201346214603A81AF0ADFE03A882
S31508016B50F2F762F802AB024603A94BA8F7F7DCFE87
S31508016B6095F944201346394603A81AF09DFE03A851
S31508016B70F2F752F802AB024603A94BA8F7F7CCFE87
S31508016B8095F844201346214603A81AF08DFE03A85A
S31508016B90F2F742F802AB024603A94BA8F7F7BCFE87
S31508016BA095F845201346214603A81AF07DFE03A849
S31508016BB0F2F732F802AB024603A94BA8F7F7ACFE87
S31508016BC095F846201346214603A81AF06DFE03A838
S31508016BD0F2F722F802AB024603A94BA8F7F79CFE87
S31508016BE096F88C251346214603A81AF05DFE03A8DC
S31508016BF0F2F712F802AB024603A94BA8F7F78CFE87
S31508016C0095F847201346214603A81AF04DFE03A816
S31508016C10F2F702F802AB024603A94BA8F7F77CFE86
S31508016C2096F88D251346214603A81AF03DFE03A8BA
S31508016C30F1F7F2FF02AB024603A94BA8F7F76CFE80
S31508016C4096F88E251346214603A81AF02DFE03A8A9
S31508016C50F1F7E2FF02AB024603A94BA8F7F75CFE80
S31508016C6096F88F251346214603A81AF01DFE03A898
S31508016C70F1F7D2FF02AB024603A94BA8F7F74CFE80
S31508016C8096F890251346214603A81AF00DFE03A887
S31508016C90F1F7C2FF02AB024603A94BA8F7F73CFE80
S31508016CA096F891251346214603A81AF0FDFD03A877
S31508016CB0F1F7B2FF02AB024603A94BA8F7F72CFE80
S31508016CC0344696F992253D461346394603A81AF0E5
S31508016CD0EBFD03A8F1F7A0FF02AB024603A94BA8F7
S31508016CE0F7F71AFE96F993251346394603A81AF0BB
S31508016CF0DBFD03A8F1F790FF02AB024603A94BA8F7
S31508016D00F7F70AFE96F994251346394603A81AF0A9
S31508016D10CBFD03A8F1F780FF02AB024603A94BA8F6
S31508016D20F7F7FAFD96F995251346394603A81AF099
S31508016D30BBFD03A8F1F770FF02AB024603A94BA8F6
S31508016D40F7F7EAFD96F996251346394603A81AF088
S31508016D50ABFD03A8F1F760FF02AB024603A94BA8F6
S31508016D60F7F7DAFD96F997251346394603A81AF077
S31508016D709BFD03A8F1F750FF02AB024603A94BA8F6
S31508016D80F7F7CAFD96F998251346394603A81AF066
S31508016D908BFD03A8F1F740FF02AB024603A94BA8F6
S31508016DA0F7F7BAFD96F999251346394603A81AF055
S31508016DB07BFD03A8F1F730FF02AB024603A94BA8F6
S31508016DC0F7F7AAFDC14F97F948201346294603A8A4
S31508016DD01AF06AFD03A8F1F71FFF02AB024603A9E1
S31508016DE04BA8F7F799FD96F99A251346294603A85C
S31508016DF01AF05AFD03A8F1F70FFF02AB024603A9E1
S31508016E004BA8F7F789FD96F99B251346294603A84A
S31508016E101AF04AFD03A8F1F7FFFE02AB024603A9E1
S31508016E204BA8F7F779FD96F99C251346294603A839
S31508016E301AF03AFD03A8F1F7EFFE02AB024603A9E1
S31508016E404BA8F7F769FD96F99D251346294603A828
S31508016E501AF02AFD03A8F1F7DFFE02AB024603A9E1
S31508016E604BA8F7F759FD96F99E251346294603A817
S31508016E701AF01AFD03A8F1F7CFFE02AB024603A9E1
S31508016E804BA8F7F749FD96F99F251346294603A806
S31508016E901AF00AFD03A8F1F7BFFE02AB024603A9E1
S31508016EA04BA8F7F739FD96F9A0251346294603A8F5
S31508016EB01AF0FAFC03A8F1F7AFFE02AB024603A9E2
S31508016EC04BA8F7F729FD96F9A1251346294603A8E4
S31508016ED01AF0EAFC03A8F1F79FFE02AB024603A9E2
S31508016EE04BA8F7F719FD96F9A2251346294603A8D3
S31508016EF01AF0DAFC03A8F1F78FFE02AB024603A9E2
S31508016F004BA8F7F709FD96F9A3251346294603A8C1
S31508016F101AF0CAFC03A8F1F77FFE02AB024603A9E1
S31508016F204BA8F7F7F9FC96F9A4251346294603A8B1
S31508016F301AF0BAFC03A8F1F76FFE02AB024603A9E1
S31508016F404BA8F7F7E9FC96F9A5251346294603A8A0
S31508016F501AF0AAFC03A8F1F75FFE02AB024603A9E1
S31508016F604BA8F7F7D9FC96F9A6251346294603A88F
S31508016F701AF09AFC03A8F1F74FFE02AB024603A9E1
S31508016F804BA8F7F7C9FC96F9A7251346294603A87E
S31508016F901AF08AFC03A8F1F73FFE02AB024603A9E1
S31508016FA04BA8F7F7B9FC96F9A8251346294603A86D
S31508016FB01AF07AFC03A8F1F72FFE02AB024603A9E1
S31508016FC04BA8F7F7A9FC96F9A9251346294603A85C
S31508016FD01AF06AFC03A8F1F71FFE02AB024603A9E1
S31508016FE04BA8F7F799FC96F9AA251346294603A84B
S31508016FF01AF05AFC03A8F1F70FFE02AB024603A9E1
S315080170004BA8F7F789FCB6F8AC25314E134631463D
S3150801701003A81AF049FC03A8F1F7FEFD02AB0246E4
S3150801702003A94BA8F7F778FC94F9AE251346294628
S3150801703003A81AF039FC03A8F1F7EEFD02AB0246E4
S3150801704003A94BA8F7F768FCD4F8C8351A462946A8
S3150801705003A81AF029FC03A8F1F7DEFD02AB0246E4
S3150801706003A94BA8F7F758FCD4F8D8351A46294688
S3150801707003A81AF019FC03A8F1F7CEFD02AB0246E4
S3150801708003A94BA8F7F748FCD4F8D0351A46314678
S3150801709003A81AF009FC03A8F1F7BEFD02AB0246E4
S315080170A003A94BA8F7F738FCD4F8D4351A46314664
S315080170B003A81AF0F9FB03A8F1F7AEFD02AB0246E5
S315080170C003A94BA8F7F728FC04E000BF98000020A5
S315080170D024BC030897F849201346314603A81AF039
S315080170E0E3FB03A8F1F798FD02AB024603A94BA8F7
S315080170F0F7F712FCD4F8D8351A46314603A81AF020
S31508017100D3FB03A8F1F788FD02AB024603A94BA8F6
S31508017110F7F702FCD4F8DC351A46314603A81AF00B
S31508017120C3FB03A8F1F778FD02AB024603A94BA8F6
S31508017130F7F7F2FBD4F8E0351A46294603A81AF000
S31508017140B3FB03A8F1F768FD02AB024603A94BA8F6
S31508017150F7F7E2FBD4F8E4351A46294603A81AF0EC
S31508017160A3FB03A8F1F758FD02AB024603A94BA8F6
S31508017170F7F7D2FBD4F8E8351A46294603A81AF0D8
S3150801718093FB03A8F1F748FD02AB024603A94BA8F6
S31508017190F7F7C2FBD4F8EC351A46294603A81AF0C4
S315080171A083FB03A8F1F738FD02AB024603A94BA8F6
S315080171B0F7F7B2FBD4F8F0351A46294603A81AF0B0
S315080171C073FB03A8F1F728FD02AB024603A94BA8F6
S315080171D0F7F7A2FBB7F94A201346294603A81AF07E
S315080171E063FB03A8F1F718FD02AB024603A94BA8F6
S315080171F0F7F792FB94F9F4251346294603A81AF0E2
S3150801720053FB03A8F1F708FD02AB024603A94BA8F5
S31508017210F7F782FB97F94C201346294603A81AF07B
S3150801722043FB03A8F1F7F8FC02AB024603A94BA8F6
S31508017230F7F772FB94F9F5251346294603A81AF0C0
S3150801724033FB03A8F1F7E8FC02AB024603A94BA8F6
S31508017250F7F762FB94F9F6251346294603A81AF0AF
S3150801726023FB03A8F1F7D8FC02AB024603A94BA8F6
S31508017270F7F752FB94F9F7251346294603A81AF09E
S3150801728013FB03A8F1F7C8FC02AB024603A94BA8F6
S31508017290F7F742FB97F94D201346294603A81AF03A
S315080172A003FB03A8F1F7B8FC02AB024603A94BA8F6
S315080172B0F7F732FB94F9F8251346294603A81AF07D
S315080172C0F3FA03A8F1F7A8FC02AB024603A94BA8F7
S315080172D0F7F722FB94F9F9251346294603A81AF06C
S315080172E0E3FA03A8F1F798FC02AB024603A94BA8F7
S315080172F0F7F712FB97F94E201346294603A81AF009
S31508017300D3FA03A8F1F788FC02AB024603A94BA8F6
S31508017310F7F702FB97F84F20C14E1346314603A8EB
S315080173201AF0C2FA03A8F1F777FC02AB024603A9E1
S315080173304BA8F7F7F1FA94F8FA251346314603A84C
S315080173401AF0B2FA03A8F1F767FC02AB024603A9E1
S315080173504BA8F7F7E1FA94F8FB251346314603A83B
S315080173601AF0A2FA03A8F1F757FC02AB024603A9E1
S315080173704BA8F7F7D1FAD4F8FC351A46294603A8DB
S315080173801AF092FA03A8F1F747FC02AB024603A9E1
S315080173904BA8F7F7C1FA94F800261346314603A815
S315080173A01AF082FA03A8F1F737FC02AB024603A9E1
S315080173B04BA8F7F7B1FA94F801261346294603A80C
S315080173C01AF072FA03A8F1F727FC02AB024603A9E1
S315080173D04BA8F7F7A1FA94F802261346294603A8FB
S315080173E01AF062FA03A8F1F717FC02AB024603A9E1
S315080173F04BA8F7F791FA94F803261346294603A8EA
S315080174001AF052FA03A8F1F707FC02AB024603A9E0
S315080174104BA8F7F781FA94F804261346294603A8D8
S315080174201AF042FA03A8F1F7F7FB02AB024603A9E1
S315080174304BA8F7F771FA94F805261346294603A8C7
S315080174401AF032FA03A8F1F7E7FB02AB024603A9E1
S315080174504BA8F7F761FA94F806261346294603A8B6
S315080174601AF022FA03A8F1F7D7FB02AB024603A9E1
S315080174704BA8F7F751FA94F807261346294603A8A5
S315080174801AF012FA03A8F1F7C7FB02AB024603A9E1
S315080174904BA8F7F741FA94F808261346294603A894
S315080174A01AF002FA03A8F1F7B7FB02AB024603A9E1
S315080174B04BA8F7F731FA94F809261346314603A87B
S315080174C01AF0F2F903A8F1F7A7FB02AB024603A9E2
S315080174D04BA8F7F721FA94F80A261346294603A872
S315080174E01AF0E2F903A8F1F797FB02AB024603A9E2
S315080174F04BA8F7F711FA94F80B261346294603A861
S315080175001AF0D2F903A8F1F787FB02AB024603A9E1
S315080175104BA8F7F701FA94F80C261346314603A847
S315080175201AF0C2F903A8F1F777FB02AB024603A9E1
S315080175304BA8F7F7F1F9D4F810361A46314603A8DD
S315080175401AF0B2F903A8F1F767FB02AB024603A9E1
S315080175504BA8F7F7E1F9D4F814361A46314603A8C9
S315080175601AF0A2F903A8F1F757FB02AB024603A9E1
S315080175704BA8F7F7D1F994F818261346294603A814
S315080175801AF092F903A8F1F747FB02AB024603A9E1
S315080175904BA8F7F7C1F9D4F82C361A46294603A899
S315080175A01AF082F903A8F1F737FB02AB024603A9E1
S315080175B04BA8F7F7B1F9D4F83C361A46294603A879
S315080175C01AF072F903A8F1F727FB02AB024603A9E1
S315080175D04BA8F7F7A1F994F83C261346314603A8B8
S315080175E01AF062F903A8F1F717FB02AB024603A9E1
S315080175F04BA8F7F791F994F83D261346314603A8A7
S315080176001AF052F903A8F1F707FB02AB024603A9E0
S315080176104BA8F7F781F994F93E261346294601E066
S3150801762024BC030803A81AF03FF903A8F1F7F4FAF2
S3150801763002AB024603A94BA8F7F76EF9D4F8403610
S315080176401A46294603A81AF02FF903A8F1F7E4FA0E
S3150801765002AB024603A94BA8F7F75EF9D4F844260C
S31508017660D4F84436294603A81AF01EF903A8F1F7F7
S31508017670D3FA02AB024603A94BA8F7F74DF9D4F89A
S315080176804826D4F84836294603A81AF00DF903A85E
S31508017690F1F7C2FA02AB024603A94BA8F7F73CF980
S315080176A094F84C261346314603A81AF0FDF803A8A8
S315080176B0F1F7B2FA02AB024603A94BA8F7F72CF980
S315080176C0B4F85C261346314603A81AF0EDF803A868
S315080176D0F1F7A2FA02AB024603A94BA8F7F71CF980
S315080176E094F85C261346314603A81AF0DDF803A878
S315080176F0F1F792FA02AB024603A94BA8F7F70CF980
S31508017700D4F870361A46294603A81AF0CDF803A804
S31508017710F1F782FA02AB024603A94BA8F7F7FCF880
S3150801772094F870261346294603A81AF0BDF803A84B
S31508017730F1F772FA02AB024603A94BA8F7F7ECF880
S3150801774094F871261346294603A81AF0ADF803A83A
S31508017750F1F762FA02AB024603A94BA8F7F7DCF880
S3150801776094F872261346294603A81AF09DF803A829
S31508017770F1F752FA02AB024603A94BA8F7F7CCF880
S3150801778094F873261346294603A81AF08DF803A818
S31508017790F1F742FA02AB024603A94BA8F7F7BCF880
S315080177A094F874261346294603A81AF07DF803A807
S315080177B0F1F732FA02AB024603A94BA8F7F7ACF880
S315080177C094F875261346294603A81AF06DF803A8F6
S315080177D0F1F722FA02AB024603A94BA8F7F79CF880
S315080177E094F876261346294603A81AF05DF803A8E5
S315080177F0F1F712FA02AB024603A94BA8F7F78CF880
S31508017800D4F878361A46314603A81AF04DF803A873
S31508017810F1F702FA02AB024603A94BA8F7F77CF87F
S31508017820D4F87C261346314603A81AF03DF803A876
S31508017830F1F7F2F902AB024603A94BA8F7F76CF880
S315080178403E46B7F950202C461346294603A81AF096
S315080178502BF803A8F1F7E0F902AB024603A94BA8F6
S31508017860F7F75AF8BD4D95F88026BD4F13463946A8
S3150801787003A81AF019F803A8F1F7CEF902AB0246E4
S3150801788003A94BA8F7F748F895F981261346214627
S3150801789003A81AF009F803A8F1F7BEF902AB0246E4
S315080178A003A94BA8F7F738F8B5F8822613463946DF
S315080178B003A819F0F9FF03A8F1F7AEF902AB0246DE
S315080178C003A94BA8F7F728F8D5F884361A46394696
S315080178D003A819F0E9FF03A8F1F79EF902AB0246DE
S315080178E003A94BA8F7F718F8706DF0F7F5FD0246EE
S315080178F00B469C4903A819F0D7FF03A8F1F78CF9A1
S3150801790002AB024603A94BA8F7F706F8B36D1A4668
S31508017910214603A819F0C8FF03A8F1F77DF902ABC0
S31508017920024603A94BA8F6F7F7FFB5F988261346C9
S31508017930214603A819F0B8FF03A8F1F76DF902ABC0
S31508017940024603A94BA8F6F7E7FFB5F98A261346B7
S31508017950214603A819F0A8FF03A8F1F75DF902ABC0
S31508017960024603A94BA8F6F7D7FFF36D1A46214637
S3150801797003A819F099FF03A8F1F74EF902AB0246DD
S3150801798003A94BA8F6F7C8FFD5F88C361A46394627
S3150801799003A819F089FF03A8F1F73EF902AB0246DD
S315080179A003A94BA8F6F7B8FFD5F890361A4621462B
S315080179B003A819F079FF03A8F1F72EF902AB0246DD
S315080179C003A94BA8F6F7A8FFD5F894361A46214617
S315080179D003A819F069FF03A8F1F71EF902AB0246DD
S315080179E003A94BA8F6F798FF336E1A46214603A852
S315080179F019F05AFF03A8F1F70FF902AB024603A9DA
S31508017A004BA8F6F789FF2B6C1A46214603A819F0ED
S31508017A104BFF03A8F1F700F902AB024603A94BA8ED
S31508017A20F6F77AFF736E1A46214603A819F03CFF4A
S31508017A3003A8F1F7F1F802AB024603A94BA8F6F73A
S31508017A406BFFB6F868201346394603A819F02CFFD0
S31508017A5003A8F1F7E1F802AB024603A94BA8F6F72A
S31508017A605BFFF36E1A46214603A819F01DFF03A80A
S31508017A70F1F7D2F802AB024603A94BA8F6F74CFF79
S31508017A80B6F970201346214603A819F00DFF03A87D
S31508017A90F1F7C2F802AB024603A94BA8F6F73CFF79
S31508017AA0B5F998261346214603A819F0FDFE03A841
S31508017AB0F1F7B2F802AB024603A94BA8F6F72CFF79
S31508017AC0B5F99A261346214603A819F0EDFE03A82F
S31508017AD0F1F7A2F802AB024603A94BA8F6F71CFF79
S31508017AE0D5F8EC361A46214603A819F0DDFE03A897
S31508017AF0F1F792F802AB024603A94BA8F6F70CFF79
S31508017B00B6F97C201346214603A819F0CDFE03A831
S31508017B10F1F782F802AB024603A94BA8F6F7FCFE79
S31508017B20B6F984201346214603A819F0BDFE03A819
S31508017B30F1F772F802AB024603A94BA8F6F7ECFE79
S31508017B4095F9E0261346214603A819F0ADFE03A8C8
S31508017B50F1F762F802AB024603A905E0101200200C
S31508017B6024BC03083CBC03084BA8F6F7D5FEB6F8B7
S31508017B7084201346394603A819F096FE03A8F1F79F
S31508017B804BF802AB024603A94BA8F6F7C5FEB6F8B1
S31508017B9098201346394603A819F086FE03A8F1F77B
S31508017BA03BF802AB024603A94BA8F6F7B5FE96F9D0
S31508017BB098201346214603A819F076FE03A8F1F783
S31508017BC02BF802AB024603A94BA8F6F7A5FEB6F8B1
S31508017BD0BC201346394603A819F066FE03A8F1F737
S31508017BE01BF802AB024603A94BA8F6F795FE96F9D0
S31508017BF0BC201346214603A819F056FE03A8F1F73F
S31508017C000BF802AB024603A94BA8F6F785FEB6F8B0
S31508017C10BE201346394603A819F046FE03A8F0F715
S31508017C20FBFF02AB024603A94BA8F6F775FED6F889
S31508017C30C0301A46214603A819F036FE03A8F0F704
S31508017C40EBFF02AB024603A94BA8F6F765FE8A4A83
S31508017C504BF21043D2581346214603A819F024FEC5
S31508017C6003A8F0F7D9FF02AB024603A94BA8F6F71A
S31508017C7053FED5F8E8361A46394603A819F014FE14
S31508017C8003A8F0F7C9FF02AB024603A94BA8F6F70A
S31508017C9043FE95F8E8261346394603A819F004FE6B
S31508017CA003A8F0F7B9FF02AB024603A94BA8F6F7FA
S31508017CB033FED5F8EC361A46394603A819F0F4FD11
S31508017CC003A8F0F7A9FF02AB024603A94BA8F6F7EA
S31508017CD023FED5F8F0361A46394603A819F0E4FD0D
S31508017CE003A8F0F799FF02AB024603A94BA8F6F7DA
S31508017CF013FED5F8F4361A46394603A819F0D4FD09
S31508017D0003A8F0F789FF02AB024603A94BA8F6F7C9
S31508017D1003FED5F8F8361A46394603A819F0C4FD04
S31508017D2003A8F0F779FF02AB024603A94BA8F6F7B9
S31508017D30F3FD95F8FC261346214603A819F0B4FD70
S31508017D4003A8F0F769FF02AB024603A94BA8F6F7A9
S31508017D50E3FDD5F800371A46394603A819F0A4FDFC
S31508017D6003A8F0F759FF02AB024603A94BA8F6F799
S31508017D70D3FDD5F804371A46214603A819F094FD10
S31508017D8003A8F0F749FF02AB024603A94BA8F6F789
S31508017D90C3FDD5F808371A46214603A819F084FD0C
S31508017DA003A8F0F739FF02AB024603A94BA8F6F779
S31508017DB0B3FDD5F8AC271346214603A819F074FD7F
S31508017DC003A8F0F729FF02AB024603A94BA8F6F769
S31508017DD0A3FD96F9C4201346214603A819F064FDAC
S31508017DE003A8F0F719FF02AB024603A94BA8F6F759
S31508017DF093FD96F9C5201346214603A819F054FDAB
S31508017E0003A8F0F709FF02AB024603A94BA8F6F748
S31508017E1083FDB5F8B2271346394603A819F044FD80
S31508017E2003A8F0F7F9FE02AB024603A94BA8F6F739
S31508017E3073FD95F8B2271346394603A819F034FDA0
S31508017E4003A8F0F7E9FE02AB024603A94BA8F6F729
S31508017E5063FD4BA8F6F7D7FE0446AB8F01332946D7
S31508017E6021F83C3F02220520FDF7CCFBB4FA84F049
S31508017E704009FEF76CB900BF8C24002010B5144CDC
S31508017E8004F2B4711348F7F71DFB0122124904F5F0
S31508017E90F760F6F7E7FBC0B10D2804D00F48F7F7EE
S31508017EA035FB002010BD0022114604F2B470F6F726
S31508017EB0DFFF0028F2D10122074904F5F760F6F73A
S31508017EC0D1FB0028EAD10120ECE70120EAE700BF4F
S31508017ED0101200205041030840BC0308C4190020B1
S31508017EE010B504460649F6F7A7FE08B9012010BDE4
S31508017EF02046F6F7CFFEB0FA80F04009F7E700BF53
S31508017F00FC1B002030B597B005460C464D220021D2
S31508017F100DF10A0019F0C4FB52238DF8083011231C
S31508017F208DF8093080238DF80A30FF238DF80C303F
S31508017F3063788DF80F3023788DF81030A3788DF893
S31508017F401130E3788DF8123023798DF8133063797F
S31508017F508DF81430A3798DF815300023E371A989BA
S31508017F60A868EB7D0193AB7D00934F2302AAF1F735
S31508017F703BFE17B030BD30B597B005460C464D22CD
S31508017F8000210DF10A0019F08BFB52238DF80830F8
S31508017F9011238DF8093080238DF80A30FF238DF8D7
S31508017FA00C3063788DF80F3023788DF81030A3786C
S31508017FB08DF81130E3788DF8123023798DF8133066
S31508017FC063798DF81430A3798DF815300023E371A0
S31508017FD035F8201C55F8240C15F8153C019315F8AD
S31508017FE0163C00934F2302AAF1F7FEFD17B030BDE8
S31508017FF008B52C30F2F71EFE08BD10B47F2380F8B1
S31508018000303080F8313080F8323080F83330416BC7
S315080180106FF317014163C26E6FF31702C26600233D
S3150801802080F8373080F8383090F8524044F08004B0
S3150801803080F8524090F8564044F0800480F8564043
S3150801804090F85B4044F0800480F85B4090F85F400C
S3150801805044F0800480F85F4090F8644044F080045E
S3150801806080F8644090F8684044F0800480F86840DD
S31508018070082464F3030180F83410114664F30301FC
S3150801808080F86C10C2F3076263F3030280F86F206D
S3150801809080F87A3080F8733080F8723080F876305C
S315080180A080F8753080F8743080F8783080F8773049
S315080180B080F879305DF8044B704710B584B00446F2
S315080180C07F2380F8303080F8313080F8323080F8FC
S315080180D03330416B6FF317014163C26E6FF31702B9
S315080180E0C266002380F8373080F8383090F852009D
S315080180F040F0800084F8520094F8560040F0800061
S3150801810084F8560094F85B0040F0800084F85B0020
S3150801811094F85F0040F0800084F85F0094F86400EA
S3150801812040F0800084F8640094F8680040F080000C
S3150801813084F86800082060F3030184F834101146B6
S3150801814060F3030184F86C10C2F3076263F3030258
S3150801815084F86F2084F87A3084F8733084F87230A2
S3150801816084F8763084F8753084F8743084F8783079
S3150801817084F8773084F8793043238DF80C3002235C
S315080181808DF80D30A189E27D0192A27D009203AAA4
S31508018190A068F1F729FD636813B1984704B010BDCB
S315080181A0002384F8743084F87530142384F8763003
S315080181B0012384F87930F1E738B54FF4C0612048D6
S315080181C0F8F7C4F81720F7F723FD2820F7F720FD5D
S315080181D01C4C04F60C252846FBF7E4FC2846FBF75D
S315080181E05DFB3A20F7F738FD3A20F7F711FD3A20FB
S315080181F0F7F702FD144BC4F80C3A4FF4E133C4F80F
S31508018200103A0023C4F8143AC4F8183AC4F81C3AC8
S315080182100C22C4F8202AC4F8243AC4F8283A284675
S31508018220FBF70DFB58B90748D0F80C3A5B680122F1
S3150801823000F1C40100F60C20FBF768FC38BDFEE727
S3150801824000000240101200200010014070B586B0EF
S31508018250574B93F9A43553B1012B32D0022B73D066
S31508018260032B74D0042B00F09F8006B070BD514AD1
S31508018270536C23F0100353644F4C4FF4C0612046EE
S31508018280F8F764F82520F7F7C3FC4FF4C0630193A8
S315080182904A4B02930123039301A92046F7F778FF76
S315080182A0002206211720F7F775FC1720F7F7A4FC1B
S315080182B0002207212820F7F76DFC2820F7F79CFCF8
S315080182C0D3E74FF4C0613C48F8F740F81720F7F7B1
S315080182D09FFC2820F7F79CFC354C04F60C2528460C
S315080182E0FBF760FC2846FBF7D9FA3A20F7F7B4FC06
S315080182F03A20F7F78DFC3A20F7F77EFC304BC4F8A5
S315080183000C3A4FF46143C4F8103A0023C4F8143AFE
S31508018310C4F8183AC4F81C3A0C22C4F8202AC4F83E
S31508018320243AC4F8283A2846FBF789FA58B9204866
S31508018330D0F80C3A5B68012200F1C40100F60C2062
S31508018340FBF7E4FB91E7FEE7FFF736FF8DE7194AEE
S31508018350536C23F010035364174D4FF4C06128463C
S31508018360F7F7F4FF1720F7F753FC2820F7F750FC27
S315080183704FF4806601960123029300240394049422
S3150801838001A92846F7F704FF4FF4007301930294F5
S315080183900394049401A92846F7F7FAFE22463146C2
S315080183A02846F8F771F860E7FFF706FF5DE700BFB3
S315080183B0101200200038024000000240000031106F
S315080183C00010014000B5ADB0002101913D4B1A6C7A
S315080183D042F080521A641B6C03F080530193019B8F
S315080183E00291394B1A6842F440421A601B6803F439
S315080183F040430293029B05231F9301232093219354
S31508018400022325934FF480022692102227924FF4D5
S31508018410B4722892299308222A922B931FA8F9F756
S3150801842051F9002849D1F8F791FC002846D10F23C4
S315080184301A9302231B9300231C934FF4A0531D93F5
S315080184404FF480531E9305211AA8F8F71DFD00283D
S3150801845035D14FF448730393102309934FF4C0732E
S315080184600A9302230C9308230B9301230E934FF4CB
S31508018470807313934FF0006318930023149303A892
S31508018480F8F708FEE0B900224FF480011046F8F724
S31508018490ADFCF8F7C9FD0D4BA3FB00308009F7F7D2
S315080184A0C5FB0420F7F7E6FB002211464FF0FF3023
S315080184B0F7F770FB2DB05DF804FBFEE7FEE7FEE774
S315080184C0FEE700BF0038024000700040D34D62103D
S315080184D0F8B51D4CB4F87C1A04F64C274900384601
S315080184E0FDF74FF9B4F8C01A04F529664900304674
S315080184F0FDF747F9B4F8040BEFF7DCFF0022134B3D
S31508018500F0F742F8F0F718FB04F6D4250146284699
S31508018510FDF737F9B4F8481B04F618344900204624
S31508018520FDF72FF900213846FDF700F900213046FD
S31508018530FDF7FCF800212846FDF7F8F8002120464A
S31508018540FDF7F4F8F8BD00BF101200200000F83F4F
S315080185502DE9F04389B0002406948DF81C402123A7
S315080185608DF8183004948DF814406F238DF8103067
S31508018570324D334EA046DFF8CC9009F65C370CE055
S31508018580304A82F84E1AC2F8503A09B0BDE8F0836B
S3150801859089F8921AC9F8943A0134424669883046EC
S315080185A0F7F772FF4FF47A73052206A93846FAF7E8
S315080185B077FB012235F8021F3046F7F765FF424679
S315080185C029883046F7F760FF4FF47A73009305233D
S315080185D002AA04A93846FAF733FC0122298830464B
S315080185E0F7F752FF9DF808109DF809209DF80A3003
S315080185F01B0443EA02639DF80C2013439DF80B20E4
S3150801860043EA0223032C15D801A252F824F000BF2D
S315080186102B860108218601089185010881850108B3
S3150801862089F8D61AC9F8D83AB6E789F81A1BC9F8E3
S315080186301C3BB1E7631C032BAEDDA6E79E000020B9
S31508018640000C0240101200202DE9F04389B00023E6
S3150801865006938DF81C3022228DF8182004938DF884
S3150801866014306F238DF81030394C04F10808394D50
S315080186700027394E3A4621882846F7F705FF4FF471
S315080186807A73052206A93046FAF70AFB012234F85D
S31508018690021B2846F7F7F8FE4445EBD12F4D002477
S315080186A02C4EA1462E4F07F65C380CE02C4A82F870
S315080186B04E1AC2F85C3A09B0BDE8F08387F8921AF7
S315080186C0C7F8A03A01344A4635F8021F3046F7F78B
S315080186D0DBFE4FF47A730093052302AA04A94046E8
S315080186E0FAF7AEFB012229883046F7F7CDFE9DF849
S315080186F008109DF809209DF80A301B0443EA026315
S315080187009DF80C2013439DF80B2043EA0223B3F589
S31508018710000FC8BF03F17F43032C15D801A252F8F5
S3150801872024F000BF3F87010835870108BD86010887
S31508018730AD86010887F8D61AC7F8E43AC2E787F87A
S315080187401A1BC7F8283BBDE7631C032BBADDB2E742
S31508018750A0000020000C02406C1D00209E00002095
S315080187601012002070B5FFF76FFF4FF400717C48B7
S31508018770F7F784FE002875D17A4B5E6876424FF486
S3150801878000517748F7F77AFE00287BD1754B5E686A
S315080187904FF480417248F7F771FE002840F0838054
S315080187A0704B5C684FF400616D48F7F767FE002867
S315080187B040F08A806B4B5C6864426B4B93F9743565
S315080187C0012B00F0B380684B93F97535012B08BF6F
S315080187D00024664D4FF47A712846FCF7D2FF86EAE3
S315080187E0E671A1EBE6712846FCF7A0FF002E00F022
S315080187F0AC80002E0ADD5C4BD3F8601AD3F8643AD4
S315080188009942D8BF19465948FCF780FF002E0CDA61
S31508018810554BD3F8602AD3F8641A8A42CEBF03F6B9
S315080188204C2011465148FCF771FF514D4FF47A71AE
S315080188302846FCF7A6FF84EAE471A1EBE471284611
S31508018840FCF774FF002C50D0002C57DD464BD3F8AB
S31508018850A41AD3F8A83A9942D8BF19464448FCF74E
S3150801886055FF70BD4FF480713D48F7F707FE0028A4
S3150801887082D080213A48F7F701FE00283FF47CAF01
S3150801888000267CE74FF480513548F7F7F7FD0028B5
S315080188903FF47CAF4FF400613148F7F7EFFD00284C
S315080188A07FF476AF72E74FF400512D48F7F7E6FDEE
S315080188B000283FF475AF80212948F7F7DFFD002826
S315080188C03FF46EAF00246DE74FF480612448F7F753
S315080188D0D5FD00283FF46EAF4FF400712048F7F735
S315080188E0CDFD00287FF469AF64E74FF4FA612846A5
S315080188F0FCF747FF00212846FCF718FF1A4BD3F867
S31508018900A41AD3F8A83A9942C8BF19461848FCF7D9
S31508018910FDFEA6E7154C4FF47A712046FCF731FFA8
S3150801892000212046FCF702FF00240EE00E4B93F9C6
S315080189307535012BEED00D4D4FF47A712846FCF7AB
S3150801894020FF00212846FCF7F1FE084D4FF4FA6195
S315080189502846FCF716FF00212846FCF7E7FE64E7E0
S315080189600010024098000020101200205C1C002014
S31508018970A01C002070B5FFF767FE4FF40071884808
S31508018980F7F77CFD002840F08480864BD3F8085B16
S315080189906D424FF400518248F7F770FD002840F008
S315080189A08980804BD3F8085B4FF480417C48F7F700
S315080189B065FD002840F08F807A4BD3F84C4B4FF475
S315080189C000617748F7F75AFD002840F09580754B06
S315080189D0D3F84C4B6442734B93F97635012B00F06F
